:100000000C9404080C9423080C9423080C942308E3
:100010000C9423080C9423080C942E0A0C94640A64
:100020000C9423080C9423080C9423080C942308A4
:100030000C9423080C9423080C9423080C94D10DE1
:100040000C9423080C9423080C9423080C94230884
:100050000C9448520C946A490C9423080C9423087D
:100060000C9423080C943F4A0C9423080C94334AB4
:100070000C9423080C9423080C9423080C94230854
:100080000C94C05D0C9423080C9423080C94230852
:100090000C947D4A0C9423080C94714A0C94230808
:1000A0000C9423080C9423080C9423080C94230824
:1000B0000C9423080C9423080C9423080C94230814
:1000C0000C9423080C9423080C9423080C94230804
:1000D0000C9423080C9423080C9423080C942308F4
:1000E0000C9423080C9401520C940B520C94F7516D
:1000F0000C94B1510C943C520C942D520C942152FE
:100100000C9415520C9423080C9423080C94230887
:100110000C9423080C9423080C9423080C942308B3
:1001200007634236B79BD8A71A39685618AEBAABE0
:10013000558C1D3CB7CC5763BD6DEDFD753EF61774
:100140007231BF000000803F08000000BE922449C9
:10015000123EABAAAA2ABECDCCCC4C3E00000080F9
:10016000BEABAAAAAA3E00000000BF000000803F6C
:100170000000000000084178D3BB4387D1133D192C
:100180000E3CC3BD4282AD2B3E68EC8276BED98F59
:10019000E1A93E4C80EFFFBE01C4FF7F3F0000009D
:1001A00000000A0025303278002025362E326620E5
:1001B0004F6E2D426F61726400202573002530322E
:1001C00078002025362E326620002025730048490D
:1001D00048363133302000424D5030383520004110
:1001E00044584C3334352000484D4338383533209B
:1001F000004C3347343230304420004E48444330C2
:100200003231362000756E6B6E6F776E20636D64D1
:100210000A002563006820202020202020202020A4
:1002200020202020202020202020202020202020CE
:10023000202D2068656C700A0D007620202020207B
:1002400020202020202020202020202020202020AE
:100250002020202020202D2076657273696F6E0A81
:100260000D0075202020202020202020202020206C
:1002700020202020202020202020202020202D2071
:10028000757074696D650A0D00616573205B6F6E32
:100290007C6F66665D2020202020202020202020EA
:1002A00020202020202D20696E7465677265747986
:1002B0000A0D0061646320202020202020202020BF
:1002C0002020202020202020202020202020202D21
:1002D0002073686F7720765F696E2C2061312C2047
:1002E000613220766F6C74616765730A0D0063611B
:1002F0006C69205B5B765F696E7C61317C61325D2D
:1003000020766F6C747C72657365747C6E6F6E653D
:100310005D202D2063616C6962726174650A0D0055
:100320006465205B6D61736B5D20202020202020A0
:100330002020202020202020202020202D20646527
:100340006275670A0D0068756D202020202020202E
:10035000202020202020202020202020202020209D
:1003600020202D2068756D69646974792073656E2D
:10037000736F720A0D0068756D70205B6F6E7C6F15
:1003800066665D20202020202020202020202020A4
:1003900020202D2068756D696469747920706572FC
:1003A0006D2073656E736F72207077720A0D00692D
:1003B00064205B72657365745D20202020202020FE
:1003C00020202020202020202020202D2069642093
:1003D00068616E646C696E670A0D006D637520203C
:1003E000202020202020202020202020202020200D
:1003F000202020202020202D206D637520696E662E
:100400006F0A0D00657272202020202020202020FD
:1004100020202020202020202020202020202020DC
:100420002D206572726F7220696E666F0A0D006E04
:1004300065205B666C7573685D202020202020207D
:1004400020202020202020202020202D206E6569C3
:100450006768626F72207461626C650A0D006C6F70
:1004600067205B6175746F7C6F6E7C6F66665D2064
:10047000202020202020202020202D206D6F74653A
:10048000732064617461206F6E205553420A0D0021
:100490006F772020202020202020202020202020B6
:1004A0002020202020202020202020202D206F6EA2
:1004B000652D776972652073656E736F72730A0DAF
:1004C000007265205B6D61736B5D20202020202011
:1004D000202020202020202020202020202D206DC2
:1004E0006F7465207265706F7274207365747469BF
:1004F0006E670A0D007269205B696E745D202020B2
:1005000020202020202020202020202020202020EB
:10051000202D207265706F727420696E746572761A
:10052000616C0A0D007273202020202020202020E2
:1005300020202020202020202020202020202020BB
:10054000202D20726164696F2073746174730A0DC9
:100550000073732020202020202020202020202015
:10056000202020202020202020202020202D20732B
:10057000797374656D2073756D6D6172790A0D0004
:1005800074787077205B302D31355D20202020205D
:100590002020202020202020202020202D205458E2
:1005A000205077720A0D0070777231205B6F6E7C7D
:1005B0006F66665D20202020202020202020202023
:1005C0002020202D2070696E31207077720A0D0076
:1005D0007031205B6F6E7C6F66665D20202020206E
:1005E0002020202020202020202020202D20646971
:1005F0007361626C652070756C7365207031207456
:100600006F207361766520706F7765720A0D0072D6
:1006100065737420656570726F6D20202020202026
:1006200020202020202020202020202D20726573D3
:10063000746F726520656570726F6D0A0D0070775A
:100640007273205B646565707C666F7263655F6959
:10065000646C655D2020202020202D206D63752096
:10066000736C656570206D6F64650A0D00626F6F55
:100670007420202020202020202020202020202026
:100680002020202020202020202D207265626F6FE6
:10069000740A0D0075706772202020202020202011
:1006A000202020202020202020202020202020204A
:1006B0002D207265626F6F742076696120626F6FA2
:1006C000746C6F616465720A0D0074657374205BED
:1006D0006F66667C317C327C335D202020202020B8
:1006E0002020202020202D2074657374206D6F64DD
:1006F00065730A0D00557074696D6520256420646A
:100700006179732C20253032643A253032643A25E1
:100710003032640A00204E657665722D757365640B
:1007200020737461636B203E2025642062797465B8
:10073000730A0025352E3266200025372E336620B9
:1007400025372E3366002530327800525F49442029
:1007500000525F542000525F54312000525F545FBA
:100760004D43552000525F565F4D43552000525F68
:1007700050302000525F50305F542000525F5031A3
:100780002000525F50315F542000525F5550544951
:100790004D452000525F52482000525F565F494E3F
:1007A0002000525F41312000525F41322000525FF1
:1007B000502000525F50412000525F49443D0909DA
:1007C0003078257800525F543D090930782578004B
:1007D000525F54313D09093078257800525F545FEB
:1007E0004D43553D093078257800525F565F4D43A3
:1007F000553D093078257800525F50303D09093069
:1008000078257800525F50305F543D0909307825D3
:100810007800525F50313D09093078257800525FE9
:1008200050315F543D09093078257800525F5550AA
:1008300054494D453D093078257800525F52483D76
:1008400009093078257800525F565F494E3D090905
:100850003078257800525F41313D0909307825789C
:1008600000525F41323D09093078257800525F50CF
:100870003D09093078257800525F50413D09093023
:100880007825780025730A004E65772064656275C7
:10089000673D307825580A0043757272656E742082
:1008A00064656275673D307825580A00445F4F5093
:1008B00045523D307825780A00445F52583D3078E3
:1008C00025780A00445F54583D307825780A004462
:1008D0005F504B543D6E307825780A00445F4F5787
:1008E0003D307825780A00445F4C45443D307825FA
:1008F000780A00445F504F5745523D307825780ABA
:1009000000445F4556454E543D307825780A0044F2
:100910005F50305F4C45443D307825780A00445F95
:1009200050315F4C45443D307825780A00445F41A2
:1009300045533D307825780A00445F5057525F3167
:100940003D307825780A00445F505245533D307859
:1009500025780A00445F414343454C3D3078257873
:100960000A00445F434F4D504153533D3078257842
:100970000A00256300256300256300545820506F4A
:100980007765723D25640A004F4B0A0025630074A9
:1009900078206C656E20202020207268206D69739D
:1009A00073202020207268207374616C65202020E1
:1009B0007268206D6973630A00252D31306C7520D3
:1009C000252D31306C7520252D31306C7520252D6D
:1009D00031306C75200A002563004D43553D2530AC
:1009E000366C780020467573653A2065653D253084
:1009F00032782068663D25303278206C663D25309F
:100A00003278206C623D2530327800204F534343CA
:100A1000414C3D25642000256300256300256300CB
:100A20002563004E6577207265706F72743D307873
:100A3000255820005573696E67207265706F727457
:100A40003D3078255820002563004E65772072657B
:100A5000706F727420696E74657276616C3D252DBD
:100A600064207365630A0043757272656E74207248
:100A700065706F727420696E74657276616C3D2565
:100A80002D64207365630A00256300256300537994
:100A90007374656D2053756D6D6172790A004944F8
:100AA0003D004932433A2000545820506F77657218
:100AB0003D25640A004E65696768626F7220746143
:100AC000626C652073697A653D25640A0052494D60
:100AD0004520616464723D252D642E252D640A0035
:100AE0005265706F727420496E74657276616C3DE8
:100AF000252D640A005265706F7274204D61736B0E
:100B00003D3078252D782000565F494E3D252D3506
:100B10002E32660A00565F4D43553D252D352E3247
:100B2000660A005553425F5057523D25730A0049EB
:100B30006E74722E20546F74616C3A2050303D25D3
:100B40002D6C642050313D252D6C640A00496E7473
:100B5000722E205365633A20202050303D252D37DA
:100B60002E33662050313D252D372E33660A004C3A
:100B70006F67206D6F64653D006175746F0A0025B5
:100B8000730A0048554D5F5057525F414C574159C9
:100B9000533D25730A00496E7075742050313D2510
:100BA000730A0044656275673D3078252D780A0028
:100BB000507772313D25730A00256300256300528A
:100BC000483D252D342E31662000545F52483D2586
:100BD0002D342E31662000256300256C64204320CF
:100BE00000256C642050612020252D372E32662090
:100BF0006D002563005854414C5F5452494D3D25CA
:100C000064004572726F72203020566F6C7400451C
:100C100072726F72203020566F6C74004E6F7420A9
:100C2000737570706F727465640A004572726F72CA
:100C3000203020566F6C740025352E32662000253A
:100C4000372E33662025372E33660025730A00546D
:100C500065737420312025730A0054657374203243
:100C60002025730A005465737420332025730A000D
:100C70005465737420342025730A0025730A0025F7
:100C8000730A0025730A0025730A00256300256393
:100C900000503A20256C642050612020252D372EED
:100CA0003266206D0A00532025642E256420636C73
:100CB0006F636B20256C7520747820256C7520720D
:100CC0007820256C752072747820256C75207272DE
:100CD0007820256C75207265786D697420256C7597
:100CE0002061636B747820256C75206E6F61636B77
:100CF000747820256C752061636B727820256C7583
:100D00002074696D65646F757420256C752062614F
:100D10006461636B727820256C7520746F6F6C6FE3
:100D20006E6720256C7520746F6F73686F72742006
:100D3000256C752062616473796E636820256C751B
:100D40002062616463726320256C7520636F6E742A
:100D5000656E74696F6E64726F7020256C75207398
:100D6000656E64696E6764726F7020256C75206CA7
:100D70006C747820256C75206C6C727820256C75ED
:100D80000A00452025642E256420636C6F636B2068
:100D9000256C752063707520256C75206C706D2036
:100DA000256C752069727120256C7520676C6564EF
:100DB00020256C7520796C656420256C7520726C1B
:100DC000656420256C7520747820256C75206C690D
:100DD0007374656E20256C752073656E736F727306
:100DE00020256C752073657269616C20256C750A0D
:100DF000000A2A2A2A2A2A2A2A426F6F74696E67F1
:100E00002025732A2A2A2A2A2A2A0A0052616E6475
:100E10006F6D204555493634206164647265737383
:100E20002067656E6572617465640A004D414320F8
:100E300061646472657373200025783A000A0025A6
:100E4000732025732C206368616E6E656C20257598
:100E500020706F776572202575002C2063686563AC
:100E60006B207261746520257520487A000A004F56
:100E70006E6C696E650A00257325730A006C6F63DA
:100E8000616C686F73740041544D4547413132388D
:100E90007266613100020000FFFE0000014545500E
:100EA000524F4D20697320636F72727570742C20DD
:100EB000726577726974696E6720776974682064F7
:100EC000656661756C74732E0A006E616E00696EE2
:100ED000660000407A10F35A00A0724E1809001004
:100EE000A5D4E80000E87648170000E40B5402009F
:100EF00000CA9A3B000000E1F505000080969800CA
:100F0000000040420F000000A086010000001027F2
:100F100000000000E8030000000064000000000082
:100F20000A00000000000100000000002C76D888B4
:100F3000DC674F0823DFC1DFAE59E1B1B796E5E3C7
:100F4000E453C63AE651997696E8E6C28426EB89E0
:100F50008C9B62ED407C6FFCEFBC9C9F40F2BAA57D
:100F60006FA5F490055A2AF75C936B6CF9676DC115
:100F70001BFCE0E40D47FEF520E6B500D0ED902E19
:100F80000300943577050080841E080000204E0A77
:100F9000000000C80C333333330F986E12831141B5
:100FA000EF8D2114893BE65516CFFEE6DB18D18480
:100FB0004B381BF77C1D901DA4BBE42420328472A7
:100FC0005E228100C9F124ECA1E53D27494E464946
:100FD0004E4954594E414E000020410000C8420085
:100FE000401C4620BCBE4CCA1B0E5AAEC59D74CDDB
:100FF000CCCC3D0AD7233C17B7D13877CC2B3295D0
:1010000095E6241FB14F0A0011241FBECFEFD1E493
:10101000DEBFCDBF16E0A0E0B2E0EEE6F2EF00E00A
:101020000BBF02C007900D92A239B107D9F71DE29C
:10103000A2E9B6E001C01D92AB33B107E1F70E940F
:10104000E86A0C9435790C940000E0916017F0E0A8
:10105000EF71F070EB54F84E8083809160178F5FD2
:10106000809360178091752488608093752443EC89
:1010700054E0CA0161E10E941E3A80E090E00895C8
:101080004F925F926F927F928F929F92AF92BF9298
:10109000CF92DF92EF92FF920F931F93CF93DF9344
:1010A000CDB7DEB760970FB6F894DEBF0FBECDBFE9
:1010B0004B01809198069091990681FD74980E9449
:1010C000AA403C018EE996E00E941A3B0AC0C80182
:1010D0000296B4010E94F5370097F1F4C8010E940E
:1010E000C03B8C01009799F725C1C8010296B40155
:1010F0000E94EC37D3018C918150F801808780E009
:1011000091E0A0E0B0E081879287A387B4878EE961
:1011100096E0B8010E94893BC8010D9660E074E634
:101120004AEB59E098010E94AB3D84E00E94CE4119
:10113000D80115969C938E93149783E00E94CE411C
:101140002C01F80197838683D301CC908085C81A3F
:10115000DD24EE24FF2486E0CC0CDD1CEE1CFF1CFD
:101160008A95D1F7618572858385948520EC30E07E
:1011700040E050E00E943572DC01CB01892F9A2FAC
:10118000AB2FBB27C80ED91EEA1EFB1EF801C18675
:10119000D286E386F486D3018C918087809198066D
:1011A0009091990681FD08C08091E40480FD04C0FF
:1011B00081FFB8C01D9BB6C0EDB7FEB772970FB6E2
:1011C000F894FEBF0FBEEDBFADB6BEB60894A11C2D
:1011D000B11C80E092E092838183C3010196D50126
:1011E00013969C938E931297F401808114968C939E
:1011F000149715961C921597818116968C931697C5
:1012000017961C92D3018C91F50180871186D80125
:1012100014968D919C911597938782875586448665
:10122000BB27AF2D9E2D8D2D97878687C701B601D1
:1012300024E630E040E050E00E943572672F782FBE
:10124000892F99270E947B72DC01CB01F501918BDC
:10125000808B0E942676209100058DB79EB742961E
:101260000FB6F8949EBF0FBE8DBF2223A9F000D009
:1012700000D0EDB7FEB731968EE89CE0ADB7BEB7B3
:1012800012969C938E931197228313820E94387634
:101290000F900F900F900F908091FE1B85FF42C022
:1012A0000E945346C30104960E941446EDB7FEB750
:1012B0003C970FB6F894FEBF0FBEEDBF31966E019E
:1012C0000894C11CD11CADB7BEB71296DC92CE9269
:1012D000119780E190E0938382838CE392E0958381
:1012E0008483D80114968D919C911597978386835A
:1012F00016968D919C91179791878087D3018C9139
:10130000828713860E948D76EDB7FEB73C960FB6A6
:10131000F894FEBF0FBEEDBF82E00E942F46C601CB
:101320000E941446809198069091990681FF0BC007
:10133000749A09C081E195E00E94A73A8C01009758
:1013400009F0D3CEEFCF60960FB6F894DEBF0FBE94
:10135000CDBFDF91CF911F910F91FF90EF90DF9064
:10136000CF90BF90AF909F908F907F906F905F9045
:101370004F900895CF93DF93EC0180919806909160
:10138000990687FF2EC08DB79EB70C970FB6F894BD
:101390009EBF0FBE8DBFEDB7FEB731968FE492E0D2
:1013A000ADB7BEB712969C938E9311978A818283B4
:1013B00013828B81848315828885868317828C8132
:1013C0009D81918780878E819F81938782870E94EC
:1013D00026768DB79EB70C960FB6F8949EBF0FBEBB
:1013E0008DBF8EE996E0BE010E94543B81E195E0FD
:1013F000BE010E94D23ADF91CF91089587EE93E02B
:101400008115910511F00197F1F70895882369F08E
:101410006D987598ED9A80916A00886080936A0053
:10142000809168008160809368008091E4049091CD
:10143000E50491FF10C06E988EB18F6B8EB9EE9A55
:1014400080916A00806280936A0080916800816068
:10145000809368000895769AEE9808951F920F92EF
:101460000FB60F9211248F939F93AF93BF938091E8
:10147000680080FF20C08091552490915624A0914F
:101480005724B09158240196A11DB11D8093552475
:1014900090935624A0935724B09358248091980693
:1014A0009091990690FF07C0749882E090E0909325
:1014B0000E0580930D05BF91AF919F918F910F9075
:1014C0000FBE0F901F9018951F920F920FB60F929C
:1014D00011248F939F93AF93BF938091680080FFF7
:1014E00020C08091592490915A24A0915B24B091FE
:1014F0005C240196A11DB11D8093592490935A2418
:10150000A0935B24B0935C248091980690919906F7
:1015100091FF07C0739882E090E090930E0580934E
:101520000D05BF91AF919F918F910F900FBE0F90BE
:101530001F90189580937C0080917B00877F80931B
:101540007B0080917C00806C80937C0085E08093A0
:101550007A0080917A00806880937A0080917B0085
:1015600087FFFCCF80917B0085FFFCCF80917A00C4
:10157000806480937A0080917A0086FDFCCF10927F
:1015800079001092780084E090E060E070E02091B3
:101590007A00206420937A0020917A0026FDFCCF07
:1015A0002091780030917900620F731F019779F7CD
:1015B00010927C0080917A008F7780937A007695E4
:1015C00067957695679580E090E00E94BB6F462F07
:1015D000572F682F792FCB01BA01089580E00E9420
:1015E0009A0A2091090530910A0540910B05509106
:1015F0000C050E946D7021EE3AE744E95EE30E941B
:10160000EB6E462F572F682F792FCB01BA01089523
:1016100080E180935101809351019091510195FF98
:1016200003C08F5F8F31B9F76BE4869FB00111243F
:10163000882777FD8095982F0E94BD6F20E030E6C7
:101640004FE954E40E94EB6E462F572F682F792FF5
:10165000CB01BA0120E030E04AE754E40E94536F26
:10166000462F572F682F792FCB01BA01089580910B
:10167000E80483FF4DC080917B00886080937B00ED
:1016800089EC80937C0085E080937A0080917A00D9
:10169000806880937A0080917B0087FFFCCF8091E7
:1016A0007B0085FFFCCF80917A00806480937A0074
:1016B00080917A0086FDFCCF80917A0080648093CF
:1016C0007A0080917A0086FDFCCF6091780070915D
:1016D000790080E090E00E94BB6F27ED33EA40E99B
:1016E0005FE30E946D7026E636E648E853E40E9408
:1016F000EA6EDC01CB018093551790935617A093A7
:101700005717B093581780917A008F7780937A009B
:101710000895CF92DF92EF92FF921F93CF93DF93C2
:10172000CDB7DEB729970FB6F894DEBF0FBECDBF99
:101730006C01109292068FEF8983A1E7EA2EA7E150
:10174000FA2E10E03FC0183009F440C0CE010196D7
:10175000BE016E5F7F4F0E94914389818F3F11F0E0
:101760008E3F19F48093920631C0CE010296C114C7
:10177000D10479F40E94AA4380937224DE01129668
:10178000EAE6F4E288E09D9191938150E1F711E05F
:101790001DC00E94AA43F7018083DE01129620E05B
:1017A00030E0C70108974D91FC01E20FF31F408321
:1017B0002F5F3F4F28303105B1F71F5F89E090E080
:1017C000E80EF91E8981882309F0BDCF812F299663
:1017D0000FB6F894DEBF0FBECDBFDF91CF911F9142
:1017E000FF90EF90DF90CF90089500D082EA91E0D3
:1017F000EDB7FEB7928381830E9438760F900F90E9
:1018000008952F923F924F925F926F927F928F92A4
:101810009F92AF92BF92CF92DF92EF92FF920F937F
:101820001F93CF93DF9300D000D0CDB7DEB78C01EC
:10183000009741F489E290E06BE270E04AE250E008
:1018400027E00AC08130910549F489E290E06BE21B
:1018500070E04AE250E026E00E946642C8010E9421
:10186000890B63E9862E66E0962E800E911ED401C8
:101870008C930115110599F021E7A22E27E1B22ED4
:1018800000E010E03DEB632E31E0732E42EC442E7D
:1018900041E0542E5AEC252E51E0352E10C18AE637
:1018A00094E20E94CD44FC01BF01882777FD80951A
:1018B000982F0E94BD6FF82EE92E0AE614E2AA24A2
:1018C000BB2494EAC92E91E0D92ED8018D918D01C7
:1018D00000D000D0EDB7FEB73196ADB7BEB71296C7
:1018E000DC92CE921197828313826B837C830E9459
:1018F00038760894A11CB11C0F900F900F900F9098
:101900006B817C81B8E0AB16B104F9F600D000D051
:1019100000D00DB71EB70F5F1F4F89EA91E0EDB7FA
:10192000FEB7928381839701862F972FA32FBE2D19
:10193000BC01CD0120E030E048EC52E40E94536F3E
:10194000DC01CB01F80182839383A483B5830E94D9
:1019500038762DB73EB72A5F3F4F0FB6F8943EBF9B
:101960000FBE2DBF80917224882319F08EE792E07C
:1019700002C087E892E000D000D029EB31E0ADB79B
:10198000BEB712963C932E93119714969C938E9308
:1019900013970E9438760F900F900F900F900E942F
:1019A000F50B94C0C801B3E0880F991FBA95E1F711
:1019B000800F911F8759984E0E94CD44FC01BF01B2
:1019C000882777FD8095982F0E94BD6F6C0120E0DD
:1019D00030E088EFE82E8FEFF82EEA0CFB1C00D0E9
:1019E00000D0ADB7BEB71196EDB7FEB77282618277
:1019F000F701E20FF31F808112968C9312971396D2
:101A00001C9229833A836B837C830E9438762981D8
:101A10003A812F5F3F4F0F900F900F900F906B8187
:101A20007C8128303105D9F600D000D000D0EDB649
:101A3000FEB60894E11CF11CADB7BEB712965C92DD
:101A40004E921197862F972FAC2DBD2DBC01CD0145
:101A500020E030E048EC52E40E94536FDC01CB01FF
:101A6000F70182839383A483B5830E9438762DB7D0
:101A70003EB72A5F3F4F0FB6F8943EBF0FBE2DBF53
:101A8000D5018C91882319F08EE792E002C087E897
:101A900092E000D000D0EDB7FEB73282218294836D
:101AA00083830E9438760F900F900F900F900E94C2
:101AB000F50B0F5F1F4F29E030E0A20EB31ED401DB
:101AC0008C9190E0081719070CF46CCF0F900F90D1
:101AD0000F900F90DF91CF911F910F91FF90EF909A
:101AE000DF90CF90BF90AF909F908F907F906F903E
:101AF0005F904F903F902F900895CF93DF9300D049
:101B0000CDB7DEB780916B248983809171248A835D
:101B1000CE0101960E9407380F900F90DF91CF9170
:101B20000895CF93DF93EC0180916A248F3FB1F544
:101B300080916B248F3F91F580916C248F3F71F5DC
:101B400080916D248F3F51F580916E248F3F31F548
:101B500080916F248F3F11F5809170248F3FF1F4B5
:101B6000809171248F3FD1F489E290E06BE270E0C4
:101B70004AE250E027E00E94664280E090E00E9446
:101B8000890BCD56D94F88838AE694E260E070E0F5
:101B900049E050E00E947E770E947D0DDF91CF9159
:101BA00008951F920F920FB60F920BB60F92112449
:101BB0002F933F934F935F936F937F938F939F9355
:101BC000AF93BF93EF93FF938091752482608093CE
:101BD00075248091E40486FD2B9A87FD2B9A8091D1
:101BE0000D0590910E051816190614F4749A739A3F
:101BF000809198069091990685FF02C07498739819
:101C000080910F0590911005019790931005809396
:101C10000F05009709F068C080919C0690919D0681
:101C20009C012F5F3F4F30939D0620939C0640916F
:101C300000205091012060910220709103204F5F9D
:101C40005F4F6F4F7F4F4093002050930120609370
:101C500002207093032020E130E0309310052093A0
:101C60000F052091E40420FD02C01D9B05C01092C9
:101C700096061092950606C021E030E03093960655
:101C8000209395062091E6043091E7042115310553
:101C9000A1F00296B9010E945472009771F47798EE
:101CA000809198069091990693FF07C0749884E0FC
:101CB00090E090930E0580930D052115310581F07C
:101CC00080919C0690919D06B9010E9454720097E4
:101CD00039F48BEA94E062E140E050E00E941E3A61
:101CE0008091E40486FD2B9885E395E060E040E078
:101CF00050E00E941E3AFF91EF91BF91AF919F91EA
:101D00008F917F916F915F914F913F912F910F90A4
:101D10000BBE0F900FBE0F901F901895809160170B
:101D200090911420891B08950E948E0E882379F0CB
:101D3000E0911420F0E0EF71F070EB54F84E8081E8
:101D400090E0209114202F5F2093142008958FEFAE
:101D50009FEF0895CF93DF93EC0110929B061092B2
:101D60009A0688819981009731F022E0873B92079B
:101D700009F0B7C009C00E948E0E882341F487EB9A
:101D800092E099838883B1C0613109F0AEC0F894C4
:101D900078940E94940E90E09093A6068093A506F6
:101DA0008D3009F47CC08F3F31F38231910569F1A8
:101DB0008F37910521F08830910509F053C080914B
:101DC000A7069091A806181619060CF060C060913D
:101DD000352D7091362D88E090E00E94FA75609163
:101DE000352D7091362D80E290E00E94FA75609159
:101DF000352D7091362D88E090E00E94FA75809123
:101E0000A7069091A80601973EC06091352D70916C
:101E1000362D8DE090E00E94FA751092AA0610927D
:101E2000A90614C08B5E9F4DFC0180816091352D09
:101E30007091362D90E00E94FA758091A9069091DC
:101E4000AA0601969093AA068093A9068091A906F6
:101E50009091AA062091A7063091A80682179307B1
:101E60000CF315C06091352D7091362D0E94FA75D6
:101E70008091A7069091A8062091A506FC01EB5E33
:101E8000FF4D208301969093A8068093A70680912A
:101E9000A7069091A8068F33910509F06CCF109298
:101EA0001420109260178091A7069091A806FC015B
:101EB000EB5EFF4D108290939B0680939A061092E2
:101EC000A8061092A706809173249091742400971D
:101ED00009F451CF6091A30640E050E00E941E3A01
:101EE0004ACF1982188283E001C081E0DF91CF914F
:101EF000089578948091950690919606009731F018
:101F00008091E4049091E50490FF03C083B7817F42
:101F100003C083B7817F866083BFF89483B78160F5
:101F200083BF7894889583B78E7F83BF7894089514
:101F3000CF93DF93EC0188819981009721F029E00C
:101F40008A39920789F40E94790F8091490E909105
:101F50004A0E65E840E050E00E941E3A8AE999E0A6
:101F60009983888381E003C01982188283E0DF911E
:101F7000CF910895CF93DF938EE40E944B45882341
:101F8000B1F40E949A458091FE1B9091FF1B8160E5
:101F90009093FF1B8093FE1B00D08EEC91E0EDB779
:101FA000FEB7928381830E9438760F900F908EEE59
:101FB0000E944B458823B1F40E949A458091FE1BF4
:101FC0009091FF1B82609093FF1B8093FE1B00D0BB
:101FD00087ED91E0EDB7FEB7928381830E9438765A
:101FE0000F900F9086EA0E944B458823B1F40E941F
:101FF0009A458091FE1B9091FF1B84609093FF1B7C
:102000008093FE1B00D08FED91E0EDB7FEB7928379
:1020100081830E9438760F900F908CE30E944B458D
:102020008823B1F40E949A458091FE1B9091FF1B7A
:1020300088609093FF1B8093FE1B00D088EE91E098
:10204000EDB7FEB7928381830E9438760F900F9090
:1020500082ED0E944B458823B1F40E949A458091FD
:10206000FE1B9091FF1B80619093FF1B8093FE1BD2
:1020700000D081EF91E0EDB7FEB7928381830E949B
:1020800038760F900F90C7E0D0E08CE70E944B4568
:102090008823B9F40E949A458091FE1B9091FF1B02
:1020A00080629093FF1B8093FE1B00D08BEF91E02A
:1020B000EDB7FEB7928381830E9438760F900F9020
:1020C00002C0219711F70E94F50BDF91CF9108957F
:1020D000CF93DF9300D0CDB7DEB74A8369830E94E8
:1020E00070456981862F0E94A2454A81842F0E94F3
:1020F000A2450E949A450F900F90DF91CF910895CD
:10210000AF92BF92DF92EF92FF920F931F93CF9304
:10211000DF9300D00F92CDB7DEB7082FD22E4A83BF
:102120005B8369830E9470456981862F0E94A24566
:10213000802F81600E9497454A81042F5B81152F73
:10214000EE24FF24AD2CBB240894A108B1080FC0D5
:10215000EA14FB0419F40E94BD4502C00E94B34575
:10216000F80180830894E11CF11C0F5F1F4FED14F0
:1021700078F30E949A450F900F900F90DF91CF91C6
:102180001F910F91FF90EF90DF90BF90AF90089557
:10219000CF93DF9300D0CDB7DEB71A8219828EEECF
:1021A0006AEAAE014F5F5F4F22E00E9480103981E2
:1021B00020E08A8190E0822B932B9093D617809316
:1021C000D5178EEE6CEAAE014F5F5F4F22E00E94A2
:1021D0008010398120E08A8190E0822B932B9093AC
:1021E000D8178093D7178EEE6EEAAE014F5F5F4F20
:1021F00022E00E948010398120E08A8190E0822BC9
:10220000932B9093DA178093D9178EEE60EBAE0183
:102210004F5F5F4F22E00E948010398120E08A8169
:1022200090E0822B932B9093E8178093E7178EEE24
:1022300062EBAE014F5F5F4F22E00E948010398158
:1022400020E08A8190E0822B932B9093EA17809371
:10225000E9178EEE64EBAE014F5F5F4F22E00E9404
:102260008010398120E08A8190E0822B932B90931B
:10227000EC178093EB178EEE66EBAE014F5F5F4F6E
:1022800022E00E948010398120E08A8190E0822B38
:10229000932B9093DC178093DB178EEE68EBAE01E7
:1022A0004F5F5F4F22E00E948010398120E08A81D9
:1022B00090E0822B932B9093DE178093DD178EEEA8
:1022C0006AEBAE014F5F5F4F22E00E9480103981C0
:1022D00020E08A8190E0822B932B9093E2178093E9
:1022E000E1178EEE6CEBAE014F5F5F4F22E00E9474
:1022F0008010398120E08A8190E0822B932B90938B
:10230000E4178093E3178EEE6EEBAE014F5F5F4FE5
:1023100022E00E948010398120E08A8190E0822BA7
:10232000932B9093E6178093E5170F900F90DF9112
:10233000CF9108952F923F924F925F926F927F922A
:102340008F929F92AF92BF92CF92DF92EF92FF92C5
:102350000F931F93CF93DF93CDB7DEB76C970FB674
:10236000F894DEBF0FBECDBF882E4A8F2B8FFE01A3
:10237000319683E0DF011D928A95E9F78091F91784
:10238000882339F46C8F0E94C81081E08093F9177C
:102390006C8D662309F478C08EEE64EF4EE20E94E5
:1023A000681069E07AE180E090E00E9438458EEEA6
:1023B00066EFAE014F5F5F4F22E00E94801089817F
:1023C00090E0A0E0B0E0BA2FA92F982F88274A818B
:1023D00050E060E070E0842B952BA62BB72B20916A
:1023E000EB173091EC17A90160E070E0841B950BAE
:1023F000A60BB70B2091E9173091EA1740E050E0A7
:10240000BC01CD010E9435726B017C01AFE0F594F7
:10241000E794D794C794AA95D1F76091E317709188
:10242000E417882777FD8095982FBBE0660F771F0C
:10243000881F991FBA95D1F72091E5173091E617BB
:10244000442737FD4095542F2C0D3D1D4E1D5F1D1B
:102450000E949D722C0D3D1D3093E0172093DF17D5
:10246000285F3F4F14E0359527951A95E1F76901EC
:10247000EE24D7FCE094FE2CC092ED17D092EE171C
:10248000E092EF17F092F017082D0295000F000F61
:10249000007C0C5C282D30E0398F288F63E070E0E1
:1024A000082C02C0660F771F0A94E2F7882777FD91
:1024B0008095982F25E335E040E050E00E9435728A
:1024C000DC01CB010296A11DB11D888B998BAA8BD3
:1024D000BB8B20E533EC40E050E004C055954795B8
:1024E000379527958A94D2F72C8B3D8B4E8B5F8B3B
:1024F00010E01C861D861E861F86E8E02E2E312CDD
:10250000488D598D241A350A73C18EEE64EF402F21
:102510000E946810688979898A899B890E94384558
:102520008EEE66EFAE014F5F5F4F23E00E9480109A
:102530008091DF179091E017805A9F409C014427BB
:1025400037FD4095542F2C833D834E835F83CA0112
:10255000B9010E9435722B013C016091D91770912D
:10256000DA17882777FD8095982F0E9435726B01C6
:102570007C01BDE0F594E794D794C794BA95D1F760
:102580006091DB177091DC17882777FD8095982F75
:10259000A3019201ECE05595479537952795EA956B
:1025A000D1F70E943572DC01CB01CD01BB2797FD2D
:1025B000B095AB2FC80ED91EEA1EFB1E82E090E03C
:1025C000A0E0B0E0C80ED91EEA1EFB1EE2E0F594C2
:1025D000E794D794C794EA95D1F720E030E840E03B
:1025E00050E0C20ED31EE41EF51E2091E717309175
:1025F000E81740E050E0C701B6010E943572DC01E7
:10260000CB01FFE0B695A79597958795FA95D1F7F9
:1026100088879987AA87BB8789809924AA24BB24A5
:102620005401992488248A8190E0A0E0B0E0BA2F78
:10263000A92F982F8827882A992AAA2ABB2A8B8112
:1026400090E0A0E0B0E0882A992AAA2ABB2A022CAE
:1026500004C0B594A794979487940A94D2F7C09035
:10266000D517D090D617EE24D7FCE094FE2CE2E0EC
:10267000CC0CDD1CEE1CFF1CEA95D1F76091DD1738
:102680007091DE17882777FD8095982FA30192011E
:102690000E9435722B013C01F7E1759467945794C1
:1026A0004794FA95D1F76091D7177091D81788277A
:1026B00077FD8095982F2C813D814E815F810E940E
:1026C0003572DC01CB01EBE0B595A7959795879521
:1026D000EA95D1F7480E591E6A1E7B1EC40CD51C04
:1026E000E61CF71C088C04C0CC0CDD1CEE1CFF1C87
:1026F0000A94D2F722E030E040E050E0C20ED31E50
:10270000E41EF51EF2E0F594E794D794C794FA9589
:10271000D1F78C189D08AE08BF08C501B4012C89FB
:102720003D894E895F890E94357297FD0DC0660F05
:10273000771F881F991F288539854A855B850E94E8
:102740007B7249015A010CC0288539854A855B8511
:102750000E947B7249015A01880C991CAA1CBB1C5F
:102760005527B7FC5A954B2D3A2D292DCA01B90191
:102770000E9435722EED3BE040E050E00E94357241
:102780006C01FF24D7FCF094EF2CC501B40123E4C5
:1027900033EE4FEF5FEF0E943572DC01CB01CD01CC
:1027A000BB2797FDB095AB2FC80ED91EEA1EFB1EA6
:1027B0008FEC9EE0A0E0B0E0C80ED91EEA1EFB1E22
:1027C000E4E0F594E794D794C794EA95D1F7C80C60
:1027D000D91CEA1CFB1C2C853D854E855F852C0D84
:1027E0003D1D4E1D5F1D2C873D874E875F871F5FF8
:1027F0003A8D131709F089CE112391F0212F30E083
:1028000040E050E06C857D858E859F850E947B72BF
:102810002093F1173093F2174093F3175093F41766
:102820004B8D4423E9F16091F1177091F21780917B
:10283000F3179091F417611571058105910581F1E8
:102840000E94BD6F20E836EE45EC57E40E94536FBE
:1028500021E03EED42E45EE30E94D070B62FA72F48
:10286000382F292F60E070E080E89FE3FD01A90187
:102870000F2F1E2F252F342FA90198010E94EA6ED9
:102880002BE43AE34DEB57E30E94536FDC01CB019D
:102890008093F5179093F617A093F717B093F81756
:1028A0006C960FB6F894DEBF0FBECDBFDF91CF910F
:1028B0001F910F91FF90EF90DF90CF90BF90AF905E
:1028C0009F908F907F906F905F904F903F902F9050
:1028D0000895CF93DF9300D000D000D0CDB7DEB7FE
:1028E000FE01319686E0DF011D928A95E9F780911D
:1028F0005F17882399F486EA61E340E00E9468103C
:1029000086EA6CE24AE00E94681081E080935F17DB
:102910006CE77EE380E090E00E94384586EA6DE255
:1029200048E00E9468106CE77EE380E090E00E943F
:10293000384586EA62E3AE014F5F5F4F26E00E94B2
:10294000801086EA6DE247E00E9468109A8180E07C
:10295000698170E0682B792B70935A17609359172F
:102960009C8180E04B8150E0482B592B50935C17A1
:1029700040935B173E8120E08D8190E0822B932B6A
:1029800090935E1780935D172DB73EB72850304067
:102990000FB6F8943EBF0FBE2DBFEDB7FEB7319610
:1029A00028E832E0ADB7BEB712963C932E9311974C
:1029B0007383628355834483978386830E9426763C
:1029C0002DB73EB7285F3F4F0FB6F8943EBF0FBEFE
:1029D0002DBF26960FB6F894DEBF0FBECDBFDF9198
:1029E000CF9108950F931F93CF93DF9300D000D022
:1029F00000D0CDB7DEB78E010F5F1F4F86E0D80144
:102A00001D928A95E9F78CE362E041E00E9468102C
:102A10008CE360E048E50E94681062E174E380E0C6
:102A200090E00E9438458CE363E0A80126E00E9414
:102A300080108CE362E043E00E946810998180E09E
:102A40006A8170E0682B792B7093401760933F1771
:102A50009B8180E04C8150E0482B592B50934217CA
:102A6000409341173D8120E08E8190E0822B932B93
:102A70009093441780934317EDB7FEB738970FB67E
:102A8000F894FEBF0FBEEDBF319626E932E0ADB738
:102A9000BEB712963C932E9311977383628355832E
:102AA0004483978386830E942676EDB7FEB73896D7
:102AB0000FB6F894FEBF0FBEEDBF26960FB6F89482
:102AC000DEBF0FBECDBFDF91CF911F910F91089553
:102AD000CF93DF93EC0188819981009731F029E051
:102AE0008438920709F071C00BC08FEB96E060E864
:102AF00070E00E94B23C84E899E09983888369C0C1
:102B00008FEB96E00E94DD3C009709F462C0809153
:102B100098069091990694FF3FC08091FE1B81FF1B
:102B20003BC083E061E048E021E00E949A118DB74C
:102B30009EB70A970FB6F8949EBF0FBE8DBFEDB734
:102B4000FEB7319681E99CE0ADB7BEB712969C9373
:102B50008E9311978091F1179091F217A091F3172E
:102B6000B091F41782839383A483B5838091F51782
:102B70009091F617A091F717B091F8178683978375
:102B8000A087B1870E9438768DB79EB70A960FB698
:102B9000F8949EBF0FBE8DBF8091980690919906C4
:102BA00095FF06C08091FE1B82FF02C00E9469143F
:102BB000809198069091990696FF97CF8091FE1B81
:102BC00083FF93CF0E94F21490CF1982188283E082
:102BD00001C081E0DF91CF910895FF920F931F9381
:102BE000CF93DF93729A8091E40483FD06C0C0E521
:102BF000D0E00E94FE092197E1F78EE40E944B4548
:102C0000882309F08BC0C0E5D0E00E94FE0921971F
:102C1000E1F78FE40E944B450E94B345C82F82958F
:102C20008695869583708130A9F440910820509153
:102C3000092060910A2070910B204F5F5F4F6F4F0A
:102C40007F4F409308205093092060930A2070938F
:102C50000B2016C08230A0F040910C2050910D2026
:102C600060910E2070910F204F5F5F4F6F4F7F4F2D
:102C700040930C2050930D2060930E2070930F20F2
:102C80000E94B3451C2F1F7300E0080F111D0E9406
:102C9000B345F82E0E94BD45DF2D90E0C92FC80F27
:102CA000D11DD695C795D695C7950E949A45809116
:102CB000E40483FF7298B80180E090E00E94BB6F4B
:102CC00020E134E048EC5BE30E946D70DC01CB0155
:102CD0008093FA179093FB17A093FC17B093FD17FE
:102CE000BE0180E090E00E94BB6F24EA3CEF44E22A
:102CF0005CE30E946D7020E030E040E252E40E940C
:102D0000EA6EDC01CB018093762490937724A09324
:102D10007824B093792480E090E015C0809104205D
:102D200090910520A0910620B09107200196A11D49
:102D3000B11D8093042090930520A0930620B093AA
:102D4000072081E090E0DF91CF911F910F91FF90DC
:102D500008957298729A8EE40E944B4580EA0E9410
:102D6000A24580E00E94A24580E00E94A2458FE437
:102D70000E944B450E94B345829586958695837047
:102D80008130A9F4409108205091092060910A20D7
:102D900070910B204F5F5F4F6F4F7F4F4093082024
:102DA0005093092060930A2070930B2016C0823044
:102DB000A0F040910C2050910D2060910E20709158
:102DC0000F204F5F5F4F6F4F7F4F40930C2050930A
:102DD0000D2060930E2070930F2000D000D0EDB72F
:102DE000FEB7319624EA32E0ADB7BEB712963C93F7
:102DF0002E931197828313820E9426760F900F9054
:102E00000F900F908EE40E944B4580E80E94A245EF
:102E100080E00E94A24580E00E94A2450E949A455F
:102E200080E090E0089500D085E092E0ADB7BEB7B5
:102E300012969C938E9311970E94387620910005EC
:102E40000F900F902223A9F000D000D0EDB7FEB76D
:102E5000319682E192E0ADB7BEB712969C938E9305
:102E60001197228313820E9438760F900F900F9053
:102E70000F90089500D085E192E0EDB7FEB7928300
:102E800081830E9438768AE392E0EDB7FEB79283A1
:102E900081830E94387682E692E0EDB7FEB7928396
:102EA00081830E94387689E892E0EDB7FEB792837D
:102EB00081830E94387683EB92E0EDB7FEB7928370
:102EC00081830E9438768EEE92E0EDB7FEB7928352
:102ED00081830E94387680E293E0EDB7FEB792835B
:102EE00081830E94387686E493E0EDB7FEB7928343
:102EF00081830E94387686E793E0EDB7FEB7928330
:102F000081830E9438768FEA93E0EDB7FEB7928313
:102F100081830E9438768BED93E0EDB7FEB7928304
:102F200081830E94387684E094E0EDB7FEB7928307
:102F300081830E9438768FE294E0EDB7FEB79283EA
:102F400081830E9438768EE594E0EDB7FEB79283D8
:102F500081830E94387680E994E0EDB7FEB79283D2
:102F600081830E94387681EC94E0EDB7FEB79283BE
:102F700081830E94387685EF94E0EDB7FEB79283A7
:102F800081830E94387685E295E0EDB7FEB79283A3
:102F900081830E94387681E595E0EDB7FEB7928394
:102FA00081830E94387680E895E0EDB7FEB7928382
:102FB00081830E94387687EA95E0EDB7FEB7928369
:102FC00081830E94387680ED95E0EDB7FEB792835D
:102FD00081830E9438768FE096E0EDB7FEB792834A
:102FE00081830E9438768EE396E0EDB7FEB7928338
:102FF00081830E9438768DE696E0EDB7FEB7928326
:1030000081830E94387684E996E0EDB7FEB792831B
:1030100081830E9438768AEC96E0EDB7FEB7928302
:1030200081830E9438760F900F90089584EB92E090
:103030000E945F7608954F925F926F927F928F9277
:103040009F92AF92BF92CF92DF92EF92FF920F9337
:103050001F93CF93DF9300D000D0CDB7DEB7609140
:103060000020709101208091022090910320809097
:10307000002090900120A0900220B090032040906A
:103080000020509001206090022070900320209139
:10309000002030910120409102205091032029838B
:1030A0003A834B835C834DB75EB74A5050400FB6AE
:1030B000F8945EBF0FBE4DBF0DB71EB70F5F1F4F19
:1030C00025EF36E0EDB7FEB732832183A0E8CA2EA4
:1030D000A1E5DA2EA1E0EA2EF12CA70196010E94CB
:1030E0007B72F80133832283C501B401A7019601E5
:1030F0000E947B72B0E1CB2EBEE0DB2EE12CF12CE6
:10310000A70196010E947B72332727FD3095F801B5
:1031100035832483C301B201A70196010E947B720B
:103120002CE3C22ED12CE12CF12CA70196010E9498
:103130007B72332727FD3095F80137832683698119
:103140007A818B819C81A70196010E947B727727EF
:1031500067FD7095F801718760870E9438762DB7FA
:103160003EB7265F3F4F0FB6F8943EBF0FBE2DBF50
:103170000F900F900F900F90DF91CF911F910F91B3
:10318000FF90EF90DF90CF90BF90AF909F908F9087
:103190007F906F905F904F900895EBE3FDE2808108
:1031A000918122E482349207B9F000D000D085E109
:1031B00097E0ADB7BEB712969C938E931197EB53E1
:1031C000FD421496FC93EE9313970E9438760F906D
:1031D0000F900F900F9008953A96B1E4E53FFB07EA
:1031E000F0F20895EF92FF920F931F93CF93DF9326
:1031F0000E94EE0ADC01CB0100D000D000D023E316
:1032000037E0EDB7FEB73283218383839483A583B0
:10321000B6830E9438768DB79EB706960FB6F8949F
:103220009EBF0FBE8DBF81E00E949A0A20910505C6
:103230003091060540910705509108050E946D7078
:103240008B01D82FC92F82E00E949A0AAB01BC01E2
:10325000EDB7FEB73A970FB6F894FEBF0FBEEDBFBD
:10326000EDB6FEB60894E11CF11C2AE337E0328388
:1032700021839E01802F912FA32FB22FF7018283EC
:103280009383A483B583CB01BA01209101053091CA
:10329000020540910305509104050E946D70DC0108
:1032A000CB01F70186839783A087B1870E94387688
:1032B0008DB79EB70A960FB6F8949EBF0FBE8DBF0E
:1032C0000E94F50BDF91CF911F910F91FF90EF902E
:1032D0000895EF92FF920F931F93CF93DF9388236C
:1032E00089F08AE694E26FEF70E049E050E00E94D6
:1032F000B0758AE694E260E070E049E050E00E9438
:103300007E7722C00AE614E2C0E0D0E036E4E32E85
:1033100037E0F32ED8018D918D0100D000D0EDB7AC
:10332000FEB73196ADB7BEB71296FC92EE921197EA
:10333000828313820E94387621960F900F900F900F
:103340000F90C830D10531F70E94F50BDF91CF9176
:103350001F910F91FF90EF900895CF92DF92EF921F
:10336000FF926091FE047091FF0480E090E00E9463
:10337000A27565ED72E00E94B775009709F086C0EE
:1033800083E19AE09093E9048093E80488EE94E066
:103390006EE070E042E050E00E947E778CE390E0C7
:1033A0009093E7048093E60486EE94E06CE070E08E
:1033B00042E050E00E947E778AE090E09093E5043E
:1033C0008093E40484EE94E06AE070E042E050E030
:1033D0000E947E77109299061092980688E996E0EE
:1033E0006CE170E042E050E00E947E770F2EF2E246
:1033F000CF2EFFEFDF2EFCECEF2EFBE3FF2EF02DA8
:10340000C0920505D0920605E0920705F0920805E6
:1034100085E095E064E170E044E050E00E947E7752
:10342000C0920105D0920205E0920305F0920405D6
:1034300081E095E060E170E044E050E00E947E773A
:103440008DEE97E4AAE8BCE38093090590930A0502
:10345000A0930B05B0930C0589E095E068E170E05E
:1034600044E050E00E947E778FE08093E30483EE97
:1034700094E069E070E041E050E00E947E7781E0F6
:103480000E94691980E090E00E94910DFF90EF90FA
:10349000DF90CF900895882309F401C18091E8045A
:1034A00080FF0BC000D08BE497E0EDB7FEB79283AE
:1034B00081830E9438760F900F908091E80481FFFD
:1034C0000BC000D081E597E0EDB7FEB79283818312
:1034D0000E9438760F900F908091E80482FF0BC015
:1034E00000D086E597E0EDB7FEB7928381830E9416
:1034F00038760F900F908091E80483FF0BC000D0C6
:103500008CE597E0EDB7FEB7928381830E94387611
:103510000F900F908091E80484FF0BC000D085E6E7
:1035200097E0EDB7FEB7928381830E9438760F90C3
:103530000F908091E80485FF0BC000D08EE697E0E5
:10354000EDB7FEB7928381830E9438760F900F907B
:103550008091E80486FF0BC000D084E797E0EDB7C8
:10356000FEB7928381830E9438760F900F908091EE
:10357000E80487FF0BC000D08CE797E0EDB7FEB7FB
:10358000928381830E9438760F900F908091E80497
:103590009091E90490FF0BC000D082E897E0EDB76E
:1035A000FEB7928381830E9438760F900F908091AE
:1035B000E8049091E90491FF0BC000D08AE897E0FD
:1035C000EDB7FEB7928381830E9438760F900F90FB
:1035D0008091E8049091E90492FF0BC000D084E947
:1035E00097E0EDB7FEB7928381830E9438760F9003
:1035F0000F908091E8049091E90493FF0BC000D0F4
:103600008AE997E0EDB7FEB7928381830E9438760E
:103610000F900F908091E8049091E90494FF0BC003
:1036200000D082EA97E0EDB7FEB7928381830E94D3
:1036300038760F900F908091E8049091E90495FFFF
:103640000BC000D088EA97E0EDB7FEB79283818384
:103650000E9438760F900F908091E8049091E904D1
:1036600096FF0BC000D08EEA97E0EDB7FEB79283CD
:1036700081830E9438760F900F908091E80490919A
:10368000E90497FF4AC100D083EB97E0EDB7FEB79E
:10369000928381830E9438760F900F903EC100D0B4
:1036A00000D089EB97E0EDB7FEB79283818381E08C
:1036B00090E0948383830E9438760F900F900F9050
:1036C0000F900E94F50B00D000D085EC97E0EDB78D
:1036D000FEB79283818382E090E0948383830E948B
:1036E00038760F900F900F900F900E94F50B00D03E
:1036F00000D080ED97E0EDB7FEB79283818384E040
:1037000090E0948383830E9438760F900F900F90FF
:103710000F900E94F50B00D000D08CED97E0EDB734
:10372000FEB79283818388E090E0948383830E9434
:1037300038760F900F900F900F900E94F50B00D0ED
:1037400000D08AEE97E0EDB7FEB79283818380E1E7
:1037500090E0948383830E9438760F900F900F90AF
:103760000F900E94F50B00D000D088EF97E0EDB7E6
:10377000FEB79283818380E290E0948383830E94EA
:1037800038760F900F900F900F900E94F50B00D09D
:1037900000D084E098E0EDB7FEB79283818380E4A7
:1037A00090E0948383830E9438760F900F900F905F
:1037B0000F900E94F50B00D000D082E198E0EDB7A9
:1037C000FEB79283818380E890E0948383830E9494
:1037D00038760F900F900F900F900E94F50B00D04D
:1037E00000D08EE198E0EDB7FEB79283818380E050
:1037F00091E0948383830E9438760F900F900F900E
:103800000F900E94F50B00D000D08CE298E0EDB74D
:10381000FEB79283818380E092E0948383830E9449
:1038200038760F900F900F900F900E94F50B00D0FC
:1038300000D08BE398E0EDB7FEB79283818380E000
:1038400094E0948383830E9438760F900F900F90BA
:103850000F900E94F50B00D000D087E498E0EDB700
:10386000FEB79283818380E098E0948383830E94F3
:1038700038760F900F900F900F900E94F50B00D0AC
:1038800000D085E598E0EDB7FEB79283818380E0B4
:1038900090E1948383830E9438760F900F900F906D
:1038A0000F900E94F50B00D000D081E698E0EDB7B4
:1038B000FEB79283818380E090E2948383830E94A9
:1038C00038760F900F900F900F900E94F50B00D05C
:1038D00000D08DE698E0EDB7FEB79283818380E05B
:1038E00090E4948383830E9438760F900F900F901A
:1038F0000F900E94F50B00D000D088E798E0EDB75C
:10390000FEB79283818380E090E8948383830E9452
:1039100038760F900F900F900F900E94F50B08953E
:103920002F923F924F925F926F927F928F929F92CF
:10393000AF92BF92CF92DF92EF92FF920F931F93BD
:10394000CF93DF9300D0CDB7DEB79A838983DC01B4
:103950008D919C911197009711F00C94AC2E609171
:10396000FE047091FF0485E190E20E94A27585E15A
:1039700090E260E470E00E94C075009759F4609195
:10398000352D7091362D8AE090E00E94FA7581E025
:103990000C94B22E8130910549F4209015203324E7
:1039A00044245524662477244301BEC18230910506
:1039B00099F43091152020911620932F80E0820FEA
:1039C000911D1C01892F880F880B482E582E682EB8
:1039D000782E882E982EA8C18330910509F09CC0BE
:1039E0002091152080901620B090172030E040E004
:1039F00050E060E070E080E090E000E10E942B6A1F
:103A0000922EA32E142FF52EE62EC72E282ED92E59
:103A1000282D30E040E050E060E070E080E090E091
:103A200008E00E942B6A290DB1E0291508F0B0E0EA
:103A30003A0DE1E03A1508F0E0E0B30FF1E0B3171A
:103A400008F0F0E0EF2B410F31E0411708F030E0D3
:103A5000E40FF1E0E41708F0F0E03F2B5F0D41E0E8
:103A60005F1508F040E0A32FA50F31E0A51708F07F
:103A700030E0432B6E0D31E06E1508F030E0F42F8E
:103A8000F60F41E0F61708F040E0342B7C0D41E0E2
:103A90007C1508F040E0532F570F31E0571708F01E
:103AA00030E0432B820D31E0821508F030E0480F02
:103AB00061E0481708F060E0362BD90ED30EB20E45
:103AC00081E0B21608F080E0182F1B0F71E01B1781
:103AD00008F070E07E0F61E07E1708F060E06A0F8A
:103AE00031E06A1708F030E03F0F21E03F1708F09F
:103AF00020E0250F91E0251708F090E0940F81E079
:103B0000941708F080E02B2C312E472E562E632E72
:103B1000722E892E982EFDC08430910509F0FBC0CD
:103B20002091152080901620A0901720B09018208A
:103B300030E040E050E060E070E080E090E008E1DC
:103B40000E942B6A722E932E142FF52EE62EC72E6E
:103B5000282ED92E282D30E040E050E060E070E0C3
:103B600080E090E000E10E942B6A270DF1E027152C
:103B700008F0F0E0390DE1E0391508F0E0E0F30F6E
:103B8000A1E0F31708F0A0E0EA2B410F31E0411764
:103B900008F030E0E40FA1E0E41708F0A0E03A2BD1
:103BA0005F0D41E05F1508F040E0B32FB50F31E045
:103BB000B51708F030E0432B6E0D31E06E1508F0BC
:103BC00030E0A42FA60F41E0A61708F040E0342B08
:103BD0007C0D41E07C1508F040E0532F570F31E099
:103BE000571708F030E0432B820D31E0821508F0C2
:103BF00030E0480F61E0481708F060E0362BD90E3E
:103C0000D30E222E2B0C81E0221608F080E0B82E75
:103C1000BF0E81E0BF1608F080E0982E9E0E81E076
:103C20009E1608F080E0C82ECB0E11E0CB1608F0EF
:103C300010E01A0F81E01A1708F080E0F82EF50E58
:103C400081E0F51608F080E0E82EE40E81E0E4164D
:103C500008F080E0D80E2A2D30E040E050E060E02F
:103C600070E080E090E008E00E942B6A220DE1E025
:103C7000221508F0E0E03B0DF1E03B1508F0F0E024
:103C8000E30FA1E0E31708F0A0E0FA2B490D31E0C3
:103C9000491508F030E0F40FA1E0F41708F0A0E0B7
:103CA0003A2B5C0D41E05C1508F040E0A32FA50F16
:103CB00031E0A51708F030E0432B610F31E06117C8
:103CC00008F030E0542F560F41E0561708F040E05E
:103CD000342B7F0D41E07F1508F040E0632F670F24
:103CE00031E0671708F030E0432B8E0D31E08E1580
:103CF00008F030E0480F71E0481708F070E0372B0B
:103D0000D90E222E3E2E4F2E5A2E652E762E842E22
:103D1000932E9D0C09C0FAE02F2E33244424552401
:103D200066247724882499240E94F50BBDE62B167F
:103D300091F4E5E73E1679F4F8E64F1661F4552064
:103D400051F4662041F4772031F4882021F4992041
:103D500011F40C94CB2D9101A201B301C4011DE615
:103D6000A12E05E7B02EE8E6CE2EDD24EE24FF24BA
:103D700000E010E00E94A56A823008F087C283E369
:103D8000281689F491E7391671F4442061F455201E
:103D900051F4662041F4772031F4882021F49920F1
:103DA00011F40C94BC2D9101A201B301C401A3E351
:103DB000AA2EB1E7BB2ECC24DD24EE24FF2400E0A4
:103DC00010E00E94A56A823008F022C1A5E62A16FA
:103DD00081F4B4E63B1669F4442059F4552049F4C3
:103DE000662039F4772029F4882019F4992009F401
:103DF0009EC69101A201B301C401E5E6AE2EF4E630
:103E0000BF2ECC24DD24EE24FF2400E010E00E942D
:103E1000A56A823008F07BC0E5E72E1679F43320DE
:103E200069F4442059F4552049F4662039F4772088
:103E300029F4882019F4992009F4C7C79101A20137
:103E4000B301C40105E7A02EBB24CC24DD24EE245D
:103E5000FF2400E010E00E94A56A823010F5F8E629
:103E60002F1611F00C94AA2E332011F00C94AA2EC8
:103E7000442011F00C94AA2E552011F00C94AA2E77
:103E8000662011F00C94AA2E772011F00C94AA2E23
:103E9000882011F00C94AA2E992011F00C94AA2ECF
:103EA00070C786E7281679F4332069F4442059F462
:103EB000552049F4662039F4772029F4882019F434
:103EC000992009F491C794E6291611F00C94AA2EB2
:103ED000A1E63A1611F00C94AA2E442011F00C948D
:103EE000AA2E552011F00C94AA2E662011F00C94E5
:103EF000AA2E772011F00C94AA2E882011F00C9491
:103F0000AA2E992011F00C94AA2E0C94BC2DB5E683
:103F10002B1689F4EEE63E1671F4442061F4552028
:103F200051F4662041F4772031F4882021F499205F
:103F300011F40C94E1299101A201B301C401B5E689
:103F4000AB2E1EE6B12ECC24DD24EE24FF2400E0AF
:103F500010E00E94A56A823018F5F4E62F1611F0E1
:103F60000C94AA2E89E6381611F00C94AA2E44203F
:103F700011F00C94AA2E552011F00C94AA2E662054
:103F800011F00C94AA2E772011F00C94AA2E882000
:103F900011F00C94AA2E992011F00C94AA2EF5C6BB
:103FA00097E7291689F4AFE63A1671F4442061F4D4
:103FB000552051F4662041F4772031F4882021F413
:103FC000992011F40C947D29B1E32B1611F00C9477
:103FD000AA2EE0E73E1611F00C94AA2E442011F010
:103FE0000C94AA2E552011F00C94AA2E662011F0E4
:103FF0000C94AA2E772011F00C94AA2E882011F090
:104000000C94AA2E992011F00C94AA2E0C946B2AD1
:10401000F3E62F1691F484E6381679F491E6491602
:1040200061F4552051F4662041F4772031F4882062
:1040300021F4992011F40C94BC2D9101A201B3013B
:10404000C401E3E6AE2EF4E6BF2EA1E6CA2EDD24BF
:10405000EE24FF2400E010E00E94A56A823008F000
:1040600080C0A9E62A1689F4B2E73B1671F4442011
:1040700061F4552051F4662041F4772031F4882012
:1040800021F4992011F40C94642B9101A201B30145
:10409000C40119E6A12E02E7B02ECC24DD24EE24C3
:1040A000FF2400E010E00E94A56A823018F5E5E6E2
:1040B0002E1611F00C94AA2E3B1411F00C94AA2E7B
:1040C000442011F00C94AA2E552011F00C94AA2E25
:1040D000662011F00C94AA2E772011F00C94AA2ED1
:1040E000882011F00C94AA2E992011F00C94AA2E7D
:1040F0000C94FE2AF3E72F1689F482E7381671F440
:10410000442061F4552051F4662041F4772031F4C5
:10411000882021F4992011F40C94BD2B93E72916E3
:1041200011F00C94AA2E391611F00C94AA2E4420EA
:1041300011F00C94AA2E552011F00C94AA2E662092
:1041400011F00C94AA2E772011F00C94AA2E88203E
:1041500011F00C94AA2E992011F00C94AA2E0C9414
:10416000CC2BA2E62A1689F4B5E63B1671F4E4E6F8
:104170004E1659F4552049F4662039F4772029F475
:10418000882019F4992009F4D2C49101A201B30145
:10419000C401F2E6AF2EA5E6BA2EB4E6CB2EDD249E
:1041A000EE24FF2400E010E00E94A56A8230B8F5FA
:1041B000F8E72F1681F43C1471F481E6481659F49F
:1041C000552049F4662039F4772029F4882019F421
:1041D000992009F4EBC293E7291611F00C94AA2E4A
:1041E000A5E63A1611F00C94AA2EB1E64B1611F082
:1041F0000C94AA2E552011F00C94AA2E662011F0D2
:104200000C94AA2E772011F00C94AA2E882011F07D
:104210000C94AA2E992011F00C94AA2EF4C5E2E772
:104220002E1681F43E1671F4F5E64F1659F455201A
:1042300049F4662039F4772029F4882019F499206C
:1042400009F479C783E6281611F00C94AA2E9DE68E
:10425000391611F00C94AA2EA8E64A1611F00C9407
:10426000AA2E552011F00C94AA2E662011F00C9461
:10427000AA2E772011F00C94AA2E882011F00C940D
:10428000AA2E992011F00C94AA2E98C2B0E72B16F2
:1042900091F4ECE63E1679F4F5E64F1661F488E603
:1042A000581649F4662039F4772029F4882019F447
:1042B000992009F466C59101A201B301C401B0E7D8
:1042C000AB2E1CE6B12E05E6C02EE8E6DE2EEE246F
:1042D000FF2400E010E00E94A56A823008F01AC1B5
:1042E00090E3291689F4A1E33A1671F4B1E74B166D
:1042F00059F4552049F4662039F4772029F48820B0
:1043000019F4992009F417C79101A201B301C4015E
:10431000E0E3AE2EF1E3BF2EA1E7CA2EDD24EE24AA
:10432000FF2400E010E00E94A56A823008F06EC011
:10433000E4E62E1689F4F3E63F1671F48CE648168F
:1043400059F4552049F4662039F4772029F488205F
:1043500019F4992009F493C69101A201B301C40193
:10436000B4E6AB2E13E6B12E0CE6C02EDD24EE240F
:10437000FF2400E010E00E94A56A823018F52B149B
:1043800011F00C94AA2E92E3391611F00C94AA2E77
:10439000A9E64A1611F00C94AA2E552011F00C949F
:1043A000AA2E662011F00C94AA2E772011F00C94FE
:1043B000AA2E882011F00C94AA2E992011F00C94AA
:1043C000AA2EF8C1B7E62B1689F4EFE63E1671F473
:1043D000FCE64F1659F4552049F4662039F477204D
:1043E00029F4882019F4992009F44CC685E7281689
:1043F00011F00C94AA2E93E6391611F00C94AA2E03
:10440000ADE64A1611F00C94AA2E36C0B0E72B1672
:1044100091F4E5E63E1679F4F2E74F1661F4552083
:1044200051F4662041F4772031F4882021F499205A
:1044300011F40C94FE2A9101A201B301C401E0E73A
:10444000AE2EF5E6BF2EA2E7CA2EDD24EE24FF2411
:1044500000E010E00E94A56A823018F581E328167A
:1044600011F00C94AA2E381611F00C94AA2E91E794
:10447000491611F00C94AA2E552011F00C94AA2E76
:10448000662011F00C94AA2E772011F00C94AA2E1D
:10449000882011F00C94AA2E992011F00C94AA2EC9
:1044A000ADC6A4E72A1689F4BFE63B1671F44B1695
:1044B00061F4E2E65E1649F4662039F4772029F4C7
:1044C000882019F4992009F4F9C4F9E62F1611F09F
:1044D0000C94AA2E8CE6381611F00C94AA2E91E6B4
:1044E000491611F00C94AA2EA3E65A1611F00C945A
:1044F000AA2E662011F00C94AA2E772011F00C94AD
:10450000AA2E882011F00C94AA2E992011F00C9458
:10451000AA2E80C1B3E72B1699F4E2E73E1681F488
:10452000F7E74F1669F480E7581651F4662041F416
:10453000772031F4882021F4992011F40C94B62AC4
:104540009101A201B301C401A3E7AA2EB2E7BB2ED9
:1045500017E7C12E00E7D02EEE24FF2400E010E084
:104560000E94A56A823008F085C02D1491F49DE662
:10457000391679F4A5E74A1661F4B8E65B1649F4F2
:10458000662039F4772029F4882019F4992009F459
:10459000E2C69101A201B301C40110E7A12E0DE60C
:1045A000B02EE5E7CE2EF8E6DF2EEE24FF2400E065
:1045B00010E00E94A56A823010F5E1E62E1611F097
:1045C0000C94AA2E3B1411F00C94AA2E4C1411F04A
:1045D0000C94AA2E5D1411F00C94AA2E662011F0F2
:1045E0000C94AA2E772011F00C94AA2E882011F09A
:1045F0000C94AA2E992011F00C94AA2E93C6F3E7DE
:104600002F1699F485E6381681F492E7491669F475
:10461000A0E75A1651F4662041F4772031F488203F
:1046200021F4992011F40C94152EB1E32B1611F0FE
:104630000C94AA2EE2E73E1611F00C94AA2EF7E78E
:104640004F1611F00C94AA2E80E7581611F00C9416
:10465000AA2E662011F00C94AA2E772011F00C944B
:10466000AA2E882011F00C94AA2E992011F00C94F7
:10467000AA2EA8C097E7291691F4A0E73A1679F474
:10468000B8E74B1661F4E4E75E1649F4662039F4A6
:10469000772029F4882019F4992009F4E4C39101C2
:1046A000A201B301C401E7E7AE2EF0E7BF2EA8E7F1
:1046B000CA2EB4E7DB2EEE24FF2400E010E00E94B7
:1046C000A56A8230C0F52D1491F4F3E73F1679F412
:1046D00085E6481661F492E7591649F4662039F4E4
:1046E000772029F4882019F4992009F4F1C6A4E769
:1046F0002A1611F00C94AA2EB3E73B1611F00C9475
:10470000AA2EE5E64E1611F00C94AA2E5A1611F0B8
:104710000C94AA2E662011F00C94AA2E772011F08A
:104720000C94AA2E882011F00C94AA2E992011F036
:104730000C94AA2EC6C3F2E72F1691F487E638161A
:1047400079F490E7491661F4A5E75A1649F4662012
:1047500039F4772029F4882019F4992009F460C4E9
:10476000BCE62B1611F00C94AA2EE1E63E1611F0D1
:104770000C94AA2EF4E74F1611F00C94AA2E88E799
:10478000581611F00C94AA2E662011F00C94AA2E43
:10479000772011F00C94AA2E882011F00C94AA2EE8
:1047A000992011F00C94AA2E0C94702E0E9469147A
:1047B0000C94AC2E0E94BA0F0C94AC2E0E94F214F2
:1047C0000C94AC2E6091FE047091FF0480E090E0A8
:1047D0000E94A2758C016CED72E00E94B775009783
:1047E00019F477980C94AC2EC8016FED72E00E941A
:1047F000B775009719F4779A0C94AC2E779903C08B
:104800008CED92E002C08FED92E000D000D024E861
:1048100038E08AC46091FE047091FF0480E090E06B
:104820000E94A2758C0166EF72E00E94B775009736
:1048300009F04FC06091FE047091FF0480E090E0A9
:104840000E94A2758C01009711F40C94AC2E69EFB4
:1048500072E00E94B775009729F482E29FEFACECFA
:10486000BBE30BC0C8016FEF72E00E94B775009701
:1048700099F482E29FEFACECBAE380930505909344
:104880000605A0930705B093080585E095E064E16F
:1048900070E044E050E097C6C8010E9495746B0137
:1048A0007C0120E030E040E050E00E944F6F882320
:1048B00061F081E00E949A0A9B01AC01C701B60138
:1048C0000E94536FDC01CB01D8CF00D082E09CE086
:1048D0007FC0C80164E073E00E94B775009709F0DB
:1048E0004DC06091FE047091FF0480E090E00E9452
:1048F000A2758C01009711F40C94AC2E69EF72E054
:104900000E94B775009729F482E29FEFACECBBE3FD
:1049100024C0C8016FEF72E00E94B775009729F4B8
:1049200082E29FEFACECBAE318C0C8010E94957414
:104930006B017C0120E030E040E050E00E944F6FCE
:104940008823C1F082E00E949A0A9B01AC01C70152
:10495000B6010E94536FDC01CB0180930105909357
:104960000205A0930305B093040581E095E060E1A2
:1049700070E08FCF00D08FE09CE05FC0C80167E09F
:1049800073E00E94B775009709F063C06091FE0460
:104990007091FF0480E090E00E94A2758C01009766
:1049A00011F40C94AC2E69EF72E00E94B775009779
:1049B00029F48DEE97E4AAE8BCE32FC0C8016FEF9D
:1049C00072E00E94B775009741F400D08CE19CE042
:1049D000EDB7FEB79283818336C0C8010E949574FB
:1049E0006B017C0120E030E040E050E00E944F6F1E
:1049F000882301F180E00E949A0A4B015C01C70103
:104A0000B60121EE3AE744E95EE30E94EA6EA501B1
:104A100094010E94536FDC01CB01809309059093B0
:104A20000A05A0930B05B0930C0589E095E068E1B9
:104A300070E02FCF00D08BE29CE0ADB7BEB71296EE
:104A40009C938E9311970E9438760F900F900C9440
:104A5000AC2E0E94EE0AAB01BC0100D000D000D009
:104A600088E39CE0EDB7FEB7928381834383548350
:104A7000658376830E943876EDB7FEB736960FB61B
:104A8000F894FEBF0FBEEDBF81E00E949A0A20910C
:104A900005053091060540910705509108050E94D3
:104AA0006D706B01182F092F82E00E949A0AAB01EA
:104AB000BC018DB79EB70A970FB6F8949EBF0FBE84
:104AC0008DBFEDB6FEB60894E11CF11C8FE39CE0AF
:104AD000ADB7BEB712969C938E93119798018C2D0B
:104AE0009D2DA32FB22FF70182839383A483B583D7
:104AF000CB01BA01209101053091020540910305D7
:104B0000509104050E946D70DC01CB01F701868392
:104B10009783A087B1870E9438768DB79EB70A9693
:104B20000FB6F8949EBF0FBE8DBF0C94A72E609158
:104B3000FE047091FF0480E090E00E94A27500974F
:104B400071F160E070E040E150E00E945473AB010D
:104B5000BC0180919806909199068417950799F168
:104B6000509399064093980688E996E06CE170E0CE
:104B700042E050E00E947E778091980690919906DD
:104B800000D000D028E838E0ADB7BEB712963C930D
:104B90002E93119714969C938E9313970EC0809129
:104BA00098069091990600D000D028E938E0EDB73A
:104BB000FEB732832183948383830E9438760F90DB
:104BC0000F900F900F900E94F50B00D000D08CEA50
:104BD00098E0ADB7BEB712969C938E93119781E083
:104BE00090E014969C938E9313970E94387689EBED
:104BF00098E0EDB7FEB79283818382E090E09483E2
:104C000083830E94387684EC98E0ADB7BEB71296E5
:104C10009C938E93119784E090E014969C938E93CE
:104C200013970E9438768FEC98E0EDB7FEB7928329
:104C3000818388E090E0948383830E9438768CEDB2
:104C400098E0ADB7BEB712969C938E93119780E112
:104C500090E014969C938E9313970E94387687EE7B
:104C600098E0EDB7FEB79283818380E290E0948371
:104C700083830E94387683EF98E0ADB7BEB7129673
:104C80009C938E93119780E490E014969C938E935E
:104C900013970E94387681E099E0EDB7FEB79283D2
:104CA000818380E890E0948383830E9438768FE04C
:104CB00099E0ADB7BEB712969C938E93119780E0A2
:104CC00091E014969C938E9313970E9438768EE110
:104CD00099E0EDB7FEB79283818380E092E0948300
:104CE00083830E9438768DE299E0ADB7BEB7129605
:104CF0009C938E93119780E094E014969C938E93EE
:104D000013970E94387689E399E0EDB7FEB7928356
:104D1000818380E098E0948383830E94387687E4DF
:104D200099E0ADB7BEB712969C938E93119780E031
:104D300090E114969C938E9313970E94387684E5A5
:104D400099E0EDB7FEB79283818380E090E294838F
:104D500083830E94387682E699E0ADB7BEB712969B
:104D60009C938E93119780E090E414969C938E937D
:104D700013970E9438760F900F900F900F900C941D
:104D8000AC2E0E943A170C94AC2E6091FE047091E8
:104D9000FF0480E090E00E94A27569EF72E00E943B
:104DA000B775009711F481E001C080E00E94691995
:104DB00020910005222309F4CFC700D000D0EDB721
:104DC000FEB7319682E799E0BDC20E941B18209180
:104DD0000005222309F4C0C700D000D0EDB7FEB70C
:104DE000319685E799E0AEC20E9416182091000521
:104DF000222309F4B1C700D000D0EDB7FEB7319639
:104E000088E799E09FC26091FE047091FF0480E002
:104E100090E00E94A2758C016CED72E00E94B77563
:104E2000009731F48091E4049091E5048460C1C35B
:104E3000C8016FED72E00E94B7759C018091E40497
:104E40009091E5042115310511F48B7FB2C382FFE7
:104E500003C08CED92E002C08FED92E000D000D054
:104E60002BE43CE0A7C26091FE047091FF0480E057
:104E700090E00E94A2750E949974982F91509F30E3
:104E800060F48093E30490E00E94CC4F83EE94E0C2
:104E900069E070E041E050E096C300D000D0EDB78B
:104EA000FEB731968BE799E0ADB7BEB712969C93EB
:104EB0008E9311978091E30482834BC20C9400007F
:104EC0004BC76091FE047091FF0480E090E00E9467
:104ED000A2758C016CE073E00E94B775009739F4FD
:104EE000219A8091E4049091E504806162C3C80135
:104EF0006EE073E00E94B775009739F4229A8091B2
:104F0000E4049091E504806254C3C80160E173E059
:104F10000E94B775009739F4239A8091E404909128
:104F2000E504806446C3C80162E173E00E94B7757E
:104F3000009739F4239A8091E4049091E504806805
:104F400038C3C8016FED72E00E94B7759C01809173
:104F5000E4049091E5042115310539F48F709093A4
:104F6000E5048093E4042B9A28C384FF03C08CEDEE
:104F700092E002C08FED92E000D000D02FE43CE040
:104F8000EDB7FEB732832183948383830E94387602
:104F90008091E4040F900F900F900F9085FF03C055
:104FA0008CED92E002C08FED92E000D000D02AE5B7
:104FB0003CE0ADB7BEB712963C932E931197149672
:104FC0009C938E9313970E9438768091E4040F90FF
:104FD0000F900F900F9086FF03C08CED92E002C0FF
:104FE0008FED92E000D000D025E63CE0EDB7FEB7B3
:104FF00032832183948383830E9438768091E404F2
:105000000F900F900F900F9087FF03C08CED92E0F0
:1050100002C08FED92E000D000D020E73CE084C0D9
:1050200000D088E899E0EDB7FEB7928381830E94B3
:105030003876209100050F900F902223A9F000D020
:1050400000D0EDB7FEB731968CE899E0ADB7BEB7AA
:1050500012969C938E931197228313820E94387626
:105060000F900F900F900F9088E10FB6F8948093F7
:105070006000109260000FBE0C94007C6DC60E9410
:10508000B7466AC66091FE047091FF0480E090E02C
:105090000E94A2757C016CED72E00E94B7750097CA
:1050A00049F40E947A4C8091E4049091E504816077
:1050B0008D7F7FC2C7016FED72E00E94B7750097C8
:1050C00041F40E946B4D8091E4049091E5048C7F43
:1050D00070C204E113E0C701B8010E94B7750097E0
:1050E00049F40E946B4D8091E4049091E5048E7F19
:1050F00082605FC28091E40481FF0BC000D000D0C9
:105100008BE79CE0EDB7FEB7928381831483038322
:1051100030CE80FF03C08CED92E002C08FED92E0B4
:1051200000D000D02FE73CE0ADB7BEB712963C935D
:105130002E9311971ACE00D08FE899E0EDB7FEB705
:10514000928381830E9438768DB79EB740970FB6C1
:10515000F8949EBF0FBE8DBFEDB7FEB7319689EBB9
:1051600099E0ADB7BEB712969C938E93119780913C
:10517000102090911120A0911220B09113208283D1
:105180009383A483B5838091042090910520A091FE
:105190000620B091072086839783A087B1878091EE
:1051A000082090910920A0910A20B0910B208287BD
:1051B0009387A487B58780910C2090910D20A091B2
:1051C0000E20B0910F2086879787A08BB18B0E940D
:1051D000387620910005EDB7FEB772960FB6F894B9
:1051E000FEBF0FBEEDBF222309F4B6C500D000D02C
:1051F000EDB7FEB7319687ED99E0A4C0F89409E0C9
:1052000081E090E0FC0100935700C895F02C20E06D
:1052100030E0F90100935700C895E02C7894F89499
:1052200023E030E0F90100935700C895102D82E08B
:1052300090E0FC0100935700C895002D789400D0B1
:1052400000D000D02AED39E0EDB7FEB732832183DC
:105250008091B1179091B217A091B317B091B41784
:1052600083839483A583B6830E94387600D000D0D0
:10527000EDB7FEB7319684EE99E0ADB7BEB71296A2
:105280009C938E9311970283138214831582E68276
:105290001782F08611860E943876EDB7FEB73A96EF
:1052A0000FB6F894FEBF0FBEEDBF0E94CD1820913F
:1052B000660000D000D0EDB7FEB731968BE09AE0E3
:1052C000ADB7BEB712969C938E931197228313822B
:1052D0000E9438760F900F900F900F900E94F50B60
:1052E00020910005222309F437C500D000D0EDB786
:1052F000FEB7319687E19AE025C080E090E00E94F9
:10530000010C81E090E00E94010C20910005222315
:1053100009F422C500D000D0EDB7FEB731968AE17E
:105320009AE010C00E94A9160E94F50B209100057A
:10533000222309F411C500D000D0EDB7FEB7319695
:105340008DE19AE0ADB7BEB712969C938E931197FC
:10535000228313820ECD6091FE047091FF0480E0E1
:1053600090E00E94A2758C016CED72E00E94B7750E
:10537000009731F48091E4049091E504886019C1AC
:10538000C8016FED72E00E94B7759C018091E40442
:105390009091E5042115310511F4877F0AC183FF3F
:1053A00003C08CED92E002C08FED92E000D000D0FF
:1053B00023E83CE0EDB7FEB73283218394838383F7
:1053C000D8CC6091FE047091FF0480E090E00E94D0
:1053D000A27569E173E00E94B775009731F5F89402
:1053E0008EE996E00E941A3B0CC0C8010D960E94FF
:1053F000323E81E195E0B8010E94D23AC8010E9494
:10540000C03B8C01009789F704C08EE996E00E94AA
:10541000473B8EE996E00E94A23B0097B1F78EE9E8
:1054200096E00E94163B789446C08EE996E00E9472
:105430001A3B7C010FE113E03BC08DB79EB70C9780
:105440000FB6F8949EBF0FBE8DBFEDB7FEB7319675
:10545000ADB7BEB712961C930E931197D701129653
:105460008C9112978283138213968C911397848365
:10547000158218968C9118978683178214968D91B1
:105480009C9115979187808716968D919C9117977F
:10549000938782870E942676EDB7FEB73C960FB6BB
:1054A000F894FEBF0FBEEDBFC7010E94C03B7C0158
:1054B000E114F10411F620910005222309F44CC4F3
:1054C00000D000D0EDB7FEB7319680E29AE03ACF37
:1054D0000E94AD1941C46091FE047091FF0480E008
:1054E00090E00E94A2758C016CED72E00E94B7758D
:1054F000009731F48091E4049091E50492600EC02D
:10550000C8016FED72E00E94B7759C018091E404C0
:105510009091E5042115310571F49D7F9093E50488
:105520008093E40484EE94E06AE070E042E050E0AE
:105530000E947E7717C091FF03C08CED92E002C0FD
:105540008FED92E000D000D027E83CE0EDB7FEB749
:1055500032832183948383830E9438760F900F9047
:105560000F900F9081E00E94060AF6C36091FE043E
:105570007091FF0480E090E00E94A2758C016EEEB5
:1055800072E00E94B775009731F48091E404909125
:10559000E5049E7F0EC0C80163EE72E00E94B775FD
:1055A0009C018091E4049091E5042115310571F48A
:1055B00091609093E5048093E40484EE94E06AE0C3
:1055C00070E042E050E00E947E77C6C390FF03C0C7
:1055D00083EE92E002C08EEE92E000D000D026E48E
:1055E00033E0ADB7BEB712963C932E931197149645
:1055F0009C938E9313970E942676BDCB6091FE04F8
:105600007091FF0480E090E00E94A275009769F11C
:1056100060E070E040E150E00E945473DC01CB0197
:105620009093E9048093E80400D000D04DB75EB7B2
:105630004F5F5F4F23E23AE0EDB7FEB7328321833D
:10564000FA01938382830E9438760F900F900F9017
:105650000F9088EE94E06EE070E042E050E00E942F
:105660007E7781E00E944B1A77C380E00E944B1A3C
:105670000E94F50B00D000D084E39AE0ADB7BEB72E
:1056800012969C938E9311978091E8049091E9046F
:1056900014969C938E9313970E9438760F900F90D8
:1056A0000F900F9081E00E944B1A0E94F50B209101
:1056B0000005222309F450C300D000D0EDB7FEB797
:1056C000319687E49AE03ECE6091FE047091FF042B
:1056D00080E090E00E94A275009751F160E070E0D8
:1056E0004AE050E00E945473DC01CB019093E70440
:1056F0008093E60400D000D04DB75EB74F5F5F4F98
:105700002AE43AE0EDB7FEB732832183FA019383AE
:1057100082830E9438760F900F900F900F9086EE44
:1057200094E06CE070E042E050E00E947E7718C0A8
:1057300000D000D087E69AE0ADB7BEB712969C9332
:105740008E9311978091E6049091E70414969C93B0
:105750008E9313970E9438760F900F900F900F90B2
:1057600020910005222309F4F7C200D000D0EDB744
:10577000FEB7319688E89AE0E5CD0E946B3E209115
:105780000005222309F4E8C200D000D0EDB7FEB72F
:1057900031968BE89AE0D6CD00D08EE89AE0EDB74E
:1057A000FEB7928381830E9438760F900F900E94FB
:1057B000161800D08EE99AE0ADB7BEB712969C934A
:1057C0008E9311970E9438760F900F9080E00E9480
:1057D000691900D082EA9AE0EDB7FEB7928381831F
:1057E0000E9438760F900F900E94BA0F0E941B18EB
:1057F00000D000D0EDB7FEB7319688EA9AE0ADB799
:10580000BEB712969C938E9311978091E304828386
:1058100013820E94387685EB9AE0EDB7FEB792834B
:10582000818380E490E0948383830E94387600D063
:10583000EDB7FEB731968DEC9AE0ADB7BEB71296D4
:105840009C938E93119780917A2482831382809106
:105850007B24848315820E9438760F900F9080EE0F
:105860009AE0EDB7FEB7928381838091E604909130
:10587000E704948383830E94387685EF9AE0ADB77E
:10588000BEB712969C938E9311978091E8049091E5
:10589000E90414969C938E9313970E9438760F9088
:1058A0000F900F900F9081E00E944B1A0E94EE0A19
:1058B000AB01BC0100D000D000D088E09BE0EDB788
:1058C000FEB79283818343835483658376830E94EA
:1058D0003876EDB7FEB736960FB6F894FEBF0FBE1A
:1058E000EDBF0E94370B0E94080BAB01BC0100D03A
:1058F00000D000D085E19BE0ADB7BEB712969C9377
:105900008E931197EDB7FEB74383548365837683F7
:105910000E9438768DB79EB706960FB6F8949EBF54
:105920000FBE8DBF1D9B03C083EF92E002C08FEDC1
:1059300092E000D000D023E23BE0ADB7BEB71296B4
:105940003C932E93119714969C938E9313970E94D9
:1059500038768091552490915624A0915724B09187
:1059600058244091592450915A2460915B2470919D
:105970005C2400D000D000D00DB71EB70F5F1F4FC2
:105980002FE23BE0EDB7FEB732832183F80182833B
:105990009383A483B58346835783608771870E946E
:1059A0003876EDB7FEB731968DE49BE0ADB7BEB764
:1059B00012969C938E931197809162249091632408
:1059C000A0916424B091652482839383A483B583DA
:1059D0008091662490916724A0916824B0916924F5
:1059E00086839783A087B1870E943876EDB7FEB78C
:1059F00038960FB6F894FEBF0FBEEDBF8FE69BE062
:105A0000928381830E9438768091E4040F900F90F6
:105A100081FF0EC000D089E79BE0ADB7BEB71296FC
:105A20009C938E9311970E9438760F900F9017C019
:105A300080FF03C08CED92E002C08FED92E000D0B9
:105A400000D02FE73BE0EDB7FEB73283218394838C
:105A500083830E9438760F900F900F900F90809163
:105A6000E40483FF03C08CED92E002C08FED92E06E
:105A700000D000D023E83BE0ADB7BEB712963C9310
:105A80002E93119714969C938E9313970E943876B9
:105A90008091E4049091E5040F900F900F900F9087
:105AA00091FF03C08CED92E002C08FED92E000D038
:105AB00000D026E93BE0EDB7FEB732832183948323
:105AC00083830E943876809198069091990623EA04
:105AD0003BE0ADB7BEB712963C932E931197149648
:105AE0009C938E9313970E9438760F900F900F908F
:105AF0000F90779903C08CED92E002C08FED92E099
:105B000000D000D020EB3BE0EDB7FEB7328321831D
:105B1000948383830E9438768091E4049091E50415
:105B20000F900F900F900F9090FF03C083EE92E0C4
:105B300002C08EEE92E000D000D026E433E0ADB794
:105B4000BEB712963C932E93119714969C938E9306
:105B500013970E942676209100050F900F900F90CA
:105B60000F90222309F4F8C000D000D0EDB7FEB7A3
:105B7000319689EB9BE0E6CB0E94F218209100055C
:105B8000222309F4E9C000D000D0EDB7FEB731966A
:105B90008CEB9BE0D7CB0E94ED150097B9F500D0B8
:105BA00000D000D08FEB9BE0EDB7FEB792838183EE
:105BB0008091FA179091FB17A091FC17B091FD17F7
:105BC00083839483A583B6830E9438768AEC9BE016
:105BD000ADB7BEB712969C938E93119780917624A1
:105BE00090917724A0917824B0917924EDB7FEB7F5
:105BF00083839483A583B6830E9438768DB79EB73E
:105C000006960FB6F8949EBF0FBE8DBF0E94F50B8F
:105C100020910005222309F49FC000D000D0EDB7E9
:105C2000FEB7319687ED9BE08DCB83E061E048E0E5
:105C300021E00E949A1100D000D000D08AED9BE0B4
:105C4000EDB7FEB7928381838091ED179091EE17A7
:105C5000A091EF17B091F01783839483A583B68347
:105C60000E94387600D000D0EDB7FEB7319681EEB5
:105C70009BE0ADB7BEB712969C938E93119780911F
:105C8000F1179091F217A091F317B091F417828356
:105C90009383A483B5838091F5179091F617A09113
:105CA000F717B091F81786839783A087B1870E9472
:105CB0003876EDB7FEB73A960FB6F894FEBF0FBE32
:105CC000EDBF0E94F50B20910005222309F444C08A
:105CD00000D000D0EDB7FEB7319682EF9BE032CB1B
:105CE0006091FE047091FF0480E090E00E94A27534
:105CF0006FE473E00E94B7750097A1F46091FE0411
:105D00007091FF0480E090E00E94A275009721F15D
:105D10000E949974803100F590915201982B9093D4
:105D200052011AC08091520100D000D025EF3BE013
:105D3000EDB7FEB73283218390E08F70907094832B
:105D400083830E9438760F900F900F900F900E94DF
:105D5000F50B02C00E941317A981BA8111961C92FB
:105D60001E9283E00F900F90DF91CF911F910F91C2
:105D7000FF90EF90DF90CF90BF90AF909F908F906B
:105D80007F906F905F904F903F902F900895F89480
:105D900091E2E0E0F0E0909357008491E2E0F0E0DF
:105DA000909357004491E4E0F0E090935700E49121
:105DB00090E0A0E0B0E0DC019927882750E060E0A7
:105DC00070E0762F652F542F4427840F951FA61F50
:105DD000B71F8E0F911DA11DB11D8093B117909318
:105DE000B217A093B317B093B41778940895CF93D4
:105DF000DF93CDB7DEB727970FB6F894DEBF0FBE9F
:105E0000CDBFCE0102966EE070E042E050E00E940D
:105E100060778A819B812FEF8F3F920749F488EE4C
:105E200094E06EE070E042E050E00E947E7704C0B3
:105E30009093E9048093E804CE0102966CE070E050
:105E400042E050E00E9460778A819B812FEF8F3F74
:105E5000920779F48CE390E09093E7048093E60452
:105E600086EE94E06CE070E042E050E00E947E77C5
:105E700004C09093E7048093E604CE0102966AE0A2
:105E800070E042E050E00E9460778A819B812FEFB2
:105E90008F3F920779F48AE090E09093E504809335
:105EA000E40484EE94E06AE070E042E050E00E9496
:105EB0007E7704C09093E5048093E404CE010296BB
:105EC0006CE170E042E050E00E9460778A819B8143
:105ED0002FEF8F3F920769F410929906109298065F
:105EE00088E996E06CE170E042E050E00E947E7745
:105EF00004C090939906809398068AE694E260E045
:105F000070E049E050E00E9460770E947D0DCE0174
:105F1000049664E170E044E050E00E9460778C8178
:105F20009D81AE81BF818F3F2FEF92072FEFA20798
:105F30002FEFB20749F485E095E064E170E044E0BA
:105F400050E00E947E7708C085E095E064E170E053
:105F500044E050E00E946077CE01049660E170E07A
:105F600044E050E00E9460778C819D81AE81BF81CA
:105F70008F3F2FEF92072FEFA2072FEFB20749F4C1
:105F800081E095E060E170E044E050E00E947E77BF
:105F900008C081E095E060E170E044E050E00E94DC
:105FA0006077CE01049668E170E044E050E00E9422
:105FB00060778C819D81AE81BF818F3F2FEF9207EB
:105FC0002FEFA2072FEFB20749F489E095E068E1CF
:105FD00070E044E050E00E947E7708C089E095E0E0
:105FE00068E170E044E050E00E946077CE010196E5
:105FF00069E070E041E050E00E94607789818F3F66
:1060000049F483EE94E069E070E041E050E00E94E2
:106010007E7708C083EE94E069E070E041E050E0F4
:106020000E94607727960FB6F894DEBF0FBECDBFF3
:10603000DF91CF9108956C9A6B9A6A9A6F9A729ACF
:10604000749A739A779A809880B3897F80BB87E02F
:1060500080937E00549A0E94C72E0E94F72E81E002
:106060000E94060A80E090E00E94910D0E94454542
:106070008091E40486FD239A0895CF93DF93EC0189
:1060800088819981009731F029E08537920709F0DE
:106090007BC071C00E941B308091E40480FD02C06F
:1060A0000E946B4D809170008C7F80937000809176
:1060B000B60080628093B6001092B20082E08093B6
:1060C000B1008091B60090E0877090700097C9F79A
:1060D0008091700081608093700080E090E065E2C4
:1060E00078E00E943D4B0E94161880E00E946919DA
:1060F0000E94BA0F8091FE1B85FF02C00E9462467B
:106100008FE090E00E94CC4F0E942D4E8093A0061D
:1061100000D000D000D0EDB7FEB7319624E533E0D3
:10612000ADB7BEB712963C932E931197828313821C
:106130008091E304848315820E9426761092A20641
:106140001092A1068DB79EB706960FB6F8949EBF23
:106150000FBE8DBF89ED94E09093742480937324D7
:1061600083E290E09093A4068093A30685E799E0EC
:10617000998388830DC0633259F481EA96E060E028
:1061800070E00E94901CE6CF1982188283E001C063
:1061900081E0DF91CF9108958536910564F12091DA
:1061A00098063091990620FF10C000D000D026E656
:1061B00033E0EDB7FEB732832183948383830E945B
:1061C00026760F900F900F900F9080911020909155
:1061D0001120A0911220B09113200196A11DB11D94
:1061E0008093102090931120A0931220B09313203D
:1061F00081E090E0089580E090E008954F925F92F2
:106200006F927F928F929F92AF92BF92CF92DF92C6
:10621000EF92FF920F931F93CF93DF93CDB7DEB72B
:10622000CB57D0400FB6F894DEBF0FBECDBF2C01C8
:10623000633851F48BEA96E0EC966FAFEC970E94CE
:106240005838EC966FADEC97D2018D919C911197D7
:10625000B8E085369B07E9F0E8E086369E0718F43B
:10626000009761F09AC6F9E08F339F0709F46EC674
:1062700029E08634920709F090C681C68BEA96E041
:1062800061E870E049E155E00E943D3885E698E01C
:1062900071C6623109F086C60E94370B8091E8040E
:1062A0009091E90492FF02C00E94ED158091E804EC
:1062B0009091E90493FF0CC00E94EE0ADC01CB012F
:1062C00080935D2490935E24A0935F24B093602418
:1062D0008091E80480FF60C000D000D000D0EDB70E
:1062E000FEB7319672E0C72ED12CCC0EDD1EADB7B5
:1062F000BEB71296DC92CE92119788E790E0938316
:1063000082838AE793E0958384830E948D768C0153
:106310008AE6A82E84E2B82EEDB7FEB736960FB601
:10632000F894FEBF0FBEEDBFEE24FF2498E7892E40
:10633000912C2EE7622E23E0722ED5012D915D0166
:10634000EDB7FEB738970FB6F894FEBF0FBEEDBF9E
:106350003196C601800F911FADB7BEB712969C93C0
:106360008E9311979382828275826482268317822C
:106370000E948D76080F191F0894E11CF11CEDB7DF
:10638000FEB738960FB6F894FEBF0FBEEDBFF8E02B
:10639000EF16F10491F602C000E010E08091E804ED
:1063A0009091E904009781F12DB73EB72850304015
:1063B0000FB6F8943EBF0FBE2DBFEDB7FEB73196B6
:1063C000CE010296800F911FADB7BEB712969C9377
:1063D0008E93119788E790E09383828383E893E01C
:1063E0009583848380919506909196069783868302
:1063F0000E948D76080F191FEDB7FEB738960FB6BD
:10640000F894FEBF0FBEEDBF8091E80481FF51C03C
:1064100089E290E06BE270E04AE250E027E00E94FF
:1064200066428AE694E20E94CD442DB73EB72A50D8
:1064300030400FB6F8943EBF0FBE2DBFEDB6FEB68E
:106440000894E11CF11C9E012E5F3F4F200F311F6D
:10645000ADB7BEB712963C932E93119728E730E064
:10646000F701338322832AE833E0358324839C01B8
:10647000B901882777FD8095982F0E94BD6F20E095
:1064800030E048EC52E40E94536FDC01CB01F7018D
:1064900086839783A087B1870E948D76080F191F86
:1064A0002DB73EB7265F3F4F0FB6F8943EBF0FBEE5
:1064B0002DBF8091E80482FF57C089E290E06BE233
:1064C00070E04AE250E026E00E94664281E090E0FF
:1064D0000E94890B8093940689E697E10E94CD443F
:1064E0004DB75EB74A5050400FB6F8945EBF0FBE2E
:1064F0004DBFEDB6FEB60894E11CF11C9E012E5F67
:106500003F4F200F311FADB7BEB712963C932E936D
:10651000119728E730E0F7013383228324E933E041
:10652000358324839C01B901882777FD8095982FB6
:106530000E94BD6F20E030E048EC52E40E94536FAF
:10654000DC01CB01F70186839783A087B1870E9486
:106550008D76080F191F2DB73EB7265F3F4F0FB638
:10656000F8943EBF0FBE2DBF8091E80483FF36C074
:106570004DB75EB74A5050400FB6F8945EBF0FBE9D
:106580004DBFEDB7FEB73196CE010296800F911F39
:10659000ADB7BEB712969C938E93119788E790E0A3
:1065A000938382838FE993E0958384838091551749
:1065B00090915617A0915717B091581786839783DB
:1065C000A087B1870E948D76080F191FEDB7FEB71F
:1065D0003A960FB6F894FEBF0FBEEDBF8091E80467
:1065E00084FF32C00E94080BAB01BC012DB73EB73F
:1065F0002A5030400FB6F8943EBF0FBE2DBFEDB706
:10660000FEB73196CE010296800F911FADB7BEB78F
:1066100012969C938E93119788E790E093838283E0
:106620008DEA93E0958384834683578360877187DF
:106630000E948D76080F191FEDB7FEB73A960FB678
:10664000F894FEBF0FBEEDBF8091E80485FF38C00F
:10665000F89440915524509156246091572470919C
:10666000582478942DB73EB72A5030400FB6F8948E
:106670003EBF0FBE2DBFEDB7FEB73196CE010296DD
:10668000800F911FADB7BEB712969C938E93119752
:1066900088E790E0938382838BEB93E095838483F8
:1066A00046835783608771870E948D76080F191F74
:1066B000EDB7FEB73A960FB6F894FEBF0FBEEDBF2A
:1066C0008091E80486FF8DC08091E6049091E704F4
:1066D000009709F486C0F894809055249090562431
:1066E000A0905724B090582478948091611790918D
:1066F0006217A0916317B0916417A5019401281B3C
:10670000390B4A0B5B0BCA01B9010E94BB6FE62E25
:10671000C72EF82ED92E6091E6047091E70480E030
:1067200090E00E94BB6F9B01AC018E2D9C2DAF2D84
:10673000BD2DBC01CD010E94536FE82EC92E4DB76F
:106740005EB74A5050400FB6F8945EBF0FBE4DBFC3
:10675000EDB7FEB73196CE010296800F911FADB70F
:10676000BEB712969C938E93119788E790E093831F
:10677000828384EC93E095838483862F972FAE2DBC
:10678000BC2D86839783A087B187EC966FAFEC977B
:10679000EB967FAFEB970E948D76080F191FEC9652
:1067A0006FADEC97EB967FADEB97862F972FAE2DC5
:1067B000BC2D8093622490936324A0936424B093AF
:1067C00065248092611790926217A0926317B0922D
:1067D0006417EDB7FEB73A960FB6F894FEBF0FBE3A
:1067E000EDBF8091E80487FF3EC0F89440915924A2
:1067F00050915A2460915B2470915C2478942DB759
:106800003EB72A5030400FB6F8943EBF0FBE2DBFA2
:10681000EDB7FEB73196CE010296800F911FADB74E
:10682000BEB712969C938E93119788E790E093835E
:10683000828381ED93E095838483468357836087C9
:1068400071870E948D76080F191FEDB7FEB73A9633
:106850000FB6F894FEBF0FBEEDBFC8010E94CC304A
:10686000009709F013CD8091E8049091E90490FF1E
:106870008DC08091E6049091E704009709F486C0EA
:10688000F8948090592490905A24A0905B24B09062
:106890005C2478948091651790916617A091671792
:1068A000B0916817A5019401281B390B4A0B5B0BAB
:1068B000CA01B9010E94BB6FE62EC72EF82ED92E51
:1068C0006091E6047091E70480E090E00E94BB6F65
:1068D0009B01AC018E2D9C2DAF2DBD2DBC01CD019A
:1068E0000E94536FE82EC92E4DB75EB74A505040F4
:1068F0000FB6F8945EBF0FBE4DBFEDB7FEB7319631
:10690000CE010296800F911FADB7BEB712969C9331
:106910008E93119788E790E0938382838AED93E0CA
:1069200095838483862F972FAE2DBC2D86839783E6
:10693000A087B187EC966FAFEC97EB967FAFEB97A4
:106940000E948D76080F191FEC966FADEC97EB96B1
:106950007FADEB97862F972FAE2DBC2D80936624AD
:1069600090936724A0936824B0936924809265175C
:1069700090926617A0926717B0926817EDB7FEB7AE
:106980003A960FB6F894FEBF0FBEEDBF8091E804B3
:106990009091E90491FF3CC040910020509101206A
:1069A00060910220709103202DB73EB72A503040ED
:1069B0000FB6F8943EBF0FBE2DBFEDB7FEB73196B0
:1069C000CE010296800F911FADB7BEB712969C9371
:1069D0008E93119788E790E09383828387EE93E00C
:1069E0009583848346835783608771870E948D7661
:1069F000080F191FEDB7FEB73A960FB6F894FEBF11
:106A00000FBEEDBFC8010E94CC30009709F03ECC0C
:106A10008091E8049091E90492FF3CC02DB73EB705
:106A20002A5030400FB6F8943EBF0FBE2DBFEDB7D1
:106A3000FEB73196CE010296800F911FADB7BEB75B
:106A400012969C938E93119788E790E093838283AC
:106A500080EF93E0958384838091FA179091FB17E0
:106A6000A091FC17B091FD1786839783A087B1870B
:106A70000E948D76080F191FEDB7FEB73A960FB634
:106A8000F894FEBF0FBEEDBFC8010E94CC30009746
:106A900009F0FCCB8091E8049091E90493FF3CC09D
:106AA0002DB73EB72A5030400FB6F8943EBF0FBE08
:106AB0002DBFEDB7FEB73196CE010296800F911F24
:106AC000ADB7BEB712969C938E93119788E790E06E
:106AD000938382838BEF93E09583848380915D24FD
:106AE00090915E24A0915F24B09160248683978367
:106AF000A087B1870E948D76080F191FEDB7FEB7EA
:106B00003A960FB6F894FEBF0FBEEDBFC8010E94C3
:106B1000CC30009709F0BACB8091E8049091E90459
:106B200094FF4CC081E00E949A0AAB01BC012DB7D2
:106B30003EB72A5030400FB6F8943EBF0FBE2DBF6F
:106B4000EDB6FEB60894E11CF11CCE010296800F52
:106B5000911FADB7BEB712969C938E93119788E79D
:106B600090E0F7019383828388E094E095838483A7
:106B7000CB01BA012091050530910605409107052A
:106B8000509108050E946D70DC01CB01F7018683EE
:106B90009783A087B1870E948D76080F191F2DB7A4
:106BA0003EB7265F3F4F0FB6F8943EBF0FBE2DBFD6
:106BB000C8010E94CC30009709F068CB8091E804AE
:106BC0009091E90495FF4BC082E00E949A0AAB01C4
:106BD000BC018DB79EB70A970FB6F8949EBF0FBE43
:106BE0008DBFEDB6FEB60894E11CF11CCE010296F5
:106BF000800F911FADB7BEB712969C938E931197DD
:106C000088E790E0F7019383828385E194E09583A0
:106C10008483CB01BA012091010530910205409196
:106C20000305509104050E946D70DC01CB01F70152
:106C300086839783A087B1870E948D76080F191FDE
:106C40002DB73EB7265F3F4F0FB6F8943EBF0FBE3D
:106C50002DBFC8010E94CC30009709F017CB80915E
:106C6000E8049091E90496FF06C083E061E046E005
:106C700020E00E949A118091E8049091E90497FF26
:106C800006C083E061E046E021E00E949A11809115
:106C9000E8049091E90496FF3CC04DB75EB74A50B6
:106CA00050400FB6F8945EBF0FBE4DBFEDB7FEB7B4
:106CB0003196CE010296800F911FADB7BEB71296E6
:106CC0009C938E93119788E790E09383828382E26E
:106CD00094E0958384838091F1179091F217A091AD
:106CE000F317B091F41786839783A087B1870E942A
:106CF0008D76080F191FEDB7FEB73A960FB6F894C8
:106D0000FEBF0FBEEDBFC8010E94CC30009709F056
:106D1000BDCA8091E8049091E90497FF3CC02DB76B
:106D20003EB72A5030400FB6F8943EBF0FBE2DBF7D
:106D3000EDB7FEB73196CE010296800F911FADB729
:106D4000BEB712969C938E93119788E790E0938339
:106D500082838AE294E0958384838091F5179091F1
:106D6000F617A091F717B091F81786839783A0873D
:106D7000B1870E948D76080F191FEDB7FEB73A96BE
:106D80000FB6F894FEBF0FBEEDBFC8010E94CC3015
:106D9000009709F07BCA779A80919806909199069E
:106DA00093FD749A809198069091990682FD08C08F
:106DB0008091E40480FD04C081FF31C01D9B2FC081
:106DC00000D000D085E394E0ADB7BEB712969C9397
:106DD0008E931197CE01029614969C938E931397DF
:106DE0000E942676209100050F900F900F900F9033
:106DF0002223A9F000D000D0EDB7FEB731968BE882
:106E00009CE0ADB7BEB712969C938E9311972283E8
:106E100013820E9438760F900F900F900F90809100
:106E2000B6068983FE01E00FF11F12828091980659
:106E30009091990680FF12C000D000D08CE394E0BE
:106E4000EDB7FEB792838183C80102969483838352
:106E50000E9426760F900F900F900F9062E0C62E42
:106E6000D12CC00ED11ECE010196B6010E947241F6
:106E70008091E40482FF49C08AEE94E0BE016F5F16
:106E80007F4FA60125E530E20E94C7458091980614
:106E90009091990692FF39C045E5E42E40E2F42E28
:106EA00000E010E05DE4A52E54E0B52ED7018D91F1
:106EB0007D0100D000D0EDB7FEB73196ADB7BEB7BB
:106EC0001296BC92AE921197828313820E9426760C
:106ED0000F5F1F4F0F900F900F900F900031110513
:106EE00029F78AE090E00E94587600D000D082E531
:106EF00094E0EDB7FEB792838183D482C3820E946F
:106F000026760F900F900F900F9080919806909199
:106F1000990682FD73980E947A4C8BEA96E00E9453
:106F20005B388091950690919606009711F00E942B
:106F30006B4D8091B6068F5F8093B6068091980660
:106F40009091990682FFA2C9739AA0C987EB96E037
:106F50000E94DD3C009731F10E947A4C8091E4045C
:106F600087FD2B9887EB96E060E470E00E94B23CCE
:106F700086E499E0D20111969C938E9313C087EB1F
:106F800096E00E94DD3C009769F00E946B4D809175
:106F9000E40487FF7BC92B9A79C9F2011182108220
:106FA00083E001C081E0C558DF4F0FB6F894DEBF23
:106FB0000FBECDBFDF91CF911F910F91FF90EF904A
:106FC000DF90CF90BF90AF909F908F907F906F9009
:106FD0005F904F9008950895FC01DB018C918083B0
:106FE00011968C91119781830895FC01DB019081AA
:106FF0008C91981741F421E030E0918111968C91A9
:107000001197981711F020E030E0C9010895BC01F4
:107010008AE794E20E94EC370895DC011996ED911D
:10702000FC911A970280F381E02D309709F00995C1
:1070300008950F931F93CF93DF9300D0CDB7DEB7A2
:107040008C0188E10E94E141BC01CE0101960E94C1
:10705000EC37D8011996ED91FC911A970190F081C7
:10706000E02DC801BE016F5F7F4F09950F900F9013
:10707000DF91CF911F910F910895EF92FF920F939F
:107080001F93CF93DF93EC018B017A014FE155E021
:107090000E946938FA86E986C80163E275E00E94B9
:1070A000C738DF91CF911F910F91FF90EF90089516
:1070B0000E9482380895CF93DF93EC0188E16AE75C
:1070C00074E20E94D741CE010E948538DF91CF91B2
:1070D0000895EF92FF920F931F93CF93DF93EC01EC
:1070E0008B017A010E94A338F886EF82C80167E21B
:1070F00075E00E94C738DF91CF911F910F91FF90EB
:10710000EF9008950E94AC3808950E94E3520895CC
:10711000DC011796ED91FC9118970190F081E02D1C
:1071200009950895DC011796ED91FC91189702805E
:10713000F381E02D309709F00995089587E49EE0EA
:107140000E94163B0895FC017383628387E49EE0EE
:10715000BF010E94893B0895BC0187E49EE00E9424
:10716000543B0895CF93DF93EC0187E49EE00E94A7
:107170001A3B08C0FC01228133812C173D0721F006
:107180000E94C03B0097B1F7DF91CF9108950F9314
:107190001F93CF93DF938B010E94B238EC010097CD
:1071A00031F01D830C83C8010E9426558E83DF9128
:1071B000CF911F910F9108951F93CF93DF93EC010F
:1071C000162F888580FF1DC0EC81FD813097C9F0A6
:1071D000D0934A0EC093490E82E08887CE0106966E
:1071E0000995992787FD909502978230910510F0B7
:1071F000133829F4CE01BE010E94053902C081E096
:107200008887DF91CF911F910895CF92DF92EF92FF
:10721000FF920F931F93CF93DF93EC017B01C090FC
:10722000490ED0904A0E00914B0E10914C0EF80171
:1072300003C00190F081E02DEC17FD0719F03097A5
:10724000C1F746C0209709F443C08885882309F117
:1072500018860BC0C017D10729F0C80167E8AE0136
:107260000E94DC38F801008111810115110591F7A8
:10727000EC81FD81309769F0CE15DF0551F0D09398
:107280004A0EC093490ECE01069663E840E050E0F6
:107290000995E0914B0EF0914C0ECE17DF0791F45B
:1072A0008881998190934C0E80934B0E0DC0808104
:1072B00091818C179D0729F488819981918380831E
:1072C00003C0FC01309799F7D0924A0EC092490E44
:1072D000DF91CF911F910F91FF90EF90DF90CF90B2
:1072E00008951F93CF93DF9310924D0EC0914B0ED4
:1072F000D0914C0E11E00EC08985882341F018878B
:107300001986CE0162E840E050E00E94DC38099026
:10731000D881C02D209781F7DF91CF911F910895DB
:1073200080914E0E982F9F5F90934E0E089560911E
:10733000490E70914A0E0E94053908958AE880939B
:107340004E0E10924F0E1092500E10924C0E109244
:107350004B0E10924A0E1092490E089580914D0ED8
:10736000882311F00E9471397091500E772309F42F
:1073700055C020914F0E30E0F901EE0FFF1FEE0FC8
:10738000FF1FE20FF31FEF5AF14F60816093F10E80
:10739000418152815093F30E4093F20E8381948188
:1073A0009093F50E8093F40E2F5F3F4F2F71307046
:1073B00020934F0E71507093500E009741F58091BD
:1073C0004B0E90914C0E18C080914D0E882311F0F9
:1073D0000E9471394091F20E5091F30E8091F60E99
:1073E0009091F70E6091F10E0E94DC38E091F60E5C
:1073F000F091F70E808191819093F70E8093F60EB5
:107400008091F60E9091F70E0097F1F607C0613863
:1074100019F421E0FC0120870E94DC3880914D0E98
:107420002091500E90E0820F911D089580914D0E95
:107430002091500E90E0820F911D08959C01709153
:10744000500E7032D9F080914F0E870F8F7180935C
:10745000F80E90E0FC01EE0FFF1FEE0FFF1FE80F8C
:10746000F91FEF5AF14F60835283418334832383A2
:107470007F5F7093500E80E090E0089581E090E08F
:107480000895CF93DF93C091490ED0914A0E0E9488
:10749000DC38D0934A0EC093490EDF91CF91089506
:1074A000FC01AB0190914B0E80914C0EA92FB82F8F
:1074B00003C00D90BC91A02DAE17BF0791F010979F
:1074C000C1F7309771F090838183F0934C0EE09375
:1074D0004B0E81E0808717821682CF0161E80E94FF
:1074E000413A0895FC01009741F080858150823037
:1074F00020F481E0818780934D0E089521E030E0F3
:10750000FC018085882311F420E030E0C901089552
:10751000CF93DF93EC014A815B818C819D8160E098
:1075200070E00E94B0752A813B8188819981289FF3
:10753000A001299F500D389F500D11248E819F81ED
:1075400060E070E00E94B075DF91CF910895DC019A
:1075500012962D913C91139780E090E01DC01496F7
:10756000ED91FC911597E80FF91F4081442399F4A0
:1075700021E020832D913C911197829FA001839F50
:10758000500D929F500D112416968D919C91179736
:10759000840F951F089501968217930701F780E0E5
:1075A00090E00895FC0146815781A281B38120E0DB
:1075B00030E019C04617570781F4A481B581A20FA6
:1075C000B31F8C91181614F481508C930480F581AC
:1075D000E02DE20FF31F8081089580819181480F93
:1075E000591F2F5F3F4F2A173B0721F78FEF089551
:1075F000FC014681578164177507A8F0A081B1810D
:1076000082819381A89F9001A99F300DB89F300D72
:107610001124240F351F81E090E06217730728F0D2
:1076200080E090E0089580E090E00895FC011182F0
:1076300010820895FC01808191810895FB012081D1
:107640003181FC01318320830895FC018081918187
:10765000009711F40895C901FC01208131812115A1
:107660003105C9F70895DC01ED91FC911197309730
:1076700029F40BC0DF010190F081E02D8081918120
:107680000097C1F711961C921E92CF010895DC015C
:10769000ED91FC911197309729F08081918111969D
:1076A0009C938E93CF010895CF93DF93EC01E881F3
:1076B000F9813097B9F0A0E0B0E002C0DF01FC0131
:1076C00080819181E617F70759F4109719F499838F
:1076D000888303C011969C938E931182108202C0FE
:1076E000009761F7DF91CF9108950F931F93CF9388
:1076F000DF938C01EB010E94543BF8018081918162
:1077000099838883D183C083DF91CF911F910F919B
:1077100008950F931F93CF93DF938C01EB010E9489
:10772000543B19821882C8010E94253B009711F42E
:10773000F80101C0FC01D183C083DF91CF911F917B
:107740000F910895DC01ED91FC91119780E090E09C
:1077500004C001960190F081E02D3097D1F7089593
:10776000FB01BA01309719F40E94753B089580819E
:107770009181DA0111969C938E93518340830895F1
:10778000009721F0FC0180819181089580E090E0D4
:1077900008958091F90E9091FA0E009729F41092B5
:1077A000FC0E1092FB0E08950E94EB49BC01E09183
:1077B000F90EF091FA0E4281538180819181480F38
:1077C000591F461B570B0CC0828193812081318148
:1077D000820F931F861B970B8417950708F4AC0143
:1077E0000480F581E02D309779F7460F571F5093AD
:1077F000FC0E4093FB0E089585E395E00E94723ADB
:107800000895EF92FF920F931F93CF93DF937C0124
:10781000FC0180819181009729F08A35910509F05A
:107820006DC00BC01092FA0E1092F90E8AE590E02E
:10783000F7019183808381E065C0673859F5A09195
:10784000F90EB091FA0E04C014960D90BC91A02DC3
:10785000109741F316968D919C9117978417950771
:1078600099F3A093F90EB093FA0E0DC0868197811B
:107870008417950739F48481958115969C938E938E
:107880001497FD01DF011496ED91FC911597309747
:1078900069F7CCCF623851F6C091F90ED091FA0E4B
:1078A00000E010E028C0CE010E940B590097F1F0D3
:1078B0008E819F8168E8AE010E941E3A0097A1F474
:1078C0001F821E828C819D810115110521F0F80116
:1078D0009583848304C09093FA0E8093F90E1D82E1
:1078E0001C820E94C93BD8CF0E94FC3B9C818D81A9
:1078F0008E01C92FD82F2097B1F698CFF7011182AA
:10790000108283E0DF91CF911F910F91FF90EF9054
:107910000895CF93DF93EC010E94FC3B8E819F8101
:107920003091F90E2091FA0E009759F0E32FF22FC3
:1079300006C0EC17FD0789F00480F581E02D309733
:10794000C1F78091490E90914A0E9F838E833C83AC
:107950002D83D093FA0EC093F90E0E94C93BDF919C
:10796000CF910895CF93DF93EC010E94EB58CE01A5
:107970000E94893CDF91CF910895CF93DF93EC0172
:107980000E94F758CE010E94893CDF91CF91089563
:10799000CF93DF93EC010E940159CE010E94893CF4
:1079A000DF91CF910895FC0180819181860F971F0F
:1079B000918380830E94C93B089521E030E0FC015F
:1079C00086819781009711F020E030E0C901089589
:1079D000FC012281338180819181280F391FC901E7
:1079E0000895FC0180819181089581E090E02091CB
:1079F000F90E3091FA0E2115310511F480E090E076
:107A000008958091F90E9091FA0E009729F08091D7
:107A1000FB0E9091FC0E089580E090E00895CF93C6
:107A2000DF93EC01E091F90EF091FA0E8E179F07AB
:107A300041F48C819D819093FA0E8093F90E14C0CD
:107A4000FC01309731F0848195818C179D07C1F737
:107A500007C01D821C821F821E82DF91CF91089574
:107A60008C819D81958384830E94C93BF2CFEF92E4
:107A7000FF920F931F93CF93DF937C018A01FC0148
:107A800080819181009729F08B34910509F049C0DC
:107A90001AC08EEF9EE00E941A3BEC0109C06C8177
:107AA0007D81CE0102960E94B23C0990D881C02D02
:107AB0002097A9F781E08093FD0E8BE490E0F70119
:107AC0009183808333C0683889F58EEF9EE00E94F1
:107AD0001A3BEC0123C0CE01029608171907D9F40E
:107AE0008EEF9EE0BE010E94543B0091490E109122
:107AF0004A0E8A859B8590934A0E8093490EEC85A9
:107B0000FD85309719F08E859F85099510934A0E53
:107B10000093490ED2CF0990D881C02D2097D9F675
:107B2000CCCFF7011182108283E001C081E0DF91A8
:107B3000CF911F910F91FF90EF9008951092FD0E3D
:107B40008EEF9EE00E94163B8EE495E060E070E0D0
:107B50000E94503A08950F931F93CF93DF93EC0147
:107B60000091490E10914A0E1B870A875D874C874A
:107B70003F872E878091FD0E882379F08EE495E073
:107B800090934A0E8093490ECE0102960E94B23C19
:107B900010934A0E0093490E02C07D836C838EEFD2
:107BA0009EE0BE010E94543B8EEF9EE0BE010E940B
:107BB000893BDF91CF911F910F9108950F931F93F0
:107BC000CF93DF93EC018091FD0E882391F000911B
:107BD000490E10914A0E8EE495E090934A0E8093E0
:107BE000490ECE0102960E94BD3C10934A0E0093AE
:107BF000490E8EEF9EE0BE010E94543B8EEF9EE048
:107C0000BE010E94893BDF91CF911F910F91089592
:107C10000F931F93CF93DF93EC018091FD0E882388
:107C200091F00091490E10914A0E8EE495E09093E8
:107C30004A0E8093490ECE0102960E94C83C1093D2
:107C40004A0E0093490E8EEF9EE0BE010E94543B07
:107C50008EEF9EE0BE010E94893BDF91CF911F9184
:107C60000F910895CF93DF93EC018091FD0E88234F
:107C700029F0CE0102960E940F3D04C01F821E8291
:107C8000198618868EEF9EE0BE010E94543BDF915C
:107C9000CF910895CF93DF93EC018091FD0E88235F
:107CA00029F0CE0102960E94DD3C12C08EEF9EE0CC
:107CB0000E941A3B06C08C179D0741F0FC01808191
:107CC00091810097C1F781E090E002C080E090E0F0
:107CD000DF91CF910895CF93DF93D0917A24C09113
:107CE0007B240E94174AAB01BC018DB79EB7825519
:107CF00090400FB6F8949EBF0FBE8DBFEDB7FEB794
:107D0000319686EA9CE0ADB7BEB712969C938E93EF
:107D10001197D2831382C483158246835783608769
:107D2000718780916D2690916E26A0916F26B091FB
:107D3000702682879387A487B5878091712690915A
:107D40007226A0917326B091742686879787A08BA0
:107D5000B18B8091752690917626A0917726B0916F
:107D60007826828B938BA48BB58B8091792690910A
:107D70007A26A0917B26B0917C26868B978BA08F4C
:107D8000B18F80917D2690917E26A0917F26B09123
:107D90008026828F938FA48FB58F809181269091BA
:107DA0008226A0918326B0918426868F978FA0A3E8
:107DB000B1A38091852690918626A0918726B091C7
:107DC000882682A393A3A4A3B5A38091892690912A
:107DD0008A26A0918B26B0918C2686A397A3A0A774
:107DE000B1A780918D2690918E26A0918F26B0917B
:107DF000902682A793A7A4A7B5A7809191269091DA
:107E00009226A0919326B091942686A797A7A0AB1F
:107E1000B1AB8091952690919626A0919726B0912E
:107E2000982682AB93ABA4ABB5AB80919926909189
:107E30009A26A0919B26B0919C2686AB97ABA0AFCB
:107E4000B1AF80919D2690919E26A0919F26B091E2
:107E5000A02682AF93AFA4AFB5AFEDB7FEB7FF9644
:107E60008091A1269091A226A091A326B091A4264C
:107E700080839183A283B383EDB7FEB7ED5BFF4FA1
:107E80008091A5269091A626A091A726B091A8261C
:107E900080839183A283B383EDB7FEB7E95BFF4F85
:107EA0008091A9269091AA26A091AB26B091AC26EC
:107EB00080839183A283B383EDB7FEB7E55BFF4F69
:107EC0008091AD269091AE26A091AF26B091B026BC
:107ED00080839183A283B383EDB7FEB7E15BFF4F4D
:107EE0008091B1269091B226A091B326B091B4268C
:107EF00080839183A283B3830E943876D0917A24C1
:107F0000C0917B248DB79EB78E5A9F4F0FB6F894C1
:107F10009EBF0FBE8DBF0E94174AAB01BC01ADB71B
:107F2000BEB7D2970FB6F894BEBF0FBEADBFEDB7C8
:107F3000FEB7319682E89DE012969C938E9311973E
:107F4000D2831382C48315824683578360877187E7
:107F50008091B5269091B626A091B726B091B8260B
:107F600082879387A487B5878091B9269091BA2696
:107F7000A091BB26B091BC2686879787A08BB18B3A
:107F80008091BD269091BE26A091BF26B091C026BB
:107F9000828B938BA48BB58B8091C1269091C22646
:107FA000A091C326B091C426868B978BA08FB18FEA
:107FB0008091C5269091C626A091C726B091C8266B
:107FC000828F938FA48FB58F8091C9269091CA26F6
:107FD000A091CB26B091CC26868F978FA0A3B1A37A
:107FE0008091CD269091CE26A091CF26B091D0261B
:107FF00082A393A3A4A3B5A38091D1269091D22666
:10800000A091D326B091D42686A397A3A0A7B1A709
:108010008091DD269091DE26A091DF26B091E026AA
:1080200082A793A7A4A7B5A78091E1269091E22605
:10803000A091E326B091E42686A797A7A0ABB1ABA9
:108040000E9438768DB79EB7C2960FB6F8949EBF41
:108050000FBE8DBFDF91CF91089580E38093040F11
:108060000895CF93DF936091040F70E0C0E3D0E0F8
:10807000C61BD70B695F704FAE010E94A775CE017A
:10808000DF91CF910895CF92DF92EF92FF920F93FD
:108090001F93CF93DF937C01C090020FD090030F0A
:1080A0006091040F70E08601005D1F4F061B170BE7
:1080B00001381105D8F4C0E3D0E0C61BD70B695FC7
:1080C000704FAE010E94A775C7018C0F9D1F609174
:1080D000050F7091060F2091000F3091010F620F74
:1080E000731FA6010E94A775C80102C080E090E03E
:1080F000DF91CF911F910F91FF90EF90DF90CF9084
:1081000008959091040F980F9093040F0895409153
:10811000020F5091030F9C014817590798F0809166
:10812000000F9091010F820F931F9093010F809386
:10813000000F421B530B5093030F4093020F81E03B
:1081400090E0089580E090E008959093030F80936D
:10815000020F08958091000F9091010F895C904F5C
:1081600008958091040F90E0895F904F089581E019
:1081700090E02091050F3091060F4FE02733340730
:1081800011F480E090E008950E94B740009769F0F4
:1081900087E39FE06091050F7091060F4091020FF9
:1081A0005091030F0E94A77508954091000F5091C0
:1081B000010F41155105C1F08091020F9091030FFD
:1081C000C096A7E3BFE020E330E007C0FD01E40F65
:1081D000F51F60816D932F5F3F4F28173907B4F368
:1081E0001092010F1092000F08958091050F909149
:1081F000060F08958091020F9091030F08959091BA
:10820000040F80E3891B089520E38091040F281B4D
:108210008091020F9091030F820F911D08951F937B
:10822000CF93DF93EC011091040F812F90E08C1716
:108230009D076CF00E9404418C0F9D1F81389105B1
:1082400030F41C1B1093040F81E090E002C080E02A
:1082500090E0DF91CF911F910895CF93DF93E4E8F1
:10826000F4E21192119284E2E43BF807D1F7C0E006
:10827000D0E0CE01880F991F84589B4D6DE175E0C9
:108280000E94EC372196C430D10599F7DF91CF9148
:1082900008951092010F1092000F1092030F109288
:1082A000020F80E38093040F87E39FE09093060F13
:1082B0008093050F0E942D4108950F931F93CF9334
:1082C000DF93EC018B010E944941D093060FC093CC
:1082D000050F1093030F0093020FDF91CF911F91B1
:1082E0000F910895EF92FF920F931F93CF93DF9317
:1082F00000D0CDB7DEB78C0169837A830E944941F3
:108300006981E62E7A81F72E81E8E816F10418F0EB
:1083100030E8E32EF12C8091050F9091060FB80103
:10832000A7010E94A775F092030FE092020FC70108
:108330000F900F90DF91CF911F910F91FF90EF90D1
:108340000895FC01A4E8B4E280E30D90019281500D
:10835000E1F7FB01ACE7B4E288E00D9001928150B7
:10836000E1F70895A4E8B4E2FC0180E301900D92E6
:108370008150E1F7ACE7B4E2FB0188E001900D9297
:108380008150E1F70895E82FF0E0EE0FFF1FEC5762
:10839000FB4D7183608381E090E00895E82FF0E069
:1083A000EE0FFF1FEC57FB4D80819181089590E007
:1083B000880F991F845B9B4D0E94EC3781E090E011
:1083C000089590E0880F991F845B9B4D0895811557
:1083D000910511F00197F1F70895E091B724F0911C
:1083E000B82490818091B62489230895E091B42423
:1083F000F091B52480819091B624892B8083E091FF
:10840000B924F091BA2480819091B624892B80837D
:108410000895E091B424F091B52490818091B62420
:10842000809589238083E091B924F091BA249081CA
:108430008091B62480958923808308951F93CF93DC
:10844000DF93E091B424F091B52490818091B6241B
:10845000809589238083E091B924F091BA248081AA
:108460009091B624892B80838FEB93E00E94E741A3
:108470001FB7F894E091B924F091BA2490818091CB
:10848000B62480958923808383E890E00E94E741A9
:10849000E091B724F091B824D081C091B6241FBFD9
:1084A00078948BE393E00E94E741E091B724F09148
:1084B000B82480819091B624892319F08D2F8C23C4
:1084C00001C081E0DF91CF911F9108955093BA24AC
:1084D0004093B9247093B5246093B4249093B82446
:1084E0008093B72481E090E002C0880F991F2A95FD
:1084F000E2F78093B6240E941E420895CF93DF9343
:10850000C82FDFB7F894E091B924F091BA248081A4
:108510009091B624892B808383E090E00E94E7410C
:10852000CC2351F0E091B924F091BA24908180914C
:10853000B62480958923808387E190E00E94E741FB
:10854000E091B724F091B82480819091B6248923DA
:1085500009F4C0E089E590E00E94E741E091B92488
:10856000F091BA2490818091B624809589238083EC
:10857000DFBF8BE390E00E94E7418C2FDF91CF912A
:108580000895CF93DF93C82FD8E08C2F81700E947D
:108590007E42C6958111C068D150B9F78C2FDF910A
:1085A000CF9108958FEF0E94C1420895DF92EF921C
:1085B000FF920F931F93CF93DF93182FEB010E942D
:1085C0001E42882381F580EF0E94C142EE2400E420
:1085D00098E0D92E81E00E947E42F82E81E00E9430
:1085E0007E42882319F0FF2069F020C0FF2051F45B
:1085F000011728F0888180FF05C0101719F0E02EC0
:10860000FF24F3948F2D0E947E4288818695888373
:10861000FF2011F0806888830150DA94D9F6219602
:108620000023B1F605C0EE24EA9402C08EEFE82ED6
:108630008E2DDF91CF911F910F91FF90EF90DF90E2
:1086400008950F931F93CF93DF93182FEB010E9490
:108650001E42209751F085E50E94C14208E08991B1
:108660000E94C1420150D9F703C08CEC0E94C14264
:10867000812F0E94C142DF91CF911F910F910895E8
:108680000F931F93CF93DF93E82FDB01EA01B9012A
:108690004C9150E011969C91119780E0482B592BFA
:1086A000E03181F4CA018E7F33E0880F991F3A953B
:1086B000E1F716962C9116974CE050E0421B5109B9
:1086C000480F591F57FF06C081E088835095419598
:1086D0005F4F01C01882E83299F414968C91149778
:1086E00090E09C01207630702036310549F086FFFD
:1086F00002C04E7F05C085FF02C04C7F01C0487F8D
:10870000CA0124E0969587952A95E1F7FB018083BD
:108710004F70F801408380E0DF91CF911F910F915E
:1087200008950F931F93CF93DF93EC018B01888102
:10873000B8010E94D642888381508D3F30F4F80101
:108740008081883211F0803191F7DF91CF911F91B4
:108750000F910895CF93DF93EC010E941E4284EBAA
:10876000BE010E94214381E00E947E42C82F0E94E8
:108770001E4281E0CC2309F480E0DF91CF9108957F
:108780001F93CF93DF93182FEB010E941E420E948C
:10879000ED41882349F084E4BE010E942143113059
:1087A00029F00E94F64102C082E001C080E0DF9122
:1087B000CF911F9108956F927F928F929F92BF9257
:1087C000CF92DF92EF92FF920F931F93CF93DF939D
:1087D000CDB7DEB729970FB6F894DEBF0FBECDBF79
:1087E0007C014B013A0169010E941E428EEBB701E8
:1087F0000E9421438E010F5F1F4FE9E0BE2E0E94B1
:10880000D242F80181938F01BA94C9F7CE01019643
:1088100069E070E00E94A55D882361F4F701808122
:10882000BE016F5F7F4FA401930186010E94404308
:1088300080E001C083E029960FB6F894DEBF0FBE3A
:10884000CDBFDF91CF911F910F91FF90EF90DF90FF
:10885000CF90BF909F908F907F906F9008958F9250
:108860009F92AF92BF92CF92DF92EF92FF920F93BF
:108870001F93CF93DF93CDB7DEB729970FB6F89448
:10888000DEBF0FBECDBFD82E5B014A0179018EEB52
:1088900060E070E00E9421438E010F5F1F4FF9E0FE
:1088A000CF2E0E94D242F80181938F01CA94C9F75A
:1088B000CE01019669E070E00E94A55D882359F41D
:1088C0008D2DBE016F5F7F4FA501940187010E942E
:1088D000404380E001C083E029960FB6F894DEBFE4
:1088E0000FBECDBFDF91CF911F910F91FF90EF9001
:1088F000DF90CF90BF90AF909F908F900895EF92B0
:10890000FF921F93CF93DF93CDB7DEB728970FB6B3
:10891000F894DEBF0FBECDBF182F262FDE011196B3
:10892000E8E5F5E088E001900D928150E1F7E42E52
:10893000FF24E7FCF09441E752E0E49EC001E59E8D
:10894000900DF49E900D112464E670E00E94687210
:10895000CB0134E6239F90011124820F931FFE0167
:10896000319640E0219130E0E216F30611F40196D1
:1089700003C04F5F4830B1F7112319F090958195EE
:108980009F4F28960FB6F894DEBF0FBECDBFDF9184
:10899000CF911F91FF90EF9008950F931F93CF9366
:1089A000DF93CDB7DEB72B970FB6F894DEBF0FBEBF
:1089B000CDBF182F092F885F612F792F0E94C043E8
:1089C000882309F048C066E471E48FE090E00E94DB
:1089D0003845812F902FBE016D5F7F4FAE014E5FF6
:1089E0005F4F9E012F5F3F4F0E94DB43882399F525
:1089F000DE011496E8E5F5E088E001900D928150E3
:108A0000E1F7E9814E2F50E021E732E0429FC001BB
:108A1000439F900D529F900D112464E670E00E94D8
:108A20006872CB013A8124E6329F90011124820FB3
:108A3000931FDE01149620E03D91E31711F4019697
:108A400003C02F5F2830C1F72B81222331F090958E
:108A500081959F4F02C084E391E22B960FB6F89464
:108A6000DEBF0FBECDBFDF91CF911F910F91089553
:108A7000DC01CB0181159105A105B10529F08150DB
:108A80009040A040B040D9F708951092B90080E21C
:108A90008093B800089594EA9093BC009091BC0034
:108AA00097FFFCCF9091B900987F983011F09031EA
:108AB00099F48093BB0084E88093BC008091BC0053
:108AC00087FFFCCF9091B900987F983139F081E011
:108AD000903429F480E0089581E0089580E00895BD
:108AE00044EA34E824E94093BC009091BC0097FF2D
:108AF000FCCF9091B900987F983011F0903199F7A0
:108B00008093BB003093BC009091BC0097FFFCCFDA
:108B10009091B900987F903211F0983539F42093F4
:108B2000BC009091BC0094FDFCCFDDCF08950E9465
:108B30004B45089584E98093BC008091BC0084FD7E
:108B4000FCCF08958093BB0084E88093BC008091A3
:108B5000BC0087FFFCCF9091B900987F81E09832EC
:108B600009F480E0089584EC8093BC008091BC00FF
:108B700087FFFCCF8091BB00089584E88093BC0000
:108B80008091BC0087FFFCCF8091BB000895FC0161
:108B900080E1919190933F018150D9F780913C0100
:108BA0008F7D80933C0180913C01877F80933C01C5
:108BB000FB0180E1919190933E018150D9F7809122
:108BC0003C01806880933C0180913D0180FFFCCF97
:108BD0004051504080913C01806280933C018091E3
:108BE0003C01877F80933C0112C0FB0180E19191A1
:108BF00090933E018150D9F780913C018068809329
:108C00003C0180913D0180FFFCCF40515040141643
:108C100015065CF3F90180E190913E01919381503A
:108C2000D9F781E090E008950F931F93CF93DF93DE
:108C30008C018CE70E9470458CE70E94A245C0E140
:108C4000D0E0F80181918F010E94A2452197C9F7D8
:108C50000E949A45DF91CF911F910F910895813025
:108C600039F48CE790E060E070E040E050E006C04E
:108C70008CE790E060E070E040EC50E00E9468100B
:108C80000895813039F48CE790E060E070E04EE0C8
:108C900050E006C08CE790E060E070E048E050E013
:108CA0000E94681008958CE790E060E070E041E079
:108CB00050E00E9468106AE67AE080E090E00E944E
:108CC000384508958CE790E060E070E048E350E0BC
:108CD0000E9468108CE790E060E070E049E350E0AB
:108CE0000E9468108CE790E060E070E044E150E0A2
:108CF0000E9468108CE790E060E070E048E750E088
:108D00000E9468108CE790E060E070E04EE550E073
:108D10000E9468108CE790E060E070E04DE650E063
:108D20000E9468106CE17AE186E090E00E9438458C
:108D30008CE790E060E070E04CE050E00E9468104A
:108D40008CE790E060E070E041E050E00E94681045
:108D50008CE790E060E070E046E050E00E94681030
:108D60006AE67AE080E090E00E9438450895CF936B
:108D7000DF93CDB7DEB7A2970FB6F894DEBF0FBE74
:108D8000CDBFDE015296E0E6F5E081E101900D9263
:108D90008150E1F7DE011196E1E7F5E081E1019014
:108DA0000D928150E1F70E946246CE0142960E94E8
:108DB000144682E00E942F466AE67AE080E090E066
:108DC0000E943845CE0101960E94144660E17EEA79
:108DD00088E290E00E94384580E00E94414660E1D0
:108DE0007EEA88E290E00E94384581E00E94414698
:108DF000A2960FB6F894DEBF0FBECDBFDF91CF9124
:108E00000895E6E4F1E080812081908130818295AF
:108E100086958695837022952F70822B832B929551
:108E20009F70892B0895DF92EF92FF920F931F930B
:108E3000CF93DF9300D0CDB7DEB780E06CE046E0A3
:108E40000E94AF4A89E18093C4001092C50082E07D
:108E50008093C00080E00E94514B0E94DB4984B7A0
:108E600084B784B784B784B7EBE3FDE222E432E44D
:108E7000318320833A968DB79EB70A97E817F90792
:108E8000B8F300D000D081EF9DE0ADB7BEB7129629
:108E90009C938E93119782E895E014969C938E9301
:108EA00013970E9438760F900F900F900F900E94AA
:108EB000D6590E949E3985E395E060E070E00E94FB
:108EC000503A0E949E3DE091CD05F091CE05099566
:108ED0000E94014790E00E94135ACE0101960E9421
:108EE0000D49882359F000D08CE09EE0EDB7FEB725
:108EF000928381830E9438760F900F90CE01019665
:108F00000E9407380E9417498C010E941C49BC012D
:108F1000C801AE014F5F5F4F0E944B4E0E947A48DE
:108F20000E94304E0E9421490E94CC4F00D08CE21A
:108F30009EE0ADB7BEB712969C938E9311970E9498
:108F4000387600D0EDB7FEB7319609E31EE0ADB735
:108F5000BEB712961C930E9311978A818283138257
:108F60000E943876EDB7FEB73196ADB7BEB7129610
:108F70001C930E9311978981828313820E94387605
:108F80000F900F908DE39EE0EDB7FEB79283818343
:108F90000E9438760F900F900E94195AE091500667
:108FA000F09151060995E0913706F0913806099540
:108FB000E091F905F091FA050995009135061091B7
:108FC0003606E0904E06F0904F060E942D4ED82EA9
:108FD0000E94D44F2DB73EB72A5030400FB6F894B8
:108FE0003EBF0FBE2DBFEDB7FEB731962FE33EE07B
:108FF000ADB7BEB712963C932E931197138302839D
:10900000F582E482D6821782808711860E943876A4
:10901000E0915A06F0915B062DB73EB7265F3F4FB1
:109020000FB6F8943EBF0FBE2DBF3097D1F0099513
:10903000BC0100D000D08AE59EE0ADB7BEB7129665
:109040009C938E93119780E890E00E945472EDB744
:10905000FEB7748363830E9438760F900F900F9051
:109060000F9000D08DE69EE0ADB7BEB712969C93F0
:109070008E9311970E9438760F900F9089E796E0B3
:1090800060E070E00E94503A8AE594E00E94CF5878
:1090900000D08FE69EE0EDB7FEB7928381830E94F9
:1090A00038760F900F900F900F90DF91CF911F9116
:1090B0000F91FF90EF90DF90089500D000D000D086
:1090C000EDB7FEB7319627E73EE0ADB7BEB71296D3
:1090D0003C932E93119793838283758364830E94BC
:1090E00038768DB79EB706960FB6F8949EBF0FBE22
:1090F0008DBF08950F931F93CF93DF93CDB7DEB746
:10910000A0970FB6F894DEBF0FBECDBF83E290E00C
:109110000E947877082F282F2B50203108F0982FA5
:109120009095891709F46DC000D08DE99EE0ADB728
:10913000BEB712969C938E9311970E9438768E013B
:109140000F5F1F4F0F900F90D80180E090E0FC015F
:10915000EB56F14FE491ED93019688309105B9F704
:10916000F894CE0101966FE370E048E050E00E9471
:109170007E77D80180E090E0FC01E957F14FE4915F
:10918000ED9301968E309105B9F7CE01019661E31A
:1091900070E04EE050E00E947E7780E090E0FC01BD
:1091A000E358F14FE491D801ED938D0101968A3097
:1091B0009105A9F7CE01019667E270E04AE050E020
:1091C0000E947E7781E290E06DEC7BEA0E949677C8
:1091D0008FE190E060E070E00E9496778EE190E091
:1091E00060E00E94887785E290E060E070E00E9495
:1091F00096770AE183E290E06AE175EE0E94967745
:109200007894802FA0960FB6F894DEBF0FBECDBF26
:10921000DF91CF911F910F910895F8946FE370E063
:1092200042E050E00E946077789480E0089581E207
:1092300090E00E94787708958FE190E00E9478771F
:1092400008958EE190E00E94707708954091C924BE
:109250005091CA246091CB247091CC2490E0A0E07E
:10926000B0E0480F591F6A1F7B1F4093C9245093D9
:10927000CA246093CB247093CC244091C524509190
:10928000C6246091C7247091C824480F591F6A1FD3
:109290007B1F4093C5245093C6246093C7247093CA
:1092A000C824209169262223A1F04091C124509125
:1092B000C2246091C3247091C424480F591F6A1FAF
:1092C0007B1F4093C1245093C2246093C3247093A6
:1092D000C42408951F920F920FB60F920BB60F92EF
:1092E00011242F933F934F935F936F937F938F93AB
:1092F0009F93AF93BF93EF93FF938091BB0F909198
:10930000BC0F01969093BC0F8093BB0F8091BA0F56
:109310008F5F8093BA0F8038A9F41092BA0F8091B2
:10932000C9249091CA24A091CB24B091CC24019659
:10933000A11DB11D8093C9249093CA24A093CB246E
:10934000B093CC24809169268823E1F08091B90FF5
:109350008F5F8093B90F8038A9F41092B90F809174
:10936000C1249091C224A091C324B091C424019639
:10937000A11DB11D8093C1249093C224A093C32446
:10938000B093C4240E94F53C009711F00E94FC3B6E
:10939000FF91EF91BF91AF919F918F917F916F91CD
:1093A0005F914F913F912F910F900BBE0F900FBE89
:1093B0000F901F901895F8941092B60016BC83EF8A
:1093C00087BD82E084BD94E095BD95B395BB809345
:1093D0006E00789408958091BB0F9091BC0F2091FE
:1093E000BB0F3091BC0F82179307A9F7089507C0F0
:1093F00022E330E0000021503040E1F70197009770
:10940000B9F708950F931F93CF93DF938C010E94B8
:10941000EB49EC010E94EB498C1B9D0B80179107D7
:10942000C8F3DF91CF911F910F91089508950F9385
:109430001F930091C9241091CA242091CB2430910C
:10944000CC248091C9249091CA24A091CB24B091BE
:10945000CC24081719072A073B0759F7B801C90197
:109460001F910F9108951F920F920FB60F92112422
:10947000109298050F900FBE0F901F9018951F9295
:109480000F920FB60F920BB60F9211242F933F93AA
:109490004F935F936F937F938F939F93AF93BF93FC
:1094A000EF93FF93E0918E05F0918F058081E0911D
:1094B0009905F0919A05309709F00995FF91EF9180
:1094C000BF91AF919F918F917F916F915F914F91DC
:1094D0003F912F910F900BBE0F900FBE0F901F90DA
:1094E00018951F920F920FB60F9211241092A50596
:1094F0000F900FBE0F901F9018951F920F920FB6EE
:109500000F920BB60F9211242F933F934F935F93BB
:109510006F937F938F939F93AF93BF93EF93FF933B
:10952000E0919B05F0919C058081E091A605F0916A
:10953000A705309709F00995FF91EF91BF91AF9181
:109540009F918F917F916F915F914F913F912F915B
:109550000F900BBE0F900FBE0F901F90189590E0CC
:109560002DE030E0829FF001839FF00D929FF00D7F
:109570001124E257FA4FA281B3811C92A481B581D4
:109580006C93A681B78188ED8C93A085B1854C93AF
:10959000128614861386089590E02DE030E0829FB5
:1095A000F001839FF00D929FF00D1124E257FA4FC6
:1095B00081E08287A081B1816C933A968081882373
:1095C000E9F70895CF93C82F8A3031F48091FD0FC9
:1095D0006DE00E94CC4A02C08D3029F08091FD0FD1
:1095E0006C2F0E94CC4A80E090E0CF9108951F93A9
:1095F000CF93DF93182FEB010CC08A3021F4812F19
:109600006DE00E94CC4A69916D3019F0812F0E9463
:10961000CC4A8881882389F7DF91CF911F910895E3
:109620000F931F93CF93DF93CDB7DEB79E01265FD5
:109630003F4F0DEB1FE0C80160E470E0488559859D
:109640000E94CA768F81B8010E94F74ADF91CF91BC
:109650001F910F9108951F93CF93DF93182FEB0164
:1096600004C0812F0E94CC4A2196FE01649166239A
:10967000C1F7DF91CF911F91089590E02DE030E088
:10968000829FF001839FF00D929FF00D1124E2570D
:10969000FA4F748763870895682F80E00E94CC4A50
:1096A00008958093FD0F88EA95E09093362D80937E
:1096B000352D089584B7877F84BF88E10FB6F8946D
:1096C00080936000109260000FBE08952FE088E143
:1096D00090E00FB6F894A895809360000FBE209399
:1096E00060000895A895089588E10FB6F8948093D6
:1096F0006000109260000FBE0895F89428E088E1A1
:1097000090E00FB6F894A895809360000FBE209368
:109710006000FFCF8091D4248091D42490E00895FC
:109720008091390181FD10C081E491E06FE140E05A
:109730000E946B51813059F021E030E0813111F00D
:1097400020E030E0C901089580E090E0089581E0D4
:1097500090E0089581E491E06FE140E00E946B5158
:109760000895E9E3F1E0808180818D7F80838DE041
:1097700090E00197F1F782E491E06FE140E023E0AF
:109780000E94755183E090E00197F1F70895909160
:10979000390191FD0AC0282F803108F02FE085E4BF
:1097A00091E06FE040E00E94755108958091390189
:1097B00081FD13C081E491E06FE140E00E946B51B4
:1097C000982F8151823038F09F3129F0913019F073
:1097D00081E0923019F480E0089581E008950E94BC
:1097E000D64B8823E1F30895CF93DF93C82F8830B9
:1097F00049F0863039F0893029F0863119F0893105
:1098000009F045C08091390181FD44C00E94EF4BB1
:109810000E94AA4BD82FC817B9F1C83019F40E947A
:10982000B14B2BC0C93141F48631A9F482E491E0F7
:109830006FE140E029E009C0C63169F4893159F48B
:1098400082E491E06FE140E026E00E947551E3E0A0
:10985000F0E03197F1F782E491E06FE140E02C2FE6
:109860000E947551D83029F489E691E00197F1F70B
:1098700004C0E3E0F0E03197F1F70E94AA4B8C17A7
:1098800019F083E490E008C080E490E005C082E431
:1098900090E002C084E490E0DF91CF910895809140
:1098A000940090919500909302278093012721E0E6
:1098B0002093EE268091390181FF15C02093682600
:1098C00080919400909195009093FE268093FD26C0
:1098D0002093EC26809139018D7F8093390180910E
:1098E00068268823E1F786E10E94F44B81E08093AB
:1098F0006926089580916926882351F48091FF0F8D
:10990000882321F081E08093811002C00E944F4C97
:1099100081E090E008950E94EF4B109269260E942A
:10992000B14B809139018260809339018091EC269E
:109930008823E9F180919400909195002091FD2673
:109940003091FE2682179307A0F48091C92690914A
:10995000CA26A091CB26B091CC268C57914EAF4F02
:10996000BF4F8093C9269093CA26A093CB26B0936D
:10997000CC268091940090919500821B930BA0E0DF
:10998000B0E04091C9265091CA266091CB267091D3
:10999000CC26840F951FA61FB71F8093C9269093CE
:1099A000CA26A093CB26B093CC261092EC268091A9
:1099B000EE268823E9F18091940090919500209102
:1099C00001273091022782179307A0F48091D126B6
:1099D0009091D226A091D326B091D4268C57914E47
:1099E000AF4FBF4F8093D1269093D226A093D3261A
:1099F000B093D4268091940090919500821B930B94
:109A0000A0E0B0E04091D1265091D2266091D326BB
:109A10007091D426840F951FA61FB71F8093D1265F
:109A20009093D226A093D326B093D4261092EE26FC
:109A3000089580918110882321F00E944F4C10924C
:109A4000811080918210882321F00E948B4C10920B
:109A500082101092FF0F08950F931F93CF93DF93FF
:109A6000F82FE92FAB0181E08093FF0F0091AD2625
:109A70001091AE262091AF263091B0260F5F1F4F78
:109A80002F4F3F4F0093AD261093AE262093AF2665
:109A90003093B026862F8E5F87FF0CC0809166269C
:109AA0009091672601969093672680936626CFEF64
:109AB000DFEF09C020E030E1C9016F2F7E2F0E9447
:109AC000A775C0E0D0E00E94194DCE01DF91CF9183
:109AD0001F910F91089580916926882399F08091B4
:109AE000FF0F882321F40E94D64B882331F481E0B4
:109AF0008093821081E090E008950E948B4C80E07A
:109B000090E0089580E090E008951F93CF93DF9355
:109B10000F92CDB7DEB78FB789838091FF0F88236F
:109B200031F5F89480916926882351F080913901AC
:109B300081FD1BC00E94D64B8823B9F080E003C092
:109B40000E947A4C81E0909147019E3010F010E025
:109B500001C01FEF882311F00E946B4D16FF05C056
:109B600089818FBF81E090E004C089818FBF80E050
:109B700090E00F90DF91CF911F9108958093FE0F99
:109B800008950E94AA4B8250813130F4E82FF0E012
:109B9000EF51FA4F8081089581E0089508958FEF85
:109BA00080934E018CE691E060EF44E022E00E9459
:109BB00075518CE290E06EE041E025E00E94755125
:109BC00080E880936F018091460180936D0184E469
:109BD00091E060E245E021E00E9475510895CF9345
:109BE000DF93CDEFD3E0CE010197F1F70E946151F1
:109BF0001092DD2410925F251092E1251092DC2452
:109C00001092DB24E9E3F1E080818E7F8083808104
:109C10008D7F80838DE090E00197F1F780818160F6
:109C2000808382E491E06FE140E023E00E9475517F
:109C30002197F1F780915D0180915E010E94CF4DE7
:109C400083EC95E060E070E00E94503A0E944F4C37
:109C500081E090E0DF91CF91089580918310089585
:109C6000CF93DF930F92CDB7DEB789830E94EF4B7E
:109C700029812093831088E491E06FE140E00E9405
:109C800075510F90DF91CF9108950E94304E86E07C
:109C90000E94F44B0895FA0180936201909363014E
:109CA00060936001709361013097C1F0808180936F
:109CB0006B01818180936A01828180936901838134
:109CC0008093680184818093670185818093660118
:109CD000868180936501878180936401089583EC78
:109CE00095E00E94723A81E08093D4248091D5243B
:109CF0009091D62401969093D6248093D52481E028
:109D000090E00895CF93DF935091DC24252F30E02D
:109D1000F901EE0FFF1F3695322F22273795279531
:109D2000E20FF31FE352FB4D4081442309F4F4C0DA
:109D30002091390121FDF0C020916926222309F4E8
:109D4000EBC047FF23C0852F90E0FC01EE0FFF1F03
:109D50009695982F882797958795E80FF91FE352D6
:109D6000FB4D108280919D2690919E26A0919F266A
:109D7000B091A0260196A11DB11D80939D269093C0
:109D80009E26A0939F26B093A026C6C0433018F508
:109D9000852F90E0FC01EE0FFF1F9695982F8827E6
:109DA00097958795E80FF91FE352FB4D108280913C
:109DB000992690919A26A0919B26B0919C26019677
:109DC000A11DB11D8093992690939A26A0939B265E
:109DD000B0939C26A1C0C42FD0E022976C177D07BA
:109DE00018F5852F90E0FC01EE0FFF1F9695982F38
:109DF000882797958795E80FF91FE352FB4D10824E
:109E00008091952690919626A0919726B0919826BC
:109E10000196A11DB11D8093952690939626A0933F
:109E20009726B093982678C0252F30E0B901660FA9
:109E3000771F3695322F222737952795620F731F8C
:109E400062527B4D50E00E94A7752091DC24822F46
:109E500090E0FC01EE0FFF1F9695982F88279795AD
:109E60008795E80FF91FE35AFA4D80818093CD243E
:109E7000822F90E0FC01EE0FFF1F9695982F882708
:109E800097958795E80FF91FE352FB4D10822F5FDE
:109E90002093DC24233010F01092DC248091DC2409
:109EA00090E0FC01EE0FFF1F9695982F882797955D
:109EB0008795E80FF91FE352FB4D8081882311F04D
:109EC0000E946F4E609147016093CE248091D3240D
:109ED000882311F0681710F46093D32484E070E0B5
:109EE0000E94C3416091CD2483E070E00E94C34191
:109EF0008091B1269091B226A091B326B091B4265C
:109F00000196A11DB11D8093B1269093B226A09316
:109F1000B326B093B42602C0C0E0D0E0CE01DF91FA
:109F2000CF910895CF93DF93EC01888199810097B9
:109F300029F024E08B3F920739F505C08BEF94E0C0
:109F40009983888325C0623819F51092D4240E9421
:109F500049410E94AA4060E870E00E94824E1816B3
:109F6000190644F40E94A540E0915406F09155066C
:109F70000995E4CF8091D1249091D22401969093B9
:109F8000D2248093D124DACF1982188283E001C0D1
:109F900081E0DF91CF91089591E09093FF0F0E94AF
:109FA000C74B0E94194D08958091390181FD07C06A
:109FB00085E491E06FE040E00E946B51089580E1FC
:109FC00008950F931F93CF93DF93C82F21E0209321
:109FD000FF0FD09169268091390181FF16C08091D1
:109FE0009400909195009093FE268093FD262093F7
:109FF000EC2620936826809139018D7F809339016A
:10A00000809168268823E1F7D0E00E94EF4B809191
:10A010006926882309F441C08091EE268823E9F15E
:10A020008091940090919500209101273091022712
:10A0300082179307A0F48091D1269091D226A09107
:10A04000D326B091D4268C57914EAF4FBF4F8093FB
:10A05000D1269093D226A093D326B093D426809174
:10A06000940090919500821B930BA0E0B0E040918A
:10A07000D1265091D2266091D3267091D426840F98
:10A08000951FA61FB71F8093D1269093D226A09329
:10A09000D326B093D4261092EE2689E10E94F44B89
:10A0A00086E00E94CE41009751F00E94D44F082FC5
:10A0B00086E00E94CE4181500E94C74B02C000E062
:10A0C00010E08091940090919500909300278093E8
:10A0D000FF2681E08093ED26F8948091390182601B
:10A0E00080933901809139018D7F809339016C2FE4
:10A0F0006E5F80E090E10E94A65178948091632683
:10A1000090916426019690936426809363260E9422
:10A11000EF4B82E491E060EE45E00E946B51C82F66
:10A1200086E00E94CE41009719F0802F0E94C74B15
:10A13000DD2319F00E944F4C02C00E948B4C80918D
:10A14000ED268823E9F1809194009091950020916B
:10A15000FF263091002782179307A0F48091CD2627
:10A160009091CE26A091CF26B091D0268C57914EBB
:10A17000AF4FBF4F8093CD269093CE26A093CF268E
:10A18000B093D0268091940090919500821B930B00
:10A19000A0E0B0E04091CD265091CE266091CF2630
:10A1A0007091D026840F951FA61FB71F8093CD26D0
:10A1B0009093CE26A093CF26B093D0261092ED2672
:10A1C00080916926882361F0809194009091950098
:10A1D000909302278093012781E08093EE2607C0A9
:10A1E00082E491E06FE140E023E00E9475510E941B
:10A1F000194DC130E1F0C330A9F48091A5269091AA
:10A20000A626A091A726B091A8260196A11DB11D52
:10A210008093A5269093A626A093A726B093A82660
:10A22000C2E00AC0C53029F0C73031F404C0C0E034
:10A2300003C0C3E001C0C1E08C2F90E0DF91CF915B
:10A240001F910F910895CF93DF93EB010E942C4D46
:10A25000009729F4CE010E94E14F009751F0209120
:10A260006626309167262F5F3F4F309367262093F5
:10A270006626DF91CF910895CF93DF938091692671
:10A28000882321F40E947A4CC1E001C0C0E00E9402
:10A29000AA4B863111F0813119F4D091470109C0E0
:10A2A00086E491E06FE140E00E946B51D82FDD0F12
:10A2B000D80FCC2311F00E946B4D8D2FDF91CF91E1
:10A2C00008951092851010928410EFE6F0E08081DE
:10A2D000806280830895FC018081862390E002C023
:10A2E000959587954A95E2F70895F894FC01908139
:10A2F000862F8095892330E002C0220F331F4A95B4
:10A30000E2F72623282B208378940895CF93DF93B8
:10A31000EC012196E0917B01DC01EC932E2FA0E86B
:10A32000B1E03D9139932150E1F7E150F0E0E05880
:10A33000FE4F2181FC01E058FF4F20838F579F4F34
:10A3400021E0FC012083DF91CF910895FC0160930F
:10A350008001A1E8B1E0615881918D936A17E1F71E
:10A3600008951F920F920FB60F920BB60F92112401
:10A370002F933F934F935F936F937F938F939F930D
:10A38000AF93BF93EF93FF93809147018093CE24C7
:10A390002091DB2430E0C901880F991F3695322FB8
:10A3A000222737952795820F931F83529B4D0E943A
:10A3B00086518091DB248F5F8093DB24833010F003
:10A3C0001092DB240E946F4EFF91EF91BF91AF91ED
:10A3D0009F918F917F916F915F914F913F912F91BD
:10A3E0000F900BBE0F900FBE0F901F9018951F92ED
:10A3F0000F920FB60F9211240F900FBE0F901F9067
:10A4000018951F920F920FB60F9211240F900FBE46
:10A410000F901F9018951F920F920FB60F92112454
:10A420000F900FBE0F901F9018951F920F920FB6AE
:10A430000F921124109268260F900FBE0F901F905C
:10A4400018951F920F920FB60F9211241092682642
:10A450000F900FBE0F901F9018951F920F920FB67E
:10A460000F9211248F9381E08093D4248F910F90C9
:10A470000FBE0F901F9018951F920F920FB60F925C
:10A480001124109268260F900FBE0F901F90189500
:10A490001F920F920FB60F9211248F939F9380916A
:10A4A000841090918510019690938510809384106C
:10A4B0009F918F910F900FBE0F901F9018950F9343
:10A4C0001F93CF93DF938091712690917226A09174
:10A4D0007326B09174260196A11DB11D809371263B
:10A4E00090937226A0937326B09374260E94F7541B
:10A4F0008C0186E890E10E941A3B08C0EA81FB814A
:10A50000309709F00995CE010E94C03BEC010097FD
:10A51000A9F70115110519F0C8010E948838DF91CB
:10A52000CF911F910F9108950E94195A0E9449419D
:10A530000E94105385E396E090936C2680936B26DF
:10A540000E94F45482E090E060E074E040E05EE15C
:10A550002FEF31E00E94B5540895CF92DF92EF9231
:10A56000FF920F931F93CF93DF936C018B017A01BE
:10A5700086E890E10E941A3B09C0EC81FD8130978A
:10A5800011F0C8010995CE010E94C03BEC01009773
:10A59000A1F7C601B801A7010E949238DF91CF91BF
:10A5A0001F910F91FF90EF90DF90CF900895BC0125
:10A5B00086E890E10E94893B0895BC0186E890E11D
:10A5C0000E94543B0895CF93DF93EC0180916D2658
:10A5D00090916E26A0916F26B09170260196A11DD4
:10A5E000B11D80936D2690936E26A0936F26B09335
:10A5F0007026CE010E940A55009769F00E94C4405F
:10A60000E0913906F0913A068DEA92E5BE0109958E
:10A6100081E090E002C080E090E0DF91CF9108956A
:10A6200088E890E10E94163B08950F93CF93DF9343
:10A63000EC017B836A8318865F834E8388E890E110
:10A64000BE010E94893BE0918A10F0918B103097F7
:10A6500049F04C815D818A819B81688520E030E0F2
:10A6600001E00995DF91CF910F910895BC0188E831
:10A6700090E10E94543B08950F93DC0118961C92C0
:10A680001897E0918A10F0918B10309759F012963C
:10A690008D919C91139760E040E050E020E030E025
:10A6A00000E009950F9108950F93DC01AB0114961A
:10A6B0002D913C91159781E018968C9318971596DB
:10A6C0007C936E931497E0918A10F0918B103097E1
:10A6D00039F012968D919C91139761E000E00995F5
:10A6E0000F9108950F93DC01E0918A10F0918B1087
:10A6F000309769F014962D913C91159712968D9193
:10A700009C91139718966C91A90101E009950F91FE
:10A710000895E0918C10F0918D10309709F0099513
:10A72000089590938D1080938C10089590938B10C2
:10A7300080938A10089588E890E10E941A3B08955A
:10A74000EF92FF920F931F93CF93DF938C01EB0156
:10A750007A0188E890E10E941A3B15C0DC0112964C
:10A760002D913C9113972C173D0759F41696ED91B6
:10A77000FC911797309749F0B801AE019701099500
:10A7800004C00E94C03B009749F7DF91CF911F9111
:10A790000F91FF90EF9008950895AF92BF92CF92DE
:10A7A000DF92EF92FF920F931F93CF93DF9300D02E
:10A7B000CDB7DEB75B010E94AA40FC01E080F180CA
:10A7C000FA82E982FCE0EF16F10418F400E010E0F0
:10A7D0002DC000D000D08DEF95E0EDB7FEB792838D
:10A7E0008183F482E3820E9426760F900F900F906F
:10A7F0000F901FC00E94AA40F801EE0FFF1FEE0F3E
:10A80000FF1FE80FF91FC280D3800E94AA400F5F8C
:10A810001F4FF801EE0FFF1FEE0FFF1FE80FF91F8C
:10A8200040815181C501B6010E94A0530E151F053C
:10A8300009F70F900F90DF91CF911F910F91FF902B
:10A84000EF90DF90CF90BF90AF900895CF93DF93BC
:10A85000C9EAD0E16091BF107091C010CE0149E407
:10A8600054E520E030E00E94AB3D0E94165A609112
:10A87000BF107091C0100E945472BC01CE0140976D
:10A880004DE654E520E030E00E94AB3DDF91CF91F2
:10A8900008958091BF109091C0102091BD1030910B
:10A8A000BE10880F991F2817390708F4C901909323
:10A8B000C0108093BF100E94265408950F9301305A
:10A8C00051F48091B9109091BA109093C010809378
:10A8D000BF100E9426540F910895CF93DF930E94DA
:10A8E00049410E94AA40EC01198218820E949B53A0
:10A8F00020C012962D913C911397FC01EE0FFF1F83
:10A90000EE0FFF1FEC0FFD1F3383228314962D9152
:10A910003C9115970196FC01EE0FFF1FEE0FFF1FF4
:10A92000EC0FFD1F3183208399838883CD010E9422
:10A93000C03BDC0188819981109729F018962C91F1
:10A9400018972223B1F6880F991F880F991F029636
:10A950000E94A54088819981009721F08EE890E1BE
:10A960000E945B38DF91CF910895EF92FF920F9391
:10A970001F93CF93DF93FC018B017A01E9018EE8ED
:10A9800090E1BF014AE156E00E943D381093BA10B1
:10A990000093B910F092BC10E092BB10D093BE109F
:10A9A000C093BD108EE594E50E949653DF91CF9140
:10A9B0001F910F91FF90EF900895CF93DF93C9EA15
:10A9C000D0E1CE010E94323ECE0140970E94323E3D
:10A9D000CE014B970E945838DF91CF910895809116
:10A9E000BF109091C01008950E949E380895CF9393
:10A9F000DF93E0911E06F0911F060995EC01009788
:10AA000029F06A817B8181E00E94C341CE01DF9100
:10AA1000CF9108950F931F93CF93DF93EC01E091B3
:10AA20002006F091210609958C016A817B8181E0E5
:10AA30000E94C34181E090E00115110511F480E00E
:10AA400090E0DF91CF911F910F910895E091220640
:10AA5000F0912306099508959C0180E090E005C0DF
:10AA6000F90131974081840F911D2E5F3F4FF9010D
:10AA7000329740814423A1F70895FC01308120E002
:10AA8000818190E0822B932B02C0880F991F6A95D9
:10AA9000E2F7892F9927FA01EC5DF94F208130E028
:10AAA0008223932328E030E0241B350B02C09695C7
:10AAB00087952A95E2F708956F927F928F929F92E1
:10AAC000AF92BF92CF92DF92EF92FF920F931F93BC
:10AAD000CF93DF935C013B018A0169012830310586
:10AAE00044F4CB01BA01A9010E943D55F5018083D0
:10AAF0004EC0790173E0F594E7947A95E1F741153A
:10AB0000510521F04501C0E0D0E005C0F301D501B9
:10AB100080E090E021C0C3018C0F9D1FB80148E088
:10AB200050E00E943D55F40181934F012196CE15CE
:10AB3000DF058CF3C701F7FE02C080E090E0A601BC
:10AB4000477050704115510511F1E501C80FD91F2B
:10AB5000860D971DB80118C021912D9301968E1571
:10AB60009F05D4F3C701F7FE02C080E090E0A60184
:10AB7000477050704115510551F0E501C80FD91FBC
:10AB8000860D971D60E070E00E943D558883DF913F
:10AB9000CF911F910F91FF90EF90DF90CF90BF90DA
:10ABA000AF909F908F907F906F9008958F929F921B
:10ABB000AF92BF92CF92DF92EF92FF920F931F93CB
:10ABC000CF93DF9300D000D0CDB7DEB70E94AA406C
:10ABD0008C0182E090E00E948740009709F45FC0FA
:10ABE000F801918180E02081820F911D0E94B2388E
:10ABF0007C01009709F455C00E94AA404C01F7015E
:10AC00008681482F46954695469550E090E087709E
:10AC1000907021E030E0009711F420E030E0CA01AC
:10AC2000820F931F0E9487400097C9F1F7010481AA
:10AC30001581CC24DD242EC0F801A180BB24B601EF
:10AC4000A3E075956795AA95E1F7680D791DA601B2
:10AC500047705070883168F0CE01039695010E94CC
:10AC60005C55F8018081BE016D5F7F4F0E94D74126
:10AC70000DC01A821982CE01019695010E945C5581
:10AC800069817A81F80180810E94C341CA0CDB1C72
:10AC90000E5F1F4FF8018081882371F602C0EE24F9
:10ACA000FF24C7010F900F900F900F90DF91CF916D
:10ACB0001F910F91FF90EF90DF90CF90BF90AF90DA
:10ACC0009F908F900895FC0150E080E190E0861BFA
:10ACD000970B821B930B02C0440F551F8A95E2F716
:10ACE0008081852B80838181842B818308956F925D
:10ACF0007F928F929F92AF92BF92CF92DF92EF920C
:10AD0000FF920F931F93CF93DF933C016B015A0186
:10AD100079012830310524F4C301FA01408159C07A
:10AD20008901B3E015950795BA95E1F761157105AD
:10AD300021F04A01C0E0D0E005C0FA01D30180E073
:10AD400090E023C0F40141914F01C3018C0F9D1F7E
:10AD5000B60128E030E00E9463562196C017D10763
:10AD60008CF3980117FF02C020E030E0D701A770F4
:10AD7000B070109781F1F501E20FF31F408150E0B0
:10AD8000C6018A1B9B0B089619C021912D93019631
:10AD900080179107D4F3980117FF02C020E030E03C
:10ADA000D701A770B0701097B1F0F501E20FF31F53
:10ADB000408150E088E090E08A1B9B0B02C05595D3
:10ADC00047958A95E2F7C301820F931F60E070E018
:10ADD0009D010E946356DF91CF911F910F91FF90CB
:10ADE000EF90DF90CF90BF90AF909F908F907F902B
:10ADF0006F9008956F927F928F929F92AF92BF92C1
:10AE0000CF92DF92EF92FF920F931F93CF93DF9336
:10AE100000D0CDB7DEB77C01DC0116968C91169779
:10AE2000282F26952695269530E090E08770907023
:10AE300001E010E0009711F400E010E0020F131F92
:10AE4000C80102960E940F41009709F451C00E9468
:10AE5000B140FC01D70112968C9112978083139612
:10AE60008C9181830E94B14032E0632E712C680E78
:10AE7000791EC30160E070E0A8010E94B075F7017F
:10AE8000E480F580CC24DD242CC0D7011196AC9051
:10AE90001197BB24860193E0159507959A95E1F7E4
:10AEA000060D171D27E0822E912C8C209D208831C5
:10AEB00030F00E94E141AC01C801B40109C00E9418
:10AEC000CE419A838983C801B401AE014F5F5F4FC1
:10AED00095010E947756CA0CDB1CE2E0F0E0EE0E12
:10AEE000FF1ED7018C91882381F681E090E002C09B
:10AEF00080E090E00F900F90DF91CF911F910F9124
:10AF0000FF90EF90DF90CF90BF90AF909F908F9089
:10AF10007F906F900895E0915206F0915306099545
:10AF20000895E091FB05F091FC0509950895E091E5
:10AF30005606F091570609950895E0915806F0914C
:10AF400059060995089580E090E008950895E091EC
:10AF5000DD05F091DE050995089580E090E0089503
:10AF60000F931F93CF93DF93CDB7DEB7E0970FB664
:10AF7000F894DEBF0FBECDBF0E94FA408C010E9444
:10AF8000AA40602FAE014F5F5F4F0E94A65F8823EB
:10AF900009F446C088A99801281B3109C9010E94FB
:10AFA00087400097E9F12E81222379F18A859B85DC
:10AFB0003BEA8D3C930721F03FEF8F3F930781F5EC
:10AFC000223069F088E090E00197E1E0F0E0EC0FDA
:10AFD000FD1FE80FF91F23852F3F21F007C082E0F6
:10AFE00090E0F2CF181619067CF30FC089E1BE017C
:10AFF000645F7F4F0E94D74189E10E94E1416AE787
:10B0000074E20E94F537009759F088E1BE016A5E4C
:10B010007F4F0E94D741E0913B06F0913C06099595
:10B02000E0960FB6F894DEBF0FBECDBFDF91CF9193
:10B030001F910F910895AF92BF92CF92DF92EF923E
:10B04000FF920F931F93CF93DF93CDB7DEB7E097B7
:10B050000FB6F894DEBF0FBECDBF5C016B01FE01E1
:10B06000319680E3DF011D928A95E9F781E08983BB
:10B070008CE00E94CE418C831D821F828091C31080
:10B0800089878F5F8093C31003E008878DEC9BEA6C
:10B090009B878A8789E10E94E1416DE175E00E940A
:10B0A000F537009731F082E08E838FEF8C878D87A4
:10B0B00009C089E10E94E141BC01CE010C960E94C9
:10B0C000EC370E838DEC9BEA9D8B8C8BCE014696E4
:10B0D0006AE774E20E94EC370E94AA409FA78EA7FD
:10B0E0000E94FA4088ABCE0101960E94B75E082FFD
:10B0F00090E00E940F41009749F10E94B140BC01CD
:10B10000CE010196402F0E94D55E0091D30510918B
:10B11000D4050E94B1407C010E940441BC01C701DA
:10B12000F8010995A114B10489F0009721F081304C
:10B13000910561F404C0C60160E070E003C0C6017F
:10B1400064E070E041E050E0F5010995E0960FB64B
:10B15000F894DEBF0FBECDBFDF91CF911F910F914D
:10B16000FF90EF90DF90CF90BF90AF9008950E9436
:10B17000165A8093C310E091DD05F091DE05099524
:10B180000895009731F0E091DD05F091DE05099515
:10B190000895E091DF05F091E00509950895CF93BA
:10B1A000DF93EC0104C060E070E00E94503A8991A6
:10B1B00099910097C1F7DF91CF910895CF93DF93D5
:10B1C000EC0102C00E949739899199910097D1F7BB
:10B1D000DF91CF910895CF93DF93EC017B836A8356
:10B1E0000E94EB4999838883DF91CF910895FC01F8
:10B1F0008081918122813381820F931F918380838B
:10B200000895CF93DF93EC010E94EB4999838883E3
:10B21000DF91CF910895CF93DF93EC010E94EB492A
:10B2200028813981AC01421B530B9A012F5F3F4F9C
:10B2300081E090E04A815B814217530710F080E083
:10B2400090E0DF91CF910895CF93DF93FC01C2810D
:10B25000D38180819181C80FD91F0E94EB499E0143
:10B26000281B390BC901DF91CF910895CF93DF934C
:10B27000E3EFF6E2C5EBD6E2A7EEB6E21192119249
:10B2800019921992199219921D9287E2EB30F807E0
:10B29000A9F7DF91CF9108950F931F93CF93DF9379
:10B2A000FC01E951F94D20818C01000F111F000FA5
:10B2B000111F222311F12091940030919500E80193
:10B2C000CB54D94DFC01EE0FFF1FED50F94D80819D
:10B2D0009181A901481B590BCA01A0E0B0E0488147
:10B2E00059816A817B81840F951FA61FB71F8883B0
:10B2F0009983AA83BB8331832083F801EB54F94DF2
:10B300006081718182819381DF91CF911F910F9133
:10B31000089560E070E080E090E00895FC01EE0F99
:10B32000FF1FEE0FFF1FEB54F94D408351836283E3
:10B3300073830895EF92FF920F931F93CF93DF9340
:10B34000B7EEEB2EB6E2FB2EE5EBF6E2C3EFD6E26C
:10B3500020E030E0D7018D917D018823C9F0009174
:10B3600094001091950088819981A801481B590B80
:10B3700060E070E080819181A281B381840F951F8C
:10B38000A61FB71F80839183A283B3831983088389
:10B390002F5F3F4F349622962C303105D9F6DF913E
:10B3A000CF911F910F91FF90EF9008950E94395E09
:10B3B00008950F931F93FC018091C4109091C510C4
:10B3C000338322831583048371836083F093C510D4
:10B3D000E093C410009719F4CB010E94535E80E003
:10B3E00090E01F910F9108958091C4109091C51025
:10B3F0000097C1F01092C5101092C410DC01149691
:10B400006D917C9115971296ED91FC91139709958A
:10B41000E091C410F091C510309721F080819181A6
:10B420000E94535E08950E94497308950E944473D8
:10B4300008958CE596E00E94883A84E696E00E94A2
:10B44000883A0895CF93DF930E94B7400097A9F000
:10B4500084E696E00E94A73AEC01009729F10E9449
:10B46000FA40998388830E94F5409B838A83CE01AA
:10B4700004960E9431408CAB17C08CE596E00E9488
:10B48000A73AEC01009771F002960E94434099831D
:10B490008883BE016E547F4FCE018E579F4F0E940E
:10B4A000A14102C0C0E0D0E0CE01DF91CF9108956C
:10B4B000BC016E547F4F8E579F4F0E94A14108954B
:10B4C000CF93DF93EC018CE596E0BE010E94F83A41
:10B4D000009719F08CE596E009C084E696E0BE017D
:10B4E0000E94F83A009729F084E696E0BE010E9497
:10B4F000D23ADF91CF910895CF93DF93EC018CE5A1
:10B5000096E0BE010E94F83A009779F0688179814F
:10B51000CE0102960E947241BE016E547F4FCE0151
:10B520008E579F4F0E94B2411CC084E696E0BE0138
:10B530000E94F83A0097A9F00E94494168817981F8
:10B540008A819B810E9472418CA990E00E940F41E8
:10B550000E94B1404CA9BE016C5F7F4F50E00E9439
:10B56000A775DF91CF910895CF93DF93EC018CE520
:10B5700096E0BE010E94F83A009719F0CE010296BB
:10B580000CC084E696E0BE010E94F83A009719F0DC
:10B590008A819B8102C080E090E0DF91CF91089585
:10B5A000FC0180819181089570E06F5B7F4F660F91
:10B5B000771F680F791FCB010895E62FF0E0EF5B4E
:10B5C000FF4FEE0FFF1FE80FF91F80819181089553
:10B5D00008958FE197E10E94DD3C009721F08FE113
:10B5E00097E10E94C83C0895E0910A17F0910B176B
:10B5F000309711F00995089580E00895EF92FF9239
:10B600000F931F93CF93DF937C018A01FC0180810C
:10B610009181009731F0F3E08C309F0709F0FFC073
:10B620002BC080E0E82FF0E0EE0FFF1FEE0FFF1FB2
:10B63000E35FF84E118210828F5F843098F380931D
:10B640000C178091490E90914A0EEDE0F7E1918B35
:10B65000808B0E94903980930B278FE197E160E403
:10B6600070E00E94B23C0E941B618CE093E0F70105
:10B670009183808381E0D7C0623009F4B2C0633027
:10B6800030F4662309F482C0613079F795C06738D9
:10B6900019F0683851F73AC010922717CDE0D7E17A
:10B6A00013C08A819B818017910741F48881998119
:10B6B0000E945162198218821B821A8224968091FC
:10B6C00027178F5F8093271780912717843048F3BF
:10B6D000EBE1FCE2848D958D8017910719F4158EAE
:10B6E000148E118EB0962CE2EB39F20798F3E1EB51
:10B6F000FCE2818592858017910711F415821482EE
:10B700003D968DE2E333F807A0F3AFCFE7E14F3189
:10B710005E0709F0AACFCA010E94DD3C009709F438
:10B72000A4CF109227172DC0F0E035E0EE0FFF1FD9
:10B730003A95E1F7E55EF34D818D8823E9F08FE1DD
:10B7400097E10E94C83C8091271790E025E0880F80
:10B75000991F2A95E1F7855E934D90931A2C80935B
:10B76000192C82E00E94856280910C2790910D2710
:10B77000009711F00E94F45A809127178F5F8093F1
:10B780002717E0912717E43078F26FCF4115510564
:10B7900009F46BCF50931A2C4093192C83E00E942C
:10B7A000856280910C2790910D27009711F00E94DF
:10B7B000F45A0E94E95A59CF4115510509F455CF61
:10B7C0005093162C4093152C85E00E948562809141
:10B7D0000C2790910D27009709F447CF0E94F45A47
:10B7E00044CF80910C2790910D27009709F43DCF0D
:10B7F00080911D27863031F48091352781FF02C06A
:10B800000E94E95A81E00E94856280910C27909104
:10B810000D27009709F429CF0E94215D26CFF7015B
:10B820001182108283E0DF91CF911F910F91FF90E1
:10B83000EF90089590930B1780930A1708959C0139
:10B840004091490E50914A0E60E0EDE0F7E114C0DE
:10B85000808191818217930769F482819381841793
:10B86000950741F46093281711821082C9010E9444
:10B870005162089534966F5F643050F360932817D7
:10B88000089540E0EDE0F7E116C0542F5F5F20819E
:10B8900031812115310569F4409329179183808303
:10B8A0002091490E30914A0E338322830E946B62AD
:10B8B00008953496452F443040F340932917089556
:10B8C000FC018091490E90914A0E958F848F778F5D
:10B8D000668F0895FC018091490E90914A0E9287DF
:10B8E0008187748763870895CF93DF93EA010E946D
:10B8F000DD61009749F02091490E30914A0EFC011C
:10B9000032872187D487C387DF91CF9108950F9322
:10B910001F93CF93DF9300D000D0CDB7DEB78C015B
:10B92000AB018FEF89838A838B838C83CE01019651
:10B93000B8010E94745C009719F0FC011583048320
:10B940000F900F900F900F90DF91CF911F910F915B
:10B95000089589E796E062E040E050E00E94413AB5
:10B9600010920D2710920C270895AC0189E796E0FC
:10B9700061E00E941E3A0895AC0189E796E060E01C
:10B980000E941E3A08950F931F93CF93DF938A016D
:10B990000E945161EC01009759F08091490E9091FD
:10B9A0004A0E9D8F8C8F1F8F0E8FCE010E94BC5C24
:10B9B000CE01DF91CF911F910F910895CF93DF9327
:10B9C000A091192CB0911A2C109719F0ED016C96DA
:10B9D00005C0C091152CD091162C29968091142C5D
:10B9E00086FF22C010922A1740E0EDE0F7E116C072
:10B9F0008081918114962D913C9115978217930720
:10BA000059F482819381009739F040932A179983E2
:10BA100088831B821A8206C034964F5F443040F3FD
:10BA200040932A170E94E95A88819981009731F042
:10BA30004A815B8160910B270E94413ADF91CF914F
:10BA400008950F931F93CF93DF9380911D27863026
:10BA500009F074C080910C2790910D2725E080306B
:10BA6000920709F06BC0C4E9D2E0D0930D27C093D0
:10BA70000C2702E00093162714E910931727109261
:10BA80003927109238270E941361809590959093E2
:10BA900039278093382710921F2710921E270E9463
:10BAA00002618095909590931F2780931E270E9496
:10BAB000F45AD0930D27C0930C27009316271093A8
:10BAC00017279091172C8091182CE92FF82FDF0160
:10BAD000A459BD4F8CE692E00D9001920197E1F7D9
:10BAE0008CE297E26CE672E00E94BF6080911027C2
:10BAF00080932C278091112780932D2780911227E6
:10BB000080932E278091132780932F271092392717
:10BB1000109238270E941361809590959093392751
:10BB20008093382710921F2710921E270E940261CF
:10BB30008095909590931F2780931E270E94F45A1A
:10BB4000DF91CF911F910F910895FC0120E030E02B
:10BB500080E0A8E111C0419198E0542F5827B52FFB
:10BB6000B17050FD8A278695B13009F480684695FA
:10BB7000915099F72F5F3F4F2617370761F70895C8
:10BB80001F920F920FB60F920BB60F9211242F93A4
:10BB90003F934F935F936F937F938F939F93AF9355
:10BBA000BF93EF93FF9380919400909195009093B1
:10BBB000F8268093F72681E08093E9268091710032
:10BBC000807D809371000E94F4598091E92688233A
:10BBD000E9F180919400909195002091F7263091A1
:10BBE000F82682179307A0F48091BD269091BE2677
:10BBF000A091BF26B091C0268C57914EAF4FBF4F3A
:10BC00008093BD269093BE26A093BF26B093C026F6
:10BC10008091940090919500821B930BA0E0B0E07E
:10BC20004091BD265091BE266091BF267091C026DE
:10BC3000840F951FA61FB71F8093BD269093BE2625
:10BC4000A093BF26B093C0261092E926FF91EF91F2
:10BC5000BF91AF919F918F917F916F915F914F9124
:10BC60003F912F910F900BBE0F900FBE0F901F9022
:10BC700018959FB7F894E1E7F0E08081807D80839C
:10BC800088B38F6288BB10929000E1E9F0E01082E7
:10BC9000109292001092950010929400808185601D
:10BCA00080839FBF08952FB7F89490939900809355
:10BCB000980088B38F6288BBE1E7F0E08081826002
:10BCC00080832FBF0895CF93DF93FC01DB0185E0D4
:10BCD000EB0119928A95E9F7858190E08370907065
:10BCE000009711F082E08C93878190E083709070D0
:10BCF000009721F082E012968C931297858190E054
:10BD000083709070009799F0878190E083709070B5
:10BD1000009769F02389348981859285281739072E
:10BD200031F481E0848312961C92129701C0148230
:10BD3000C581C370C250C23028F4D0E0CD57D94F6E
:10BD4000888101C080E011968C931197E781E370A0
:10BD5000E250E23028F4F0E0ED57F94F808101C065
:10BD600080E013968C931397DF91CF910895CF9332
:10BD7000DF9300D000D00F92CDB7DEB7BE016F5F6A
:10BD80007F4F0E94635E89819A81890F8D5F9B81BD
:10BD9000890F9C81890F9D81890F0F900F900F90C3
:10BDA0000F900F90DF91CF910895DF92EF92FF9265
:10BDB0000F931F93CF93DF9300D000D000D0CDB767
:10BDC000DEB78C017B01BE016F5F7F4F4E830E9407
:10BDD000635E79816A81AB81BC81872F90E0039695
:10BDE000860F911D8A0F911D8B0F911D2D81820F42
:10BDF000911D4E8150E0481759070CF498C0F80186
:10BE0000218130E02170307083E0220F331F8A954A
:10BE1000E1F7828190E08170907034E0880F991F83
:10BE20003A95E1F7822B90819770892B438150E0FE
:10BE30004170507095E0440F551F9A95E1F7842B9F
:10BE4000448150E04170507026E0440F551F2A9500
:10BE5000E1F7842BF7018083F801258130E023701E
:10BE60003070220F331F220F331F868190E08370C2
:10BE7000907054E0880F991F5A95E1F7822B9781B3
:10BE80009295990F990F907C982BF7019183F80167
:10BE90008085F7018283723051F4F8018185F701C2
:10BEA0008383F8018285F701848355E001C053E064
:10BEB00040E080E090E09801260F311D09C0F901B3
:10BEC000E80FF91FD384F701E70FF11DD0824F5F10
:10BED000742F750F0197461791F7972FA23089F4A9
:10BEE0009701270F311DF8018389F9018083872F7E
:10BEF0008F5F9701280F311DF8018489F901808334
:10BF00009E5F40E020E030E00B0F111D09C0F801FA
:10BF1000E20FF31F5589F701E80FF11D50834F5FC2
:10BF2000842F890F215030404B1789F701C080E0E2
:10BF300026960FB6F894DEBF0FBECDBFDF91CF912E
:10BF40001F910F91FF90EF90DF900895BF92CF92D5
:10BF5000DF92EF92FF920F931F93CF93DF937C01B9
:10BF6000B62EEA0182E0861708F0AEC0F7018081A4
:10BF7000D82ED294D694D69463E0D622F1E0DF2274
:10BF8000F7019181292F269526952370C92EC294F9
:10BF9000C694C69473E0C722382F37703883382F81
:10BFA00036953695369531703983382F3295317004
:10BFB0003A838295869581708B83DC822D83892FCD
:10BFC000829583708E83CF8282818887222369F154
:10BFD0003381948180E0830F911D9A878987223075
:10BFE00079F4CA010B966DE175E00E94EC37F70118
:10BFF00086818B8785818C878701095F1F4F20C0D1
:10C0000087010B5F1F4F2330D9F4F7013D96DA010A
:10C0100080E092911B969C931B978F5F11968830BE
:10C02000C1F78701035F1F4F0BC087010D5F1F4FD3
:10C03000CA010B966DE175E00E94EC371A861986ED
:10C04000CC2089F1DD2059F4F8012081918180E034
:10C05000820F911D9C8B8B8B0E5F1F4F04C08985B7
:10C060009A859C8B8B8BF2E0CF1671F4CE014596AE
:10C070006DE175E00E94EC37F80181818D8B808144
:10C080008E8B0E5F1F4F17C0F3E0CF16A1F4085F31
:10C090001F4FD801FE0180E09E91958B8F5F3196F6
:10C0A0008830D1F708C0CE0145966DE175E00E9459
:10C0B000EC371C8A1B8A802F8E199B2D981B9FA7FB
:10C0C0001EA70DA7B81608F480E0DF91CF911F914D
:10C0D0000F91FF90EF90DF90CF90BF9008959C015B
:10C0E00041505040460F571FFB010EC0B081A0E0E9
:10C0F0008181BD01680F711D260F371F2617370775
:10C1000010F42F5F3F4F3296E417F50778F3E417EA
:10C11000F50749F4908180E0280F391F2817390767
:10C1200010F42F5F3F4FC9010895CF93DF93C09163
:10C130001727D0E064973091162720E0C20FD31F55
:10C140009E01280F311DC90160E277E248E050E00E
:10C150000E946F6068E277E2AE010E946F60009714
:10C1600021F098278927982702C08FEF9FEFDF9152
:10C17000CF91089590933217809331170895FC0161
:10C180004381460F40931327872F99272281280F39
:10C1900020931227A181A09311275081509310273B
:10C1A00030E02817390748F48A2F8F5F80931127D2
:10C1B000882319F45F5F50931027842F90E07070EC
:10C1C0008617970798F4809112278F5F8093122724
:10C1D000882361F4809111278F5F80931127882332
:10C1E00029F4809110278F5F8093102708959C0178
:10C1F000AB0180E090E0B9010E946F609827892729
:10C200009827089580E090E064E177E244E150E00F
:10C210000E946F60009721F098278927982708953A
:10C220008FEF9FEF089586E00E949560089581E169
:10C230000E949560089580E0E82FF0E0EE0FFF1F68
:10C24000E556F34D118210828F5F8430A8F380E0B1
:10C25000E82FF0E035E0EE0FFF1F3A95E1F7E55EDD
:10C26000F34D118E8F5F843098F380E094E09093CB
:10C2700035178093341740E08DE090E0242F30E0B4
:10C28000289FF001299FF00D389FF00D1124EF54E5
:10C29000F34D158214824F5F4A3080F34093331779
:10C2A0000895CF93DF93EC01209134173091351727
:10C2B0002F5F3F4F8DE72030380710F020E030E14E
:10C2C000522F432FA0E012C0EA2FF0E0B5E0EE0FAE
:10C2D000FF1FBA95E1F7E55EF34D818D882329F0C4
:10C2E000848195818417950719F3AF5FA43061F7B6
:10C2F00030933517209334171092331780E0E0E025
:10C30000F0E01EC0A82FB0E055E0AA0FBB1F5A9561
:10C31000E1F7A55EB34D59969C915997992321F465
:10C3200080933317FD0110C0973049F4309731F0F6
:10C330005A962C915A97928D921708F4FD018F5FAF
:10C34000843000F380933317309799F182E0818F26
:10C3500080913617848780913717858780913817A9
:10C36000868780913917878788ED94E0938B828B3D
:10C37000958B848B81E090E0918B808B138E81E094
:10C38000828F83E0808F168A80E1878B80913417BB
:10C3900090913517982789279827958384837783E9
:10C3A000668388819981AA81BB8180839183A283DE
:10C3B000B383CF01DF91CF9108950F931F93CF9354
:10C3C000DF93EC018B0120913417309135176DE02C
:10C3D00070E02F5F3F4F8DE72030380710F020E0EE
:10C3E00030E1522F432FA0E011C08A2F90E0869FAA
:10C3F000F001879FF00D969FF00D1124EF54F34D3F
:10C4000084819581AF5F8417950719F3AA3069F786
:10C41000309335172093341740E02DE030E018C0FA
:10C42000542F5F5F842F90E0829FF001839FF00D77
:10C43000929FF00D1124EF54F34D84819581009764
:10C4400031F4409333179F01309749F424C0452FAE
:10C450004A3030F34093331720E030E01CC0809125
:10C4600034179091351798278927982795838483C7
:10C4700017830683209729F4108211821282138277
:10C4800008C088819981AA81BB8180839183A2831E
:10C49000B38380E48087C901DF91CF911F910F9111
:10C4A000089540E013C0E42FF0E0542F5F5FEE0FDB
:10C4B000FF1FE556F34D208131812817390729F4F4
:10C4C00040933317118210820895452F443058F35A
:10C4D00040933317089540E013C0E42FF0E0542F49
:10C4E0005F5FEE0FFF1FE556F34D2081318121156F
:10C4F000310529F440933317918380830895452FA4
:10C50000443058F3409333170895AF92BF92CF92BF
:10C51000DF92EF92FF920F931F93CF93DF93C0911F
:10C52000192CD0911A2C843009F4F1C12CE337E294
:10C530003093182C2093172C30930F2720930E271D
:10C54000833071F4898D90E08F7090708330910505
:10C5500009F074C088899989009709F031C78DC0A6
:10C56000823009F08EC0809139178F5F8093391720
:10C57000882399F4809138178F5F80933817882328
:10C5800061F4809137178F5F80933717882329F4E0
:10C59000809136178F5F8093361710920D27109277
:10C5A0000C271092B02C1092AF2C898D873011F08F
:10C5B000853041F48A8D8F5F8A8F843109F000C7FE
:10C5C000198EFEC6882309F4FBC6288939892115EE
:10C5D000310509F44EC09A8D292F21502A8F9923B5
:10C5E00009F0EEC69B8D983031F0282F2150223073
:10C5F00048F4953039F4198E80E88093142C0E9409
:10C60000DE5C94C5953048F423E030E0092E02C08A
:10C61000220F331F0A94E2F701C020E32A8F9F5FA5
:10C620009B8F90E08F70907083309105E1F08430A3
:10C6300091054CF48130910509F469C3823091056C
:10C6400009F0BEC60DC08630910509F47EC588305C
:10C65000910509F47AC58430910509F0B1C675C514
:10C660001092352757C384E08093142C0E94DE5C1F
:10C6700092C58F70833009F0A3C688E08093142C94
:10C680004AC5853019F5E091152CF091162C84815E
:10C690009581009709F494C610921A2C1092192CC7
:10C6A0002C5030403093182C2093172C30930F27A8
:10C6B00020930E271092B02C1092AF2C10920D27C1
:10C6C00010920C2788E08093142C1FC180911427AE
:10C6D000853409F075C61091162700E08091172760
:10C6E000080F111D80910C2790910D27801791073D
:10C6F00008F466C610930D2700930C2780911A2723
:10C7000090E08F739070009709F05AC680911B27B4
:10C71000882309F055C64091AB2C5091AC2CA090C9
:10C720008506B09086064A155B0559F48091AD2CBC
:10C730009091AE2C2091870630918806821793073E
:10C74000A1F080912427909125278417950709F05F
:10C7500037C620912627309127278091AD2C9091C4
:10C76000AE2C2817390709F02BC60E9402612FEF63
:10C770008F3F920709F024C680911D27863009F467
:10C780002EC18131D1F1813009F01AC6809128275C
:10C79000883009F015C61092282780912A27909199
:10C7A0002B272FEF873F920710F0099601C00896BC
:10C7B00090932B2780932A27E4E1F7E280912027AA
:10C7C00090912127A0912227B0912327809324279D
:10C7D00090932527A0932627B09327278091AB2CF1
:10C7E0009091AC2CA091AD2CB091AE2C8487958704
:10C7F000A687B78780E48087C0C50C51104010938E
:10C800000D2700930C2780E397E29093182C8093D8
:10C81000172C80912E2790912F27009739F00E9496
:10C8200017612FEF8F3F920709F0CAC540912A2761
:10C8300050912B274115510509F4C2C581EB9CE2AB
:10C840009093162C8093152C60912827709129279E
:10C85000A0918706B0918806C0918906D0918A067A
:10C8600000918B0610918C06E0902027F0902127F4
:10C87000C0902227D09023272EC0848195810097D5
:10C8800021F14817590709F586819781009719F01A
:10C8900068177907D1F4208131812A153B0529F4E5
:10C8A000828193818A179B07F9F02C173D0729F4A1
:10C8B0008281938180179107B9F0E216F30629F47B
:10C8C00082819381C816D90679F0CF010D96909395
:10C8D000162C8093152CE091152CF091162C8DE2DE
:10C8E000E333F80750F26CC510921A2C1092192CF1
:10C8F00082E08093142C80E397E290930F2780933B
:10C900000E271092B02C1092AF2C0E94DE5C80910A
:10C91000AF2C9091B02C009709F452C59C01245E75
:10C920003F4F30930D2720930C27309316272093E9
:10C930001727E091152CF091162C208520931C27A9
:10C9400021E120931D2708969827892798279093FF
:10C950002D2780932C2710922F2710922E27848129
:10C96000958190932927809328278681978190939A
:10C970002B2780932A278091AB2C9091AC2CA091EF
:10C98000AD2CB091AE2C8093202790932127A093BB
:10C990002227B093232780819181A281B381809344
:10C9A000242790932527A0932627B09327278CE34D
:10C9B00097E29093182C8093172C0E941761809512
:10C9C000909590932F2780932E27009709F0D5C438
:10C9D0008FEF9FEF90932F2780932E27CEC40E9436
:10C9E00013612FEF8F3F920709F0EAC420912A27A5
:10C9F00030912B272115310509F4E2C440912827F5
:10CA0000509129274115510509F4DAC4E0912027F6
:10CA1000F0912127A0912227B0912327CBE1DCE2DE
:10CA2000698D6623A9F08C819D812817390781F4CF
:10CA30008E819F814817590759F488819981E81799
:10CA4000F90731F48A819B81A817B90709F47AC1E3
:10CA5000A0968CE2CB37D80719F310F380913527D5
:10CA60008F738230B9F430933B1720933A1740E02C
:10CA70000DC0E42FF0E0EE0FFF1FE556F34D80816F
:10CA800091814F5F2817390709F47DC0443088F33E
:10CA9000409333178091352782FD92C484E18093BF
:10CAA000352788E290E090930D2780930C2780E54E
:10CAB0008093342780912F279091332790932F27AD
:10CAC00030912E279091322790932E273093322742
:10CAD00020912D279091312790932D272093312756
:10CAE00090912C27909333174091302740932C2717
:10CAF000909330278F5F80933327882379F4832F97
:10CB00008F5F80933227882349F4822F8F5F809331
:10CB10003127882319F49F5F90933027809128272D
:10CB20009091292790933B1780933A1720912A27B9
:10CB300030912B27309329272093282790932B2758
:10CB400080932A278091202790912127A091222746
:10CB5000B09123278093242790932527A0932627FD
:10CB6000B09327278091AB2C9091AC2CA091AD2C49
:10CB7000B091AE2C8093202790932127A093222759
:10CB8000B0932327DFC31092331780E0C0E0D0E0DA
:10CB900022C0E82FF0E075E0EE0FFF1F7A95E1F775
:10CBA000E55EF34D918D992321F480933317EF01C6
:10CBB00016C0973079F4209721F0228D9A8D921724
:10CBC00048F4C82FD0E065E0CC0FDD1F6A95E1F78F
:10CBD000C55ED34D8F5F8430E0F28093331720978A
:10CBE00009F4EEC3D0931A2CC093192C83E08A8FDA
:10CBF000888F1E8A84E08F8B1B8E80912A279091CC
:10CC00002B279D838C8380912827909129279F83B0
:10CC10008E838091202790912127A0912227B09187
:10CC2000232788839983AA83BB8381E0898F80919E
:10CC300036178C87809137178D87809138178E87AC
:10CC4000809139178F8781E090E0998B888B809154
:10CC50002F278B8780912E278A8780912D27898780
:10CC600080912C27888781E090E00E941C6B809146
:10CC70003427282F30E0207F3070213531050CF427
:10CC800046C082958F7090E00597880F991F880F96
:10CC9000991F30913C1720E031C0EC5EF84D30A573
:10CCA000332329F42093331710923C1730C03130CE
:10CCB00011F42F5F23C03230E9F441A54430D1F4A0
:10CCC0002093331730933C1792A580E023A530E0E2
:10CCD000282B392B30933B1720933A17C90124E0B6
:10CCE000893D920710F088ED94E09B8B8A8B9D8B99
:10CCF0008C8B0DC041A5442331F0240FE22FF0E0CE
:10CD0000E817F90754F22093331730933C1780E16A
:10CD1000809335278091352782608093352782E084
:10CD200080933C2784E080933D2780933E2788EDC5
:10CD300080933F278CE290E090930D2780930C27FF
:10CD400080E6ADC2D0931A2CC093192C1092142CEB
:10CD50004091352750E042FF03C0198E80E248C25F
:10CD60008091342782958F70880F880F80933317B6
:10CD70009801281B31092451304030930D2720930E
:10CD80000C27862F90E08F7090708230910539F4D7
:10CD9000CA018F7390708231910551F429C081309E
:10CDA000910531F4CA018F7390708230910501F1C1
:10CDB0002115310529F4CA01837090700097C1F0E4
:10CDC00090912C278885981709F05FC290912D27A4
:10CDD0008985981709F059C290912E278A8598174E
:10CDE00009F053C290912F278B85981709F04DC2F7
:10CDF00044FF4AC0688979896115710509F444C006
:10CE0000CE010C960E94BF60309130278091102790
:10CE10003817D1F520913127809111272817A1F5D6
:10CE20009091322780911227981771F580913327BE
:10CE300040911327841741F53C872D879E878F8764
:10CE40008B8D8823D1F42E89888D9A8D891B922F02
:10CE5000969596959695891B280F2E8B87FD819523
:10CE60009F89392F36953695931B980F9F8B822F6C
:10CE7000869586958695890F888F81E08093142CFE
:10CE8000888D8A8F198A188A498D50E0CA018F705F
:10CE900090708430910509F4B0C18530910564F437
:10CEA00082309105C9F1833091050CF0B6C0813014
:10CEB000910509F085C211C08630910509F4DDC1E4
:10CEC000863091050CF4B9C18730910509F4DDC1B4
:10CED0008830910509F074C285C18091142C80FFBF
:10CEE00014C083E0898F80E48093142C198A188AF7
:10CEF00080910C2790910D27009709F408C122E436
:10CF00002093142C0E941C6B02C1809135278F73D3
:10CF1000823009F055C2FBCE8091142C80FF72C084
:10CF2000809135278F73823109F06CC0809134274E
:10CF3000282F30E0207F3070213531050CF446C0B9
:10CF400082958F7090E00597880F991F880F991F21
:10CF500030913C1720E031C0EC5EF84D30A5332312
:10CF600029F42093331710923C1730C0313011F45C
:10CF70002F5F23C03230E9F441A54430D1F420932F
:10CF8000331730933C1792A580E023A530E0282B7F
:10CF9000392B30933B1720933A17C90124E0893D80
:10CFA000920710F088ED94E09B8B8A8B9D8B8C8B85
:10CFB0000DC041A5442331F0240FE22FF0E0E81723
:10CFC000F90754F22093331730933C1783E0898F8D
:10CFD00080912C27888780912D27898780912E2703
:10CFE0008A8780912F278B8781E090E00E941C6BBD
:10CFF00082E48093142C198A188A10920D271092BB
:10D000000C2785C080E28093142C0E94DE5CE091A6
:10D01000192CF0911A2C118E3DCD8091352780FF6F
:10D0200025C044FD23C088899989009709F0C8C1AB
:10D0300080910C2790910D2701960E941C6B2091E6
:10D04000142C822F80618093142C80910C27909156
:10D050000D27009719F022612093142C0E94DE5CAA
:10D0600081E090E0998B888B88E06DC085FF1CC0C3
:10D0700090913A2780E020913B2730E0282B392BF4
:10D080008091172C9091182C820F931F9093182C3D
:10D090008093172C80910C2790910D27821B930B66
:10D0A00090930D2780930C2780910C2790910D274A
:10D0B000009749F044FD07C02091142C2260209372
:10D0C000142C0E941C6B9091362780E0209137270A
:10D0D000820F911D90933B1780933A172C893D89BD
:10D0E0002817390710F0009721F430933B1720934D
:10D0F0003A1780913A1790913B179B8B8A8B8091BE
:10D10000142C90E083709070009709F459C110922C
:10D11000B02C1092AF2C0E94DE5C2091142C25FFC5
:10D1200007C01092B02C1092AF2C198E84E1AEC0C3
:10D1300024FF0DC01092B02C1092AF2C81E090E033
:10D14000998B888B84E0898F1B8E81E19FC08091B1
:10D15000AF2C9091B02C0097E9F020FF02C0198A03
:10D16000188A288939892115310581F42A893B8952
:10D170002817390720F43093B02C2093AF2C8091DE
:10D18000AF2C9091B02C998B888B04C03093B02C2D
:10D190002093AF2C1B8E80910E2790910F27909398
:10D1A000182C8093172C8091AF2C9091B02C009765
:10D1B00059F088899989009739F0889690930D27BE
:10D1C00080930C2788E10BC08091142C81FFF8C05C
:10D1D00088E290E090930D2780930C2780E1809364
:10D1E00035275CC08091142C80FFEAC0198E80E145
:10D1F0008093142C0E94DE5CE3C080910C279091F8
:10D200000D27009711F00E941C6B9091352780919B
:10D21000142C90FF0BC080FF06C087E0898F1A8E08
:10D22000198A188A19C086E0898F16C080FF1EC02F
:10D2300085E0898F198A188AC3C080910C27909144
:10D240000D27009711F00E941C6B8091352780FFFD
:10D250000DC087E0898F1A8E81E090E00E941C6BE0
:10D2600080E18093142C0E94DE5C0FC080910C271B
:10D2700090910D27009749F4A3C08091142C80FF52
:10D280009FC087E0898F1A8E9BC080E180933527ED
:10D2900088E290E090930D2780930C2780E580939F
:10D2A00034278885809330278985809331278A8524
:10D2B000809332278B85809333278C8580932C270E
:10D2C0008D8580932D278E8580932E278F85809343
:10D2D0002F2786E080931D278C819D81909329279D
:10D2E000809328278E819F8190932B2780932A27D4
:10D2F0008091AB2C9091AC2CA091AD2CB091AE2C28
:10D300008093202790932127A0932227B09323274F
:10D3100088819981AA81BB818093242790932527B6
:10D32000A0932627B0932727898D84FF05C01092EC
:10D3300037271092362706C084E08093362788ED81
:10D340008093372780E480931C2780910C2790914D
:10D350000D27909316278093172710923B27109242
:10D360003A2710923927109238270E94136180952E
:10D370009095909339278093382785E480931427DC
:10D380001092152710921B2710921A27809131179F
:10D3900090913217019690933217809331179093A2
:10D3A00018278093192710921F2710921E270E947A
:10D3B00002618095909590931F2780931E2704C04B
:10D3C00010920D2710920C271092142CDF91CF9100
:10D3D0001F910F91FF90EF90DF90CF90BF90AF9093
:10D3E000089598278927982708950F931F93DC01A4
:10D3F000CB011A2F0B2F20E030E0982789279827A0
:10D40000A0E0B0E0DC0199278827082B192B2A2BF4
:10D410003B2BB801C9011F910F910895FC01209188
:10D420000E2730910F2784E19CE2821B930BAB0106
:10D43000861797070CF4AC01141615065CF440939C
:10D44000AF2C5093B02CE217F30721F0C901BF01B4
:10D450000E94A7750895CF92DF92EF92FF920F93EB
:10D46000CF93DF93CDB7DEB760970FB6F894DEBFEA
:10D470000FBECDBF002309F45AC029873A874B87D6
:10D480005C876D877E878F87988B80E2801B4985BC
:10D490005A856B857C851816B4F019821A821B8216
:10D4A0001C82992787FD9095909581959F4F04C088
:10D4B000440F551F661F771F8A95D2F74D835E83F1
:10D4C0006F8378872CC06A017B01002E04C0CC0CCE
:10D4D000DD1CEE1CFF1C0A94D2F7C982DA82EB82B3
:10D4E000FC826A017B0104C0F694E794D794C79448
:10D4F0008A95D2F7D701C6014D855E856F857889FB
:10D5000004C0440F551F661F771F0A95D2F7842B5E
:10D51000952BA62BB72B8D839E83AF83B88729814C
:10D520003A814B815C816D817E818F819885609687
:10D530000FB6F894DEBF0FBECDBFDF91CF910F9134
:10D54000FF90EF90DF90CF900895A0E1B0E0EBEA7C
:10D55000FAE60C94C07229873A874B875C876D87FF
:10D560007E878F87988BA982BA82CB82DC82ED82FC
:10D57000FE820F8318874D855E856F8578898D8142
:10D580009E81AF81B885481759076A077B07C8F0A5
:10D5900084179507A607B70790F049855A856B85CC
:10D5A0007C8589819A81AB81BC81481759076A07BC
:10D5B0007B0738F084179507A607B70720F482E0A9
:10D5C00003C080E001C081E06096EAE00C94DC7268
:10D5D00080E880936100109261000E9413470E94CE
:10D5E000AE390E94724B8091BB249091BC2400976D
:10D5F00029F001979093BC248093BB24C090BD2454
:10D60000D090BE24E090BF24F090C0240E94174A1E
:10D61000DC01CB01C816D906EA06FB0601F30E941D
:10D62000174ADC01CB018093BD249093BE24A093C4
:10D63000BF24B093C024D3CFBC018091192C90910A
:10D640001A2C08960E94BF60E091192CF0911A2CB8
:10D6500080911027808780911127818780911227E0
:10D66000828780911327838708952F923F924F924C
:10D670005F926F927F928F929F92AF92BF92CF9262
:10D68000DF92EF92FF920F931F93CF93DF93CDB76B
:10D69000DEB765970FB6F894DEBF0FBECDBF4C0165
:10D6A0007F876E87FC0117821682838181FD04C00B
:10D6B00076C34C855D8504C01E010894211C311C75
:10D6C000F4019381EE85FF8593FD859193FF819110
:10D6D000FF87EE87882309F45EC3853241F493FD0A
:10D6E000859193FF8191FF87EE87853259F490E011
:10D6F000B4014C8B5D8B0E94FA754C895D895D8706
:10D700004C87D7CFFF24DD2410E01032B0F48B32E9
:10D7100069F08C3228F4803251F0833271F40BC0FE
:10D720008D3239F0803349F411602CC012601460DE
:10D7300029C0186027C0106125C017FD2EC0282FF2
:10D7400020532A3098F416FF08C08F2D880FF82E2A
:10D75000FF0CFF0CF80EF20E15C08D2D880FD82E81
:10D76000DD0CDD0CD80ED20E10620CC08E3221F40E
:10D7700016FD11C3106406C08C3611F4106802C087
:10D78000883659F4EE85FF8593FD859193FF81914D
:10D79000FF87EE87882309F0B8CF982F95549330F0
:10D7A00018F41061805E06C0982F9556933008F0EB
:10D7B000A2C11F7E16FD02C0E6E0FE2E1F73853655
:10D7C00011F4106406C0863611F4106802C0F1101E
:10D7D000FA9417FF07C0FBE3FF1548F0EF2CE39422
:10D7E00027E00DC027E02F1530F02F2D07C027E0D0
:10D7F0007CE3E72E04C027E067E0F62EEE24CA01A2
:10D8000004969D878C87FA01608171818281938162
:10D81000A1010E2D0E94B7745C01C9802C2D30E04F
:10D82000398B288BC0FE03C0388933FF06C011FD39
:10D8300006C012FF06C000E205C00DE203C00BE205
:10D8400001C000E0888999898C709070009709F474
:10D850003CC0002311F084E001C083E08D1558F432
:10D86000D81A13FD09C080E290E0B4010E94FA7555
:10D87000DA94C9F701C0DD24002329F0802F90E05D
:10D88000B4010E94FA75888983FD05C03EECE32E41
:10D890003EE0F32E11C02AECE22E2EE0F22E0CC058
:10D8A0000115110509F0805290E0B4010E94FA754B
:10D8B0000894E11CF11C04C0012F10E000711070ED
:10D8C000F7018491882361F763C217FF0EC0EA0C49
:10D8D000F889F4FF04C08A81813309F4EA941E14A4
:10D8E0004CF528E02E1548F12CC016FD2AC08F2DCE
:10D8F00090E08A159B0544F03CEFA3163FEFB3067A
:10D900001CF0106801C0FA94FF2049F0E2E0F0E05A
:10D91000EC0FFD1FEF0DF11D80818033A1F317FF88
:10D9200010C0EF2CE3948F2D90E0A816B90644F4B4
:10D93000FA1807C0EE24E39404C098E0E92E01C071
:10D94000FF2417FF07C01A141B043CF495012F5F36
:10D950003F4F05C025E030E002C021E030E0002369
:10D9600011F02F5F3F4FFF2029F08F2D90E001969F
:10D97000280F391F8D2D90E02817390714F4D21A7B
:10D9800001C0DD24612E7724C30189709070009757
:10D9900049F406C080E290E0B4010E94FA75DA947E
:10D9A000DD20C1F7002329F0802F90E0B4010E9410
:10D9B000FA7563FC09C006C080E390E0B4010E94E0
:10D9C000FA75DA94DD20C1F717FF48C08501B7FE6C
:10D9D00002C000E010E04424552495012E193109BD
:10D9E0003B8B2A8B3501601A710A620C731C6F2DF8
:10D9F00070E0EE24FF24E61AF70A3FEF0F3F13070B
:10DA000029F48EE290E0B4010E94FA75A016B106E6
:10DA100054F02A893B89201731072CF4F301E40DD7
:10DA2000F51D818101C080E3015010400894411C24
:10DA3000511C0E151F052CF090E0B4010E94FA75E0
:10DA4000DCCF0A151B0541F49A81963320F49533F7
:10DA500019F4388934FF81E390E049C08A81813329
:10DA600011F09FEEC92290E0B4010E94FA75FF20E8
:10DA700089F08EE290E0B4010E94FA7512E0F101A3
:10DA8000E10FF11D1F5F808190E0B4010E94FA75E3
:10DA9000FA94A9F764FE03C085E490E002C085E62D
:10DAA00090E0B4010E94FA75B7FC05C0A114B1045E
:10DAB00041F4C4FE06C0B094A194B108B3948DE2C1
:10DAC00001C08BE290E0B4010E94FA7580E305C0CA
:10DAD0008F5FE6EFFFEFAE0EBF1EFAE0AF16B104A8
:10DAE000BCF790E0B4010E94FA75C501C096B4017C
:10DAF0000E94FA754DC1833631F0833789F0833542
:10DB000009F059C022C09A012E5F3F4F3D872C87F4
:10DB1000FA018081898381E0E82EF12C510113C044
:10DB20009A012E5F3F4F3D872C87FA01A080B1807C
:10DB300016FF03C06F2D70E002C06FEF7FEFC501CD
:10DB40000E94C0757C011F7714C09A012E5F3F4F61
:10DB50003D872C87FA01A080B18016FF03C06F2D8E
:10DB600070E002C06FEF7FEFC5010E9497757C01E6
:10DB7000106813FD1CC006C080E290E0B4010E9452
:10DB8000FA75DA948D2D90E0E816F906A8F30FC027
:10DB9000F50117FD859117FF81915F0190E0B401B8
:10DBA0000E94FA75D110DA940894E108F108E114A2
:10DBB000F10471F7EDC0843611F0893671F59A01E0
:10DBC00017FF0AC02C5F3F4F3D872C87FA018081E9
:10DBD0009181A281B3810BC02E5F3F4F3D872C877F
:10DBE000FA0180819181AA2797FDA095BA2F012F74
:10DBF0000F76B7FF08C0B095A095909581959F4F7F
:10DC0000AF4FBF4F0068BC01CD01A1012AE030E059
:10DC10000E940277E82EE21841C0853721F41F7E6A
:10DC20002AE030E020C0197F8F36A9F0803720F439
:10DC3000883509F0B0C00BC0803721F0883709F073
:10DC4000AAC001C0106114FF09C0146007C014FF0E
:10DC500008C0166006C028E030E005C020E130E0D2
:10DC600002C020E132E0CA0117FF09C004969D8777
:10DC70008C87FA01608171818281938108C002964C
:10DC80009D878C87FA016081718180E090E0A1011D
:10DC90000E940277E82EE218012F0F7706FF09C0D5
:10DCA0000E7FEF1430F404FF06C002FD04C00F7EA7
:10DCB00002C01E2D01C01F2D802F90E004FF0CC05C
:10DCC000FE01EE0DF11D2081203311F4097E09C003
:10DCD00002FF06C01E5F05C086789070009709F0AD
:10DCE0001F5FA02EBB2403FD12C000FF0DC0FE2C41
:10DCF0001D1550F4FD0CF11A1D2D06C080E290E0B8
:10DD0000B4010E94FA751F5F1D15C0F304C01D15F4
:10DD100010F4D11A01C0DD24A4FE0FC080E390E00E
:10DD2000B4010E94FA75A2FE1FC0A1FE03C088E5DF
:10DD300090E010C088E790E00DC0C5018678907033
:10DD4000009791F0A1FC02C080E201C08BE207FDC8
:10DD50008DE290E0B4010E94FA7506C080E390E085
:10DD6000B4010E94FA75FA94EF14C0F3EA94F10139
:10DD7000EE0DF11D808190E0B4010E94FA75EE2055
:10DD8000A9F706C080E290E0B4010E94FA75DA9427
:10DD9000DD20C1F78ECCF4018681978102C08FEF20
:10DDA0009FEF65960FB6F894DEBF0FBECDBFDF9133
:10DDB000CF911F910F91FF90EF90DF90CF90BF9088
:10DDC000AF909F908F907F906F905F904F903F901B
:10DDD0002F9008955058BB27AA270ED044C135D1A3
:10DDE00030F03AD120F031F49F3F11F41EF42AC1F3
:10DDF0000EF4E095E7FB20C1E92F46D180F3BA1776
:10DE0000620773078407950718F071F49EF55EC1E9
:10DE10000EF4E0950B2EBA2FA02D0B01B901900145
:10DE20000C01CA01A0011124FF27591B99F0593F89
:10DE300050F4503E68F11A16F040A22F232F342FD1
:10DE40004427585FF3CF469537952795A795F0401F
:10DE50005395C9F77EF41F16BA0B620B730B840B34
:10DE6000BAF09150A1F0FF0FBB1F661F771F881FEC
:10DE7000C2F70EC0BA0F621F731F841F48F4879544
:10DE800077956795B795F7959E3F08F0B3CF939533
:10DE9000880F08F09927EE0F979587950895A8D0D9
:10DEA00008F481E008950CD0DEC0D6D040F0CDD08B
:10DEB00030F021F45F3F19F0BFC0511108C1C2C05A
:10DEC000E3D098F39923C9F35523B1F3951B550B70
:10DED000BB27AA2762177307840738F09F5F5F4F3D
:10DEE000220F331F441FAA1FA9F333D00E2E3AF07E
:10DEF000E0E830D091505040E695001CCAF729D098
:10DF0000FE2F27D0660F771F881FBB1F26173707E6
:10DF10004807AB07B0E809F0BB0B802DBF01FF2716
:10DF200093585F4F2AF09E3F510568F085C0CFC0DF
:10DF30005F3FECF3983EDCF3869577956795B79550
:10DF4000F7959F5FC9F7880F911D9695879597F96B
:10DF50000895E1E0660F771F881FBB1F62177307E4
:10DF60008407BA0720F0621B730B840BBA0BEE1FF9
:10DF700088F7E0950895E89409C097FB3EF49095E2
:10DF80008095709561957F4F8F4F9F4F9923A9F092
:10DF9000F92F96E9BB279395F69587957795679521
:10DFA000B795F111F8CFFAF4BB0F11F460FF1BC065
:10DFB0006F5F7F4F8F4F9F4F16C0882311F096E9F8
:10DFC00011C0772321F09EE8872F762F05C06623A6
:10DFD00071F096E8862F70E060E02AF09A95660F5F
:10DFE000771F881FDAF7880F9695879597F9089518
:10DFF000990F0008550FAA0BE0E8FEEF161617065A
:10E00000E807F907C0F012161306E407F50798F0C1
:10E01000621B730B840B950B39F40A2661F0232BDA
:10E02000242B252B21F408950A2609F4A140A69556
:10E030008FEF811D811D089597F99F6780E870E03B
:10E0400060E008959FEF80EC089500240A9416166E
:10E05000170618060906089500240A9412161306D6
:10E06000140605060895092E0394000C11F4882364
:10E0700052F0BB0F40F4BF2B11F460FF04C06F5F80
:10E080007F4F8F4F9F4F089557FD9058440F551F56
:10E0900059F05F3F71F04795880F97FB991F61F02A
:10E0A0009F3F79F087950895121613061406551FA1
:10E0B000F2CF4695F1DF08C0161617061806991F0D
:10E0C000F1CF86957105610508940895E894BB2702
:10E0D00066277727CB0197F908950BD0C4CFB5DF1A
:10E0E00028F0BADF18F0952309F0A6CFABCF1124A2
:10E0F000EECFCADFA0F3959FD1F3950F50E0551FE7
:10E10000629FF001729FBB27F00DB11D639FAA278C
:10E11000F00DB11DAA1F649F6627B00DA11D661FDB
:10E12000829F2227B00DA11D621F739FB00DA11DFC
:10E13000621F839FA00D611D221F749F3327A00DB6
:10E14000611D231F849F600D211D822F762F6A2F52
:10E1500011249F5750408AF0E1F088234AF0EE0FD7
:10E16000FF1FBB1F661F771F881F91505040A9F7E4
:10E170009E3F510570F060CFAACF5F3FECF3983E11
:10E18000DCF3869577956795B795F795E7959F5F4B
:10E19000C1F7FE2B880F911D9695879597F90895E5
:10E1A000FA01EE0FFF1F30962105310599F1611537
:10E1B000710561F48038BFE39B0749F1689490389A
:10E1C000810561F08038BFEF9B0741F0992342F54C
:10E1D000FF3FE1053105210511F1E8940894E79529
:10E1E000D901AA2329F4AB2FBE2FF85FD0F310C0BA
:10E1F000FF5F70F4A695E0F7F73950F019F0FF3A99
:10E2000038F49F779F930CD00F9007FC9058089597
:10E210003EF018CF60E070E080E89FE308954FE79C
:10E220009F775F934F933F932F939ED02F913F9172
:10E230004F915F9152DF05C019F40EF0FDCE46CF2D
:10E2400001CF2ADFC8F39638C0F707F80F92E89499
:10E250002BE33AEA48EB5FE74EDF0F920F920F9203
:10E260004DB75EB70F92C0D0E0E2F1E016D04F910B
:10E270005F91EF91FF91E595EE1FFF1F49F0FE576B
:10E28000E0684427EE0F441FFA95E1F74195550BDE
:10E2900032D00F9007FE26C00895DF93CF931F93CF
:10E2A0000F93FF92EF92DF927B018C01689405C07F
:10E2B000DA2EEF011EDFFE01E894A591259135913C
:10E2C00045915591AEF3EF0197DDFE019701A8014D
:10E2D000DA9479F7DF90EF90FF900F911F91CF9133
:10E2E000DF9108959B01AC0160E070E080E89FE35E
:10E2F000DACDA2CEACC0D0DEE8F39923D9F3940FE7
:10E30000511DBBF39150504094F059F0882332F0E6
:10E31000660F771F881F91505040C1F79E3F5105EF
:10E3200044F7880F911D9695879597F908955F3F5B
:10E33000ACF0983E9CF0BB27869577956795B7958E
:10E3400008F4B1609395C1F7BB0F58F711F460FF63
:10E35000E8CF6F5F7F4F8F4F9F4FE3CFB8CE0EF068
:10E3600076C070CE689468CE97DEC8F39923D1F357
:10E37000C6F3DF93CF931F930F93FF92C92FDD272F
:10E3800088232AF02197660F771F881FDAF720E08D
:10E3900030E040E85FEB9FE3883920F0803E30F0CA
:10E3A00021968F7718DDE8E4F1E003C014DDE5E79E
:10E3B000F1E073DF8B01BE01EC01FB2E6F57710999
:10E3C0007595771F880B990BD8DD28E132E741E37B
:10E3D0005FE38FDEAF2D9801AE01FF900F911F918B
:10E3E000CF91DF9109DD3FCEFA01DC01AA0FBB1FFF
:10E3F0009B01AC01BF5728F42227332744275078CC
:10E400001FC0B75188F4AB2F002446953795279548
:10E41000011CA395D2F3002069F0220F331F441F83
:10E42000B395DAF30DD0D6CC61307105A0E88A0738
:10E43000B94630F49B01AC0166277727882790788E
:10E44000309621F0208331834283538308959F3F88
:10E4500031F0915020F4879577956795B795880F9F
:10E46000911D9695879597F90895629FD001739FA6
:10E47000F001829FE00DF11D649FE00DF11D929F60
:10E48000F00D839FF00D749FF00D659FF00D99279F
:10E49000729FB00DE11DF91F639FB00DE11DF91FC3
:10E4A000BD01CF0111240895AA1BBB1B51E107C078
:10E4B000AA1FBB1FA617B70710F0A61BB70B881F14
:10E4C000991F5A95A9F780959095BC01CD010895A3
:10E4D00097FB092E07260AD077FD04D0E5DF06D08A
:10E4E00000201AF4709561957F4F0895F6F7909586
:10E4F00081959F4F0895A1E21A2EAA1BBB1BFD0117
:10E500000DC0AA1FBB1FEE1FFF1FA217B307E40712
:10E51000F50720F0A21BB30BE40BF50B661F771F6A
:10E52000881F991F1A9469F760957095809590954A
:10E530009B01AC01BD01CF01089597FB092E052673
:10E540000ED057FD04D0D7DF0AD0001C38F4509508
:10E550004095309521953F4F4F4F5F4F0895F6F707
:10E5600090958095709561957F4F8F4F9F4F08953F
:10E570002F923F924F925F926F927F928F929F92D3
:10E58000AF92BF92CF92DF92EF92FF920F931F93C1
:10E59000CF93DF93CDB7DEB7CA1BDB0B0FB6F89472
:10E5A000DEBF0FBECDBF09942A88398848885F84B2
:10E5B0006E847D848C849B84AA84B984C884DF8023
:10E5C000EE80FD800C811B81AA81B981CE0FD11D07
:10E5D0000FB6F894DEBF0FBECDBFED0108958F9248
:10E5E0009F92AF92BF92CF92DF92EF92FF92CF9322
:10E5F000DF93EC0188819981AA81BB810097A105F5
:10E60000B10521F484E299EDABE5B7E0BC01CD01A1
:10E610002DE133EF41E050E00E949D7249015A0123
:10E6200027EA31E440E050E00E9435726B017C0142
:10E63000C501B4012CEE34EF4FEF5FEF0E9435724D
:10E64000DC01CB01C80ED91EEA1EFB1EF7FE08C076
:10E650008FEF9FEFAFEFBFE7C80ED91EEA1EFB1E7C
:10E66000C882D982EA82FB82C6019F77DF91CF916F
:10E67000FF90EF90DF90CF90BF90AF909F908F90E2
:10E6800008950E94EF7208958DE896E00E94EF725F
:10E690000895A0E0B0E080938D0690938E06A0933D
:10E6A0008F06B093900608953F924F925F926F92BB
:10E6B0007F928F929F92AF92BF92CF92DF92EF9212
:10E6C000FF920F931F93CF93DF9300D000D0CDB76D
:10E6D000DEB72B017A016115710529F0DB018C93FE
:10E6E00011969C931197E114F10439F0970122508F
:10E6F00030402332310508F0FCC06C0186010894DB
:10E70000C11CD11CF80130803601832D90E00E949D
:10E710008F75009799F7FDE23F1661F4D8011196C5
:10E720003C90119792E0692E712C600E711ECC24E2
:10E73000C3940BC0BBE23B1639F4F801318082E090
:10E74000682E712C600E711ECC24E114F10421F0AE
:10E75000F0E1EF16F104F9F480E3381691F4D301F7
:10E760008C91883711F0883561F4F301318082E0B3
:10E7700090E0680E791E92E0C92AB0E1EB2EF12CF0
:10E780000AC0E114F10439F4A0E33A16D1F0AAE08A
:10E79000EA2EF12C30C0BAE0EB16F10461F1E0E1B1
:10E7A000EE16F10429F0F8E0EF16F104B1F409C017
:10E7B000FFEF8F2EFFEF9F2EFFEFAF2EFFE0BF2E5C
:10E7C00022C078E0E72EF12CEFEF8E2EEFEF9E2E99
:10E7D000EFEFAE2EEFE1BE2E16C09701442737FDB6
:10E7E0004095542F6FEF7FEF8FEF9FEF0E947B726A
:10E7F00049015A0108C069E9862E69E9962E69E93E
:10E80000A62E69E1B62E40E000E010E020E030E006
:10E81000C701AA2797FDA095BA2F89839A83AB8356
:10E82000BC8350EDD52ED30C99E09D1570F4832D4B
:10E8300081548A3118F499ECD92E06C0832D815663
:10E840008A3168F589EAD82ED30C8D2D90E08E158B
:10E850009F052CF54F3FF9F080169106A206B306EE
:10E86000B8F0C901B80129813A814B815C810E94CD
:10E8700035728B019C018D2D90E0A0E0B0E0080F77
:10E88000191F2A1F3B1F081719072A073B0710F4F7
:10E890004FEF01C041E0D3013D903D01C2CF411493
:10E8A000510489F0442339F0089461087108F20199
:10E8B0007182608208C0C1FE06C0C3010297D20106
:10E8C00011969C938E93C0FE07C0309520951095AD
:10E8D00001951F4F2F4F3F4F47FF0FC082E290E03F
:10E8E00090933A2D8093392D0FEF1FEF2FEF3FEFCD
:10E8F00004C000E010E020E030E0B801C9010F9052
:10E900000F900F900F90DF91CF911F910F91FF907B
:10E91000EF90DF90CF90BF90AF909F908F907F90BF
:10E920006F905F904F903F900895662777270C94E3
:10E930009B77FC0188279927E89421912032E9F3FD
:10E94000293010F02E30C8F32B3241F02D3239F43B
:10E95000689404C00E94F275820F911D219120538A
:10E960002A30C0F31EF4909581959F4F089528306A
:10E9700008F027E03327DA01990F311D87FD9160F8
:10E9800000966105710539F432602E5F3D9330E3E6
:10E990002A95E1F708959F3F30F0803871056105B1
:10E9A00009F03C5F3C5F3D93913008F08068911D19
:10E9B000DF93CF931F930F93FF92EF92192F987FBE
:10E9C0009695E92F96959695E90FFF27E45DF04F10
:10E9D00099273327EE24FF24A701E7010590089427
:10E9E000079428F4360FE71EF81E491F511D660FC5
:10E9F000771F881F991F0694A1F70590079428F4A4
:10EA0000E70EF81E491F561FC11D770F881F991F5B
:10EA1000661F0694A1F70590079428F4F80E491F85
:10EA2000561FC71FD11D880F991F661F771F069499
:10EA3000A1F70590079420F4490F561FC71FD81F50
:10EA4000990F661F771F881F0694A9F78491109568
:10EA5000177041F0D695C79557954795F794E79469
:10EA60001A95C1F7E2EDFEE0689415901591359185
:10EA70006591959105907FE27395E118F10A430B3A
:10EA8000560BC90BD009C0F7E10CF11E431F561FEE
:10EA9000C91FD01D7EF4703311F48A95E6CFE89437
:10EAA000015030F0080F0AF40027021708F4202F55
:10EAB0002395022F7A3328F079E37D932A95E9F79D
:10EAC00010C07D932A9589F606949795679537959A
:10EAD00017951794E118F10A430B560BC90BD0098F
:10EAE00098F023957E9173957A3308F070E37C93C8
:10EAF0002013B8F77E9170617D9330F0839571E3B8
:10EB00007D9370E32A95E1F71124EF90FF900F9128
:10EB10001F91CF91DF91992787FD909508959111CD
:10EB200089C3803219F089508550D0F70895FC01CF
:10EB30000590615070400110D8F7809590958E0F28
:10EB40009F1F08954DE357E10E94CB750895FB0187
:10EB5000DC0102C001900D9241505040D8F7089559
:10EB6000DC0101C06D9341505040E0F70895FB0176
:10EB7000DC018D91019080190110D9F3990B089552
:10EB8000FC016150704001900110D8F7809590957C
:10EB90008E0F9F1F0895FA01A191B081009719F47B
:10EBA0001097E1F0CD01DC01CD010D90002011F4B2
:10EBB000C00113C0FB012191222319F02015D9F7C0
:10EBC000F3CFFB012191201519F41E92119606C076
:10EBD0002223C1F70D900020A1F7D001FA01A193E3
:10EBE000B08308957AE0979F902D879F802D910D97
:10EBF000112408950F931F93CF93DF938C01EB01A2
:10EC00008B8181FF1BC082FF0DC02E813F818C81D3
:10EC10009D812817390764F4E881F9810193F9830C
:10EC2000E88306C0E885F985802F0995009731F4BF
:10EC30008E819F8101969F838E8302C00FEF1FEF0D
:10EC4000C801DF91CF911F910F910895CF93DF936A
:10EC5000CDB7DEB7FE013596619171918091352D6A
:10EC60009091362DAF010E94356BDF91CF910895C1
:10EC7000CF93DF93CDB7DEB7FE01359661917191E9
:10EC80008091352D9091362DDC0113962C911397A0
:10EC9000286013962C93AF010E94356BE091352DBF
:10ECA000F091362D2381277F2383DF91CF91089523
:10ECB0006091352D7091362D0E94FA7508950F934D
:10ECC0001F93CF93DF938C01E091352DF091362D7A
:10ECD000838181FF1AC0C0E0D0E005C0099500978C
:10ECE00011F0CFEFDFEFF80181918F016091352DA9
:10ECF0007091362DDB011896ED91FC9119978823C0
:10ED000069F78AE00995009711F0CFEFDFEFCE01A8
:10ED1000DF91CF911F910F9108950F931F93CF9380
:10ED2000DF93CDB7DEB72E970FB6F894DEBF0FBED8
:10ED3000CDBF0D891E898F89988D26E02C831A837B
:10ED4000098397FF02C080E090E801979E838D833E
:10ED5000AE01455E5F4FCE010196698D7A8D0E94AE
:10ED6000356B4D815E8157FD0AC02F813885421772
:10ED700053070CF49A01020F131FF80110822E960C
:10ED80000FB6F894DEBF0FBECDBFDF91CF911F91BC
:10ED90000F9108950F931F93CF93DF93CDB7DEB7F5
:10EDA0002E970FB6F894DEBF0FBECDBF8C0186E064
:10EDB0008C831A83098377FF02C060E070E861509A
:10EDC00070407E836D83CE010196BA01A9010E9435
:10EDD000356B4D815E8157FD0AC02F813885421702
:10EDE00053070CF49A01020F131FF80110822E969C
:10EDF0000FB6F894DEBF0FBECDBFDF91CF911F914C
:10EE00000F910895FA01AA27283051F1203181F19C
:10EE1000E8946F936E7F6E5F7F4F8F4F9F4FAF4F22
:10EE2000B1E03ED0B4E03CD0670F781F891F9A1F35
:10EE3000A11D680F791F8A1F911DA11D6A0F711DE9
:10EE4000811D911DA11D20D009F468943F912AE0F5
:10EE5000269F11243019305D3193DEF6CF010895DD
:10EE6000462F4770405D4193B3E00FD0C9F7F6CF0E
:10EE7000462F4F70405D4A3318F0495D31FD4052D6
:10EE8000419302D0A9F7EACFB4E0A695979587956C
:10EE900077956795BA95C9F700976105710508954B
:10EEA0009B01AC010A2E06945795479537952795F7
:10EEB000BA95C9F7620F731F841F951FA01D08958F
:10EEC000DC01CB01FC01F999FECF06C0F2BDE1BD2A
:10EED000F89A319600B40D9241505040B8F7089519
:10EEE000F999FECF92BD81BDF89A992780B5089512
:10EEF000A8E1B0E042E050E00C946277DC01CB0185
:10EF000003C02D910E94897741505040D0F7089559
:10EF1000262FF999FECF1FBA92BD81BD20BD0FB635
:10EF2000F894FA9AF99A0FBE019608950E9488778C
:10EF3000272F0C9489776F927F928F929F92AF9236
:10EF4000BF92CF92DF92EF92FF920F931F93CF93D6
:10EF5000DF935B016115710521F0DB018C93119644
:10EF60009C937C01E7010894E11CF11C0881670176
:10EF7000802F90E00E948F750097A1F70D3241F429
:10EF8000098142E0C42ED12CCC0EDD1E11E009C057
:10EF90000B3231F4098132E0C32ED12CCC0EDD1EB0
:10EFA00010E0E6012197CE016CEC7FE043E050E0F9
:10EFB0000E941D790097D1F4E6012296CE016FECF4
:10EFC0007FE045E050E00E941D79009711F4E601D2
:10EFD0002796A114B10419F0F501D183C08330E064
:10EFE00020E090E8112309F40DC107C1CE0164EDC2
:10EFF0007FE043E050E00E941D79009759F4A1148E
:10F00000B10409F4FCC0C6010296D50111969C9387
:10F010008E93F5C040E050E060E070E088249924D1
:10F0200000530A3090F51260212F30E0C90188703A
:10F03000907012FF06C0009769F50894811C911C1E
:10F0400029C0009719F0089481089108DB01CA01D2
:10F05000D2E0880F991FAA1FBB1FDA95D1F7480F7E
:10F06000591F6A1F7B1F440F551F661F771F400FD4
:10F07000511D611D711D4839B9E95B07B9E96B077D
:10F08000B9E17B0738F0146005C00E3F39F413FD79
:10F0900043C01860F60101916F01C2CF053311F032
:10F0A0000531D1F5D601EC91ED3211F4106108C0B3
:10F0B000EB3229F0C601019621E030E008C0D6010C
:10F0C0001196EC911197C601029622E030E0E053D0
:10F0D000EA3020F06C01C21AD30A1EC0DC0120E025
:10F0E00030E0FCE020383F075CF4C901880F991F2D
:10F0F000880F991F280F391F220F331F2E0F311D24
:10F10000ED91E0536D01EA3060F314FF03C03095D8
:10F1100021953F4F820E931EC12FD0E011FF08C0F2
:10F12000A114B10429F0C6010197D5018D939C93D8
:10F13000CB01BA010E94BB6F6B017C01CE018370D1
:10F1400090708330910521F4F7FAF094F7F8F09479
:10F15000C701B60120E030E040E050E00E944F6F70
:10F16000882309F445C097FE07C0909481949108C4
:10F170009394C3E0D0E102C0CBEEDFE098EE692EBD
:10F180009FEF792E6C0E7D1E20E2A22EB12C0FC0B7
:10F19000FE010591159125913491C701B601A90190
:10F1A00098010E946D706B017C018A189B088A147B
:10F1B0009B0474F72497B594A794C615D705B9F79F
:10F1C000C601D7012A2F220F2B2F221F2F3F51F0CC
:10F1D000BC01CD0120E030E040E050E00E944F6FE4
:10F1E000882331F482E290E090933A2D8093392D78
:10F1F0003C2D2D2D9E2D8F2D06C08FEF04C030E0AD
:10F2000020E090EC8FE7B901AC01872F922FA52F5A
:10F21000B42FBC01CD01DF91CF911F910F91FF90D1
:10F22000EF90DF90CF90BF90AF909F908F907F90A6
:10F230006F900895992788270895FB01DC014150BC
:10F24000504088F08D9181341CF08B350CF4805E39
:10F25000659161341CF06B350CF4605E861B6111A6
:0EF2600071F3990B0895881BFCCFF894FFCF33
:10F26E00263A202573205B414444523D252D642EC1
:10F27E00252D64205345513D252D6420525353496D
:10F28E003D252D75204C51493D252D75204452505C
:10F29E003D252D642E253032645D0A00523D252D0C
:10F2AE0075204C3D252D7520533D252D6420005491
:10F2BE00696D656F757420414444523D252D642E51
:10F2CE00252D64205345513D252D6420525353491D
:10F2DE003D252D75204C51493D252D750A0028459B
:10F2EE007874507772290000413A202564202564F5
:10F2FE00202564200A00433A202564202564202519
:10F30E0064200A007374617475733D307825303251
:10F31E00780A2000312E30204669726D7761726551
:10F32E00205665722E20332E3520323031332D305B
:10F33E00312D303200656570726F6D006F6E006F2B
:10F34E00666600666F7263655F69646C650064650E
:10F35E006570004F6E006131007265736574006EEA
:10F36E006F6E6500613200765F696E0031003200AB
:10F37E00330034006175746F00666C7573680041FC
:10F38E004444523D252D642E252D64205345513D78
:10F39E00252D6420525353493D252D75204C51493E
:10F3AE003D252D750A00707772733D25730A007422
:10F3BE0072696D0043683D252D6420547850777234
:10F3CE003D252D640A004572726F72205458204CF0
:10F3DE00656E6774683D25640A0049443D0025301A
:10F3EE003278002050533D25640020543D252D36A3
:10F3FE002E3266002054313D252D362E32660020E9
:10F40E00545F4D43553D252D352E31660020565FF8
:10F41E004D43553D252D342E3266002050303D256E
:10F42E002D6C58002050305F543D252D372E3366FD
:10F43E00002050313D252D6C58002050315F543D39
:10F44E00252D372E3366002055503D252D6C580046
:10F45E002052483D252D342E31660020565F494EF0
:10F46E003D252D352E32660020565F41313D252D2E
:10F47E00352E32660020565F41323D252D352E3217
:10F48E00660020503D252D6C64002050413D252DF9
:10F49E00372E326600263A2025730A005458207003
:10F4AE006B74206C656E203D2025640A0025303279
:10F4BE0058006C656E3D25640A00D904C304AB0484
:10F4CE0077048F040000506572696F646963207061
:10F4DE00726F6365737300000066046815000000A8
:10F4EE0000536C6565702070726F636573730000F6
:10F4FE00008104980F0000000062726F6164636106
:10F50E0073742070726F636573730000009904FE4C
:10F51E003000000000737464696E2070726F636552
:10F52E007373000000B504AA0E00000000636D6442
:10F53E002070726F63657373000000CD043D300060
:10F54E000000000F0A003C00130A616263646566E6
:10F55E006768696A6B6C6D6E6F7020090D00FA0436
:10F56E001A22FFCC3B22FFCC3BED478A3C01001018
:10F57E00001D004000C706070740080000000019E4
:10F58E00380D381810000000004576656E74207432
:10F59E00696D65720000002905013C000000004302
:10F5AE0074696D65722070726F636573730000000D
:10F5BE003F05373D00000000020306070A0B0E0F41
:10F5CE002843292032303132204865726A756C66C4
:10F5DE000055747665636B6C696E67202020202061
:10F5EE002000436F6E74696B6920322E3500C600A1
:10F5FE00C500C400C100C200000000CE00CD00CC8A
:10F60E0000C900CA00000000000000020000000057
:10F61E00E24A0000000052463233302064726976AE
:10F62E006572000000B605924F00000000EF4D2CF1
:10F63E004DE14F2351824E854D904B8A4B7A4C6B48
:10F64E004D00010101010101010101010101010151
:10F65E00010052696D6500F20594525F526164615A
:10F66E0074612E6E756D20776179206F75742074BC
:10F67E00686572653A2025640A00CD53CC53D65581
:10F68E00FA562C550080C0E0F0F8FCFEFF6E756C4B
:10F69E006C6D6163002D06A6578B57915797579D3A
:10F6AE0057A357736963736C6F776D61630043067D
:10F6BE00B7581B58B057A757C158AD57BA000800D6
:10F6CE00C610CE10350002009E16A0165443502FC1
:10F6DE00495020737461636B0000006C06FE5A0083
:10F6EE00000000020800000000FFFFFFFF01000005
:02F6FE0000000A
:00000001FF
